:020000040800F2
:1000000000000120B5740008EB330008ED33000850
:10001000EF330008F1330008F3330008000000005C
:10002000000000000000000000000000F5330008A0
:10003000F733000800000000F9330008FB33000824
:100040000575000805750008FD33000805750008F2
:100050000575000805750008093400081934000802
:1000600005750008293400080575000831340008BA
:100070003D3400084934000805750008057500087E
:100080005534000859340008057500080575000846
:1000900000000000057500086534000805750008BB
:1000A0000575000805750008057500080575000848
:1000B0000575000805750008057500080575000838
:1000C0000575000805750008693400080575000805
:1000D00005750008753400080575000805750008E9
:1000E00005750008057500088134000805750008CD
:1000F00005750008000000000000000005750008FC
:1001000005750008057500088D34000805750008A0
:1001100005750008057500080575000805750008D7
:1001200005750008057500080575000805750008C7
:080130000575000805750008C3
:1001400010B5054C237833B9044B13B10448AFF311
:1001500000800123237010BDB007002000000000C4
:10016000B419030808B5034B1BB103490348AFF3A7
:10017000008008BD00000000B4070020B419030887
:1001800014214160704714207047406A7047000096
:1001900081010008870100088B010008A101000807
:1001A00010B5044604F1100000F05CFCC4F8F8003F
:1001B0000148C4F87C0110BD90010008F8B5E6B014
:1001C00004460D4616461F460A4906A800F0CAFE18
:1001D00070996F9A05910492009733466E996D9AC3
:1001E000039102922A466C990191214600F060F831
:1001F00067B0F0BD9C010008F8B5E6B004460D46B6
:1002000016461F46094906A800F0ACFE6F996E9A83
:100210000491039200976D996C9A02910192334672
:100220002A46214600F087F867B0F0BD9C0100081F
:1002300038B500281CBF01680029184A23D1184B83
:100240001C684FF6F0710C404CF24025AC421FBFC9
:100250001B6819404CF27024A14212D1114D29683B
:1002600079B911490B68C3F30B03B3F58A6F1FBF4C
:100270000968C1F30B0140F28343994204BF012195
:10028000117028B905E0094B994204BF0121117092
:100290004068BDE8324002F073BC00BFCC070020CC
:1002A00000ED00E0002004E00010005C0000374892
:1002B0002DE9F04104460D46216816464A681F465E
:1002C00090478046B8F5403F2ED122680A9993683E
:1002D000204698478046B8F5403F25D12368089AC4
:1002E0000799D3F80CC02046E0478046B8F5403F58
:1002F0001AD12368069A39461F692046B8478046B6
:10030000B8F5403F10D1236829465D693246204642
:10031000A8478046B8F5403F06D123680B9A099953
:100320009D692046A847804621680A682046904774
:100330004046BDE8F0812DE9F04104460D462168B4
:1003400016464A681F4690478046B8F5403F2ED172
:1003500022680A999368204698478046B8F5403F3E
:1003600025D12368089A0799D3F80CC02046E047A6
:100370008046B8F5403F1AD12368069A39461F696E
:100380002046B8478046B8F5403F10D1236829463B
:100390005D6932462046A8478046B8F5403F06D101
:1003A00023680999DD6900222046A8478046216814
:1003B0000A68204690474046BDE8F0814FF440303F
:1003C00070470000F0B50C4685B0114600281A466B
:1003D0001CBF0568002D0B4B11D082B104B971B957
:1003E0000D9860B10F9E0E9F0A9B02900496039792
:1003F0000B980C9E009001962046A847034618468D
:1004000005B0F0BD020003002DE9F04F0646D0B064
:100410000868F56DD6F860E0726EB76EF36E00BADC
:1004200000906C46486800BA60600DF1400888682A
:1004300000BAA060C86800BAE060086900BA20612C
:10044000486900BA6061886900BAA061C86900BAE9
:10045000E061086A00BA2062486A00BA6062886A8D
:1004600000BAA062C86A00BAE062086B00BA2063F2
:10047000486B00BA6063886B00BAA063C86B00BAAF
:10048000E063402058F80C1C58F820CC58F838ACE1
:100490008CEA010158F840CC8AEA01018CEA010992
:1004A0004FEAF979401E48F8049BEBD187EA020035
:1004B00000EA0E00784010EBF5610098DFF824C4E4
:1004C00041186144C81882EABE032B404FEAF0612C
:1004D00053405918636859186144CF194FEAB5035E
:1004E00083EABE01014081EABE0111EBF765A16814
:1004F0004D196544A91883EAB0023A404FEAF16504
:100500005A405519E26855194FEAB70282EAB00716
:1005100065440F4005EBBE0E97EAB00717EBFE658A
:1005200027697D194FEAB10782EA0701654401EAAC
:100530000E01EB18514011EBF36561694D194FEA5B
:10054000BE0187EA010E65440EEA030E15EBB0000A
:100550008EEA070E0EEBF065D4F818E0754465449A
:10056000AA1881EAB30505404FEAF26E4D40AE4449
:10057000E569AE44E64477444FEAB00080EAB30E42
:100580000EEA020E8EEAB30E0EEBF765D4F820E009
:1005900075446544691880EAB2053D404FEAF16E42
:1005A0004540AE44656AAE44E6440EEBB3034FEA01
:1005B000B70787EAB20E0EEA010E8EEAB20E0EEB14
:1005C000F365D4F828E075446544281887EAB10536
:1005D0001D404FEAF06E7D40AE44E56AAE44E6440D
:1005E0000EEBB2024FEAB30383EAB10E0EEA000E3D
:1005F0008EEAB10E0EEBF265D4F830E07544654436
:10060000EF1983EAB00515404FEAF76E5D40AE443E
:10061000656BAE44E6440EEBB1014FEAB20282EAEA
:10062000B00E0EEA070E8EEAB00E0EEBF165D4F8AE
:1006300038E075446544EB1882EAB7050D404FEA8F
:10064000F36E5540AE44E56BAE44E6440EEBB000AD
:100650004FEAB10181EAB70E0EEA030E8EEAB70E39
:100660000EEBF065D4F840E07544654481EAB30EC2
:10067000AA180EEA000E4FEAF2658EEA010E7544E2
:10068000DDF844E04FEAB000754480EAB30E6544FB
:100690000EEA020E15EBB7078EEAB30E0EEBF76506
:1006A000DDF848E04FEAB202754480EA020E654484
:1006B0000EEA070E69188EEA000E0EEBF165DDF802
:1006C0004CE07544654405EBB3034FEAB70E1427BD
:1006D0000DF1500CDFF810528EEA010B82EA0B0B81
:1006E0000BEBF36A5CF804BBDA44AA44504483EA97
:1006F000B10B4FEAF06A8EEA0B0BDA445CF804BBEC
:10070000DA44AA44524480EAB30B4FEAF26A8BEA15
:10071000B10BDA445CF804BBDA444FEAB000AA44F7
:1007200080EA020BD6448BEAB30B0BEBFE6A5CF853
:1007300004BBDA444FEAB202AA4482EA0E0B0AEB87
:10074000B10180EA0B0B0BEBF16A5CF804BBDA44F5
:100750007F1DAA44282F0AEBB3034FEABE0EBBD37A
:100760003C2F61D3502F4DD204EB870CC7F15407B7
:100770005E4CA7FB04A504465D4FA8088EEA010A5B
:1007800082EA0A0A5CF804BB0AEBF3655D447D1952
:100790002C1983EAB10A4FEAF4658EEA0A0A554435
:1007A0005CF804AB5CF804BB55447D19AA1884EAD4
:1007B000B30A4FEAF2658AEAB10A55445D444FEA4A
:1007C000B4047D1984EA020AAE448AEAB30A0AEB49
:1007D000FE655CF804AB55444FEAB2027D1982EA2B
:1007E0000E0A15EBB10184EA0A0A5CF804BB0AEBB5
:1007F000F1655D447D1915EBB303401E4FEABE0E53
:10080000BCD12046F46D1B19F365336EC9183166EF
:10081000716E71447166B36ED218B266F16E401893
:10082000F06650B0BDE8F08F4EEA010B0EEA010A07
:100830000BEA020B4BEA0A0A0AEBF36554F827A00D
:10084000DFF8B0C0554443EAB10B654403EAB10A8E
:100850000BEA0E0B28184BEA0A0A7F1C0AEBF0651C
:1008600054F827A0554440EAB30B654400EAB30AA4
:100870000BEAB10BAA184BEA0A0A7F1C0AEBF265D5
:1008800054F827A055444FEAB00040EA020B6544F3
:1008900000EA020A0BEAB30BAE444BEA0A0A7F1CD9
:1008A0000AEBFE6554F827A055444FEAB20242EA2B
:1008B0000E0B654402EA0E0A0BEA000B15EBB101C0
:1008C0004BEA0A0A7F1C0AEBF16554F827A055444D
:1008D0007F1C65443C2F05EBB3034FEABE0EA3D348
:1008E00040E700BF9979825AA1EBD96ECDCCCCCC30
:1008F000D6C162CADCBC1B8F00B581B00168074A53
:10090000914200D110B9064801B000BD7C212DF004
:1009100000FE4FF4003001B000BD00BF040A000823
:10092000030002002DE9F0410B4A92E8F85188B02B
:10093000694681E8F8510268084B9A4200D118B91B
:10094000074808B0BDE8F0811422083000F04FFBE2
:1009500008B0BDE8F08100BFE4090008040A0008FF
:1009600003000200152904D20268044B9A4200D108
:1009700008B903487047083000F048BB040A000873
:100980000300020010B481B013460268074CA24273
:1009900000D118B901B010BC0548704701B000F192
:1009A000240210BC083000F035BB00BF040A000868
:1009B0000300020010B481B013460268074CA24243
:1009C00000D118B901B010BC054870470A4601B003
:1009D00000F1240110BC083000F070BB040A0008CC
:1009E000030002000123456789ABCDEFFEDCBA9816
:1009F00076543210F0E1D2C3000000000000000085
:100A000000000000F9080008250900086509000831
:100A100085090008B509000809040008810F0008CD
:100A2000CD0F0008890F0008F0B5A3B004460B48AD
:100A300002900D4616461F46094B0822402104A885
:100A400000F0D1FA28980190009733462A462146B3
:100A500002A800F01BF823B0F0BD00BF040A000894
:100A6000180A000810B5040008BF002408D0054883
:100A7000054B20600822402104F1080000F0B3FA81
:100A8000204610BD040A0008180A00082DE9F041AC
:100A900004460E46216817464A681D469047804620
:100AA000B8F5003F19D12268069993682046984707
:100AB0008046B8F5003F10D123683146DE683A46DB
:100AC0002046B0478046B8F5003F06D12368079A14
:100AD00029461D692046A847804621680A682046A5
:100AE00090474046BDE8F08110B500F033FA4FF46E
:100AF000403400280EBF034C4FF4C0712DF009FDA7
:100B0000204610BD0200030010B5044600F022FA92
:100B100008B9054810BD0021A160D0F87C211168FA
:100B200088474FF4403010BD0200030070B5044602
:100B30000D4600F00FFA064E40B1D0F87C01416836
:100B40008847A84224BF65604FF44036304670BDE8
:100B5000020003002DE9FF4715000C4600D02CB120
:100B6000064600F0F7F95FEA000801D16448C3E0E7
:100B7000D8F8F80001684A689047B0F5003F17D1EF
:100B8000D8F87C118A68404690478146B9F1810FB8
:100B900080F09E80A94508F1FC0A17D2D8F8F80029
:100BA0000368D3F80CC02A462146E047B0F5003F61
:100BB00040F08E80D8F8F8000368D3F810C06A4679
:100BC0005146E047B0F5003F76D10AE0002004E04E
:100BD000215C0AF800100098401C00900098A84280
:100BE000F6D34FF0000C4749474A484B01AC0098F8
:100BF000844558D2D3E9007001ADC5E90070107882
:100C000000281ABF042086464FF0000E085854F8FA
:100C10000E5028443E4D05600127D0F800E0876063
:100C2000019D4F681AF80C007D408EEA050585F09D
:100C3000040E65680F687D4085F0FC05754485F0FD
:100C4000A30568400AF80C000CF1010CCFE7D3E9CA
:100C5000004501A8C0E9004510782E4D002814BFBA
:100C60004FF0040E4FF0000E01A8744651F80EE04C
:100C70000459A6440127CEF80050DEF80040CEF813
:100C800008704D68019F40687D406C400D68684069
:100C900084F0040480F0FC00041984F057040AF87E
:100CA0000C400CF1010CCC45D1D3D8F8F800016808
:100CB0004A689047B0F5003F0AD1D8F8F8000368B9
:100CC000D3F80C804A465146C047B0F5003F01D0EA
:100CD000114811E0002006E05AF8201081F06A3136
:100CE0004AF82010401CB0EB990FF5D3B06840F0E3
:100CF0000100B0604FF4403004B0BDE8F08700BFA1
:100D000002000300EC5A0308CC0700202C0F000857
:100D1000ADBE4ED70DBE75A10100030038B50C461F
:100D2000017A1546CA0702D500F014F908B9084837
:100D300032BDD0F8F80003682146DC682A46A04797
:100D4000B0F5003F01D0034832BD4FF4403032BD12
:100D500002000300010003002DE9F84191B00546AF
:100D60000E461746402101A82DF0D3FB297AC8076B
:100D700004D5284600F0EEF8040002D1DFF8A48084
:100D80004BE0D4F8F800DFF8A0800368D3F810C077
:100D90006A4601A9E047B0F5003F3ED1D4F8F8001B
:100DA00001684A689047B0F5003F36D1D4F87C110D
:100DB0008A6820469047D4F8F830024618461B68E7
:100DC000D3F80CC004F1FC01E047B0F5003F24D19A
:100DD000D4F87C0141688847D4F8F83002461846B8
:100DE0001B68D3F80CC001A9E047B0F5003F14D14F
:100DF000D4F8F8000268696893689847B0F5003F36
:100E00000BD1D4F8F80003681C693A463146A04774
:100E1000B0F5003F08BF4FF44038404612B0BDE87F
:100E2000F08100BF02000300010003002DE9F8413A
:100E3000A5B0074688461646402115A82DF069FB47
:100E400000220492402105A82DF063FB387AC107E7
:100E50005ED5384600F07EF8050059D0D5F8F80088
:100E60002D4C0368D3F810C06A4605A9E047B0F5D9
:100E7000003F3CD1D5F8F80001684A689047B0F5CA
:100E8000003F34D1D5F87C118A6828469047D5F8C0
:100E9000F830024618461B68D3F80CC005F1FC0177
:100EA000E047B0F5003F22D1D5F87C014168884782
:100EB000D5F8F830024618461B68D3F80CC005A9CF
:100EC000E047B0F5003F12D1D5F8F8000268796824
:100ED00093689847B0F5003F09D1D5F8F80003684A
:100EE0001D6904AA15A9A847B0F5003F01D0204606
:100EF0000FE00A4B0A490B4A0396029101924046C1
:100F00001C68049B009415AA796800F0E5F900E0DC
:100F1000054826B0BDE8F08101000300F45A03083B
:100F2000936E030026C703000200030004B0010112
:100F300000170145E90A0008090B00082D0B0008FD
:100F4000BD030008550B00081D0D0008590D0008D1
:100F50002D0E00080168024A914218BF0020704718
:100F6000340F000810B5040008BF002404D0034863
:100F70002060204609688847204610BD340F0008CD
:100F800020225C302DF0C1BAF0B58468A30800229D
:100F900004F0030407E000F15C0555F8226035BA5F
:100FA00041F82250521C9A42F5D300220BE000F186
:100FB0005C0502EB830755F82360D500C5F11805E1
:100FC000EE40CE55521CA242F1D3F0BD30B5C468FC
:100FD00003690022E31AD5188C5C0544521C082AC8
:100FE0002C77F8D330BD0360C1600261704738B51B
:100FF000044615460022626023685A689047002024
:101000006061A061A5604FF4003032BD81604FF493
:10101000003070472DE9F84304462079D4F80C805D
:10102000450748BF244845D466691D46A8F101001C
:1010300000EAD60306EBC506B6EBC50F666102D221
:10104000A669761CA6611746A66906EB5576A661C9
:101050000E46E918884225D2A8EB03094A463146D4
:10106000F8182DF052FA2268136839460FE042460C
:1010700038462DF04AFA23681A68394620469047C8
:1010800007E0311811F00300F1D1226813682046FF
:101090009847484600EB0809A9F10101A942F0D39D
:1010A000002300E000202A1A3118F8182DF02DFA3C
:1010B0004FF40030BDE8F283040002002DE9FC4F3C
:1010C000024685B0D0681369DFF86CC1DFF86C8127
:1010D000A0EB030A506840F004005060002703A80A
:1010E00002900DF10C0ED8E9003403A8544DC0E96C
:1010F00000342878534D00280CBF00230423994660
:101100005CF803305EF80940234401261D601C682A
:101110009E60DCF80430039DDCF80090DEF804608B
:101120005D406540484C654089EA0606474C66408C
:101130007519474C6540D8E9006B03AC0028C4E939
:10114000006B0EBF002404200424029E5CF8000003
:10115000345920183F4C04600126046886600398C7
:10116000029E43406340384C7068634089EA000047
:10117000364C6040034438484340280018BF0120E3
:101180005B1E9B41042F2CBFC0B2D80F02F1140389
:1011900053F8200007F00303C3F10303DB00D8403A
:1011A0000DF807007F1C082F9DD315460C466A6971
:1011B000AB69E868D20842EA4372401E00EA0207BF
:1011C000002302409B420AD8524508D28020E055B5
:1011D0007F1C574516D2AAEB0701E01910E08020CA
:1011E000E05500E0E355E8687F1C8742FAD32A689F
:1011F000136828469847BAF1000F03D0514620469D
:101200002DF087F92A68069E059F9368694628464F
:1012100098472A68D2F8009021462846C8472B688C
:10122000DA683946284690470EB1A86830604FF416
:10123000003007B0BDE8F08FEC5A03085C120008DC
:10124000CC0700205FC5109304850012FC68017A6A
:10125000C0F524FF24AF33D426AF698B04B001015D
:1012600000170145F8B501240094002300240DE087
:10127000009D065D0F5D7E40F643761CF60F86F0FE
:10128000010635400095641C009DEB189442EFD395
:101290001846F2BDF8B5002301240094002A11E09D
:1012A000009C85188F1815F8016C17F8015C6E40CA
:1012B000F643761CF60F86F0010634400094009C3D
:1012C000E318521EECD11846F2BD0000651200086A
:1012D00095120008010000002DE9F84F1D46DDF8C9
:1012E00028900B9F0D9C4FF0FF3300930E469246C3
:1012F000D9F800B0804632465146D847834664B399
:10130000D9F8043032465146404698476FEA0B02FE
:10131000521C42EA0B0200996FEAD2735B1C19401F
:10132000C2430091521C024300996FEAD2735B1CC6
:101330001940009186F05531484087EA000181F05C
:101340005531216080F05531C943491C0843009A4A
:101350006FEAD070401C82430092D9F8080001283F
:1013600009D17540E943491C0D4300986FEAD572D5
:10137000521C90430AE0F11C85EA9102D243521CB0
:10138000154300986FEAD5735B1C984386F0AA3624
:10139000009086EA0B0686F0AA33F243DB430C98F2
:1013A000C2F3C0725B1C42EAD3720099D243521C52
:1013B00091430091774000998843009987F0AA37BC
:1013C0000F403843BDE8F28F00000000000000002D
:1013D00001F0FF01102A2BDB10F0070F08D010F8E6
:1013E000013B013A8B422DD010F0070F42B3F6D1EA
:1013F000F0B441EA012141EA014122F007047FF003
:1014000000070023F0E80256083C85EA010586EA59
:10141000010685FA47F5A3FA87F586FA47F6A5FA95
:1014200087F68EB9EED1F0BC01F0FF0102F00702A1
:1014300032B110F8013B013A83EA010313B1F8D14C
:101440000020704701387047002D06BF354603382D
:10145000073815F0010F07D1013015F4807F02BF66
:10146000013015F4C03F0130F0BC0138704700BFB7
:10147000034613F8012B002AFBD1181A01387047D4
:1014800081F0004102E000BF83F0004330B54FEA35
:1014900041044FEA430594EA050F08BF90EA020FA2
:1014A0001FBF54EA000C55EA020C7FEA645C7FEA35
:1014B000655C00F0E2804FEA5454D4EB5555B8BF58
:1014C0006D420CDD2C4480EA020281EA030382EAC9
:1014D000000083EA010180EA020281EA0303362D5B
:1014E00088BF30BD11F0004F4FEA01314FF4801C2E
:1014F0004CEA113102D0404261EB410113F0004F40
:101500004FEA03334CEA133302D0524263EB4303F6
:1015100094EA050F00F0A780A4F10104D5F1200E94
:101520000DDB02FA0EFC22FA05F2801841F10001EF
:1015300003FA0EF2801843FA05F359410EE0A5F1C3
:1015400020050EF1200E012A03FA0EFC28BF4CF0F4
:10155000020C43FA05F3C01851EBE37101F00045AA
:1015600007D54FF0000EDCF1000C7EEB00006EEBB7
:101570000101B1F5801F1BD3B1F5001F0CD3490841
:101580005FEA30004FEA3C0C04F101044FEA445298
:1015900012F5800F80F09A80BCF1004F08BF5FEA1F
:1015A000500C50F1000041EB045141EA050130BDFF
:1015B0005FEA4C0C404141EB0101013C28BFB1F511
:1015C000801FE9D291F0000F04BF01460020B1FA5C
:1015D00081F308BF2033A3F10B03B3F120020CDA2F
:1015E0000C3208DD02F1140CC2F10C0201FA0CF00D
:1015F00021FA02F10CE002F11402D8BFC2F1200C72
:1016000001FA02F120FA0CFCDCBF41EA0C01904027
:10161000E41AA2BF01EB0451294330BD6FEA040470
:101620001F3C1CDA0C340EDC04F11404C4F120025B
:1016300020FA04F001FA02F340EA030021FA04F36D
:1016400045EA030130BDC4F10C04C4F1200220FAC4
:1016500002F001FA04F340EA0300294630BD21FA02
:1016600004F0294630BD94F0000F83F4801306BFC8
:1016700081F480110134013D4EE77FEA645C18BFBC
:101680007FEA655C29D094EA050F08BF90EA020F53
:1016900005D054EA000C04BF1946104630BD91EA4B
:1016A000030F1EBF0021002030BD5FEA545C05D14E
:1016B0004000494128BF41F0004130BD14F580048D
:1016C0003CBF01F5801130BD01F0004545F0FE4101
:1016D00041F470014FF0000030BD7FEA645C1ABF36
:1016E000194610467FEA655C1CBF0B46024650EA6D
:1016F000013406BF52EA033591EA030F41F4002199
:1017000030BD00BF90F0000F04BF0021704730B51E
:101710004FF4806404F132044FF000054FF00001F3
:1017200050E700BF90F0000F04BF0021704730B5B4
:101730004FF4806404F1320410F0004548BF404289
:101740004FF000013EE700BF42004FEAE2014FEADE
:1017500031014FEA02701FBF12F07F4393F07F4FB9
:1017600081F06051704732F07F4208BF704793F0BC
:101770007F4F04BF41F40021704730B54FF46074CF
:1017800001F0004521F000411CE700BF50EA0102D2
:1017900008BF704730B54FF000050AE050EA01027B
:1017A00008BF704730B511F0004502D5404261EBEB
:1017B00041014FF4806404F132045FEA915C3FF42C
:1017C000D8AE4FF003025FEADC0C18BF03325FEAC9
:1017D000DC0C18BF033202EBDC02C2F1200300FA7A
:1017E00003FC20FA02F001FA03FE40EA0E0021FA9F
:1017F00002F11444BDE600BF70B54FF0FF0C4CF48D
:10180000E06C1CEA11541DBF1CEA135594EA0C0F3E
:1018100095EA0C0F00F0DEF82C4481EA030621EA79
:101820004C5123EA4C5350EA013518BF52EA0335B4
:1018300041F4801143F4801338D0A0FB02CE4FF066
:101840000005E1FB02E506F00042E0FB03E54FF096
:101850000006E1FB03569CF0000F18BF4EF0010E8E
:10186000A4F1FF04B6F5007F64F5407404D25FEA8A
:101870004E0E6D4146EB060642EAC62141EA55513D
:101880004FEAC52040EA5E504FEACE2EB4F1FD0C7F
:1018900088BFBCF5E06F1ED8BEF1004F08BF5FEAFD
:1018A000500E50F1000041EB045170BD06F00046AF
:1018B00046EA010140EA020081EA0301B4EB5C045C
:1018C000C2BFD4EB0C0541EA045170BD41F4801154
:1018D0004FF0000E013C00F3AB8014F1360FDEBF79
:1018E000002001F0004170BDC4F10004203C35DA55
:1018F0000C341BDC04F11404C4F1200500FA05F3D8
:1019000020FA04F001FA05F240EA020001F0004278
:1019100021F0004110EBD37021FA04F642EB0601EE
:101920005EEA430E08BF20EAD37070BDC4F10C0418
:10193000C4F1200500FA04F320FA05F001FA04F2DC
:1019400040EA020001F0004110EBD37041F10001C8
:101950005EEA430E08BF20EAD37070BDC4F12005D3
:1019600000FA05F24EEA020E20FA04F301FA05F23B
:1019700043EA020321FA04F001F0004121FA04F2E3
:1019800020EA020000EBD3705EEA430E08BF20EAB3
:10199000D37070BD94F0000F0FD101F000464000ED
:1019A00041EB010111F4801F08BF013CF7D041EA6F
:1019B000060195F0000F18BF704703F00046520073
:1019C00043EB030313F4801F08BF013DF7D043EA44
:1019D0000603704794EA0C0F0CEA135518BF95EAFA
:1019E0000C0F0CD050EA410618BF52EA4306D1D181
:1019F00081EA030101F000414FF0000070BD50EAA0
:101A0000410606BF1046194652EA430619D094EA29
:101A10000C0F02D150EA013613D195EA0C0F05D113
:101A200052EA03361CBF104619460AD181EA030167
:101A300001F0004141F0FE4141F470014FF000001F
:101A400070BD41F0FE4141F4780170BD70B54FF0BA
:101A5000FF0C4CF4E06C1CEA11541DBF1CEA13553A
:101A600094EA0C0F95EA0C0F00F0A7F8A4EB05041C
:101A700081EA030E52EA03354FEA013100F0888013
:101A80004FEA03334FF0805545EA131343EA1263DC
:101A90004FEA022245EA111545EA10654FEA002691
:101AA0000EF000419D4208BF964244F1FD0404F54A
:101AB000407402D25B084FEA3202B61A65EB0305A6
:101AC0005B084FEA32024FF480104FF4002CB6EB63
:101AD000020E75EB030E22BFB61A754640EA0C00E3
:101AE0005B084FEA3202B6EB020E75EB030E22BF23
:101AF000B61A754640EA5C005B084FEA3202B6EB64
:101B0000020E75EB030E22BFB61A754640EA9C0022
:101B10005B084FEA3202B6EB020E75EB030E22BFF2
:101B2000B61A754640EADC0055EA060E18D04FEAB0
:101B3000051545EA16754FEA06164FEAC30343EA50
:101B400052734FEAC2025FEA1C1CC0D111F4801F1D
:101B50000BD141EA00014FF000004FF0004CB6E716
:101B600011F4801F04BF01430020B4F1FD0C88BFB5
:101B7000BCF5E06F3FF6AFAEB5EB030C04BFB6EBC0
:101B8000020C5FEA500C50F1000041EB045170BDB3
:101B90000EF0004E4EEA113114EB5C04C2BFD4EBE0
:101BA0000C0541EA045170BD41F480114FF0000E64
:101BB000013C90E645EA060E8DE60CEA135594EAE0
:101BC0000C0F08BF95EA0C0F3FF43BAF94EA0C0FE3
:101BD0000AD150EA01347FF434AF95EA0C0F7FF458
:101BE00025AF104619462CE795EA0C0F06D152EAAC
:101BF00003353FF4FDAE1046194622E750EA410690
:101C000018BF52EA43067FF4C5AE50EA41047FF4A0
:101C10000DAF52EA43057FF4EBAE12E74FF0FF3C05
:101C200006E000BF4FF0010C02E000BF4FF0010CD6
:101C30004DF804CD4FEA410C7FEA6C5C4FEA430C4F
:101C400018BF7FEA6C5C1BD001B050EA410C0CBF9E
:101C500052EA430C91EA030F02BF90EA020F002000
:101C6000704710F1000F91EA030F58BF994208BF67
:101C700090422CBFD8176FEAE37040F00100704724
:101C80004FEA410C7FEA6C5C02D150EA013C07D17B
:101C90004FEA430C7FEA6C5CD6D152EA033CD3D0C6
:101CA0005DF8040B704700BF8446104662468C46C0
:101CB0001946634600E000BF01B5FFF7B7FF0028F3
:101CC00048BF10F1000F01BD4DF808EDFFF7F4FF1C
:101CD0000CBF012000205DF808FB00BF4DF808EDA7
:101CE000FFF7EAFF34BF012000205DF808FB00BFCA
:101CF0004DF808EDFFF7E0FF94BF012000205DF8EC
:101D000008FB00BF4DF808EDFFF7CEFF94BF0120A0
:101D100000205DF808FB00BF4DF808EDFFF7C4FF99
:101D200034BF012000205DF808FB00BF4FEA410CE2
:101D30007FEA6C5C02D150EA013C0AD14FEA430CC5
:101D40007FEA6C5C02D152EA033C02D14FF0000002
:101D500070474FF0010070474FEA410212F5001240
:101D600015D211D56FF47873B3EB625212D94FEAE2
:101D7000C12343F0004343EA505311F0004F23FACC
:101D800002F018BF404270474FF00000704750EA21
:101D9000013005D111F0004008BF6FF000407047DE
:101DA0004FF00000704700BF4FEA4102B2F1E0433C
:101DB00024BFB3F5001CDCF1FE5C0DD901F0004C32
:101DC0004FEAC0024CEA5070B2F1004F40EB830082
:101DD00008BF20F00100704711F0804F21D113F1AE
:101DE0003872BCBF01F00040704741F480114FEAE7
:101DF0005252C2F11802C2F1200C10FA0CF320FA70
:101E000002F018BF40F001004FEAC1234FEAD3238C
:101E100003FA0CFC40EA0C0023FA02F34FEA4303F6
:101E2000CCE77FEA625307D150EA01331EBF4FF07F
:101E3000FE4040F44000704701F0004040F0FE409A
:101E400040F40000704700BF80F0004002E000BF97
:101E500081F0004142001FBF5FEA410392EA030F95
:101E60007FEA226C7FEA236C6AD04FEA1262D2EBDF
:101E70001363C1BFD218414048404140B8BF5B42E4
:101E8000192B88BF704710F0004F40F4000020F07D
:101E90007F4018BF404211F0004F41F4000121F093
:101EA0007F4118BF494292EA030F3FD0A2F10102DD
:101EB00041FA03FC10EB0C00C3F1200301FA03F11B
:101EC00000F0004302D5494260EB4000B0F5000F3E
:101ED00013D3B0F1807F06D340084FEA310102F1FD
:101EE0000102FE2A51D2B1F1004F40EBC25008BFAF
:101EF00020F0010040EA03007047490040EB000079
:101F0000013A28BFB0F5000FEDD2B0FA80FCACF179
:101F1000080CB2EB0C0200FA0CF0AABF00EBC250A6
:101F200052421843BCBFD0401843704792F0000F94
:101F300081F4000106BF80F400000132013BB5E7E7
:101F40004FEA41037FEA226C18BF7FEA236C21D05D
:101F500092EA030F04D092F0000F08BF08467047C2
:101F600090EA010F1CBF0020704712F07F4F04D190
:101F7000400028BF40F00040704712F100723CBFA3
:101F800000F50000704700F0004343F0FE4040F4CD
:101F9000000070477FEA226216BF08467FEA23638B
:101FA0000146420206BF5FEA412390EA010F40F476
:101FB000800070474FF0000304E000BF10F00043C2
:101FC00048BF40425FEA000C08BF704743F09643A9
:101FD00001464FF000001CE050EA010208BF7047C4
:101FE0004FF000030AE000BF50EA010208BF70474B
:101FF00011F0004302D5404261EB41015FEA010C60
:1020000002BF84460146002043F0B64308BFA3F157
:102010008053A3F50003BCFA8CF2083AA3EBC25339
:1020200010DB01FA02FC634400FA02FCC2F1200258
:10203000BCF1004F20FA02F243EB020008BF20F08F
:102040000100704702F1200201FA02FCC2F12002F5
:1020500050EA4C0021FA02F243EB020008BF20EAEA
:10206000DC7070474FF0FF0C1CEAD0521EBF1CEA18
:10207000D15392EA0C0F93EA0C0F6FD01A4480EA06
:10208000010C400218BF5FEA41211ED04FF00063EF
:1020900043EA501043EA5111A0FB01310CF000401B
:1020A000B1F5000F3EBF490041EAD3715B0040EA41
:1020B000010062F17F02FD2A1DD8B3F1004F40EB11
:1020C000C25008BF20F00100704790F0000F0CF0E4
:1020D000004C08BF49024CEA502040EA51207F3AA8
:1020E000C2BFD2F1FF0340EAC250704740F4000083
:1020F0004FF00003013A5DDC12F1190FDCBF00F074
:1021000000407047C2F10002410021FA02F1C2F121
:10211000200200FA02FC5FEA310040F1000053EABD
:102120004C0308BF20EADC70704792F0000F00F00B
:10213000004C02BF400010F4000F013AF9D040EA11
:102140000C0093F0000F01F0004C02BF490011F4A5
:10215000000F013BF9D041EA0C018FE70CEAD153A3
:1021600092EA0C0F18BF93EA0C0F0AD030F0004C23
:1021700018BF31F0004CD8D180EA010000F00040D7
:10218000704790F0000F17BF90F0004F084691F095
:10219000000F91F0004F14D092EA0C0F01D14202CF
:1021A0000FD193EA0C0F03D14B0218BF084608D198
:1021B00080EA010000F0004040F0FE4040F40000E2
:1021C000704740F0FE4040F4400070474FF0FF0C75
:1021D0001CEAD0521EBF1CEAD15392EA0C0F93EABC
:1021E0000C0F69D0A2EB030280EA010C49024FEA0E
:1021F000402037D04FF0805343EA111143EA1013C7
:102200000CF000408B4238BF5B0042F17D024FF47E
:10221000000C8B4224BF5B1A40EA0C00B3EB510F59
:1022200024BFA3EB510340EA5C00B3EB910F24BF42
:10223000A3EB910340EA9C00B3EBD10F24BFA3EBC7
:10224000D10340EADC001B0118BF5FEA1C1CE0D18F
:10225000FD2A3FF650AF8B4240EBC25008BF20F042
:10226000010070470CF0004C4CEA50207F32C2BF96
:10227000D2F1FF0340EAC250704740F400004FF033
:102280000003013A37E792F0000F00F0004C02BF64
:10229000400010F4000F013AF9D040EA0C0093F02E
:1022A000000F01F0004C02BF490011F4000F013B88
:1022B000F9D041EA0C0195E70CEAD15392EA0C0FF0
:1022C00008D142027FF47DAF93EA0C0F7FF470AF28
:1022D000084676E793EA0C0F04D14B023FF44CAF6B
:1022E00008466EE730F0004C18BF31F0004CCAD100
:1022F00030F000427FF45CAF31F000437FF43CAF3C
:102300005FE700BF4FF0FF3C06E000BF4FF0010C5D
:1023100002E000BF4FF0010C4DF804CD4FEA40023F
:102320004FEA41037FEA226C18BF7FEA236C11D089
:1023300001B052EA530C18BF90EA010F58BFB2EB3C
:10234000030088BFC81738BF6FEAE17018BF40F0BC
:10235000010070477FEA226C02D15FEA402C05D170
:102360007FEA236CE4D15FEA412CE1D05DF8040BF5
:10237000704700BF844608466146FFE70FB5FFF788
:10238000C9FF002848BF10F1000F0FBD4DF808ED40
:10239000FFF7F4FF0CBF012000205DF808FB00BF31
:1023A0004DF808EDFFF7EAFF34BF012000205DF88B
:1023B00008FB00BF4DF808EDFFF7E0FF94BF0120D8
:1023C00000205DF808FB00BF4DF808EDFFF7D2FFD5
:1023D00094BF012000205DF808FB00BF4DF808ED18
:1023E000FFF7C8FF34BF012000205DF808FB00BFE5
:1023F0004FEA40024FEA41037FEA226C02D15FEAD2
:10240000402C08D17FEA236C02D15FEA412C02D133
:102410004FF0000070474FF0010070474FEA400254
:10242000B2F1FE4F0FD34FF09E03B3EB12620DD902
:102430004FEA002343F0004310F0004F23FA02F06C
:1024400018BF404270474FF00000704712F1610F13
:1024500001D1420205D110F0004008BF6FF00040EA
:1024600070474FF00000704742000ED2B2F1FE4FAD
:102470000BD34FF09E03B3EB126209D44FEA002353
:1024800043F0004323FA02F070474FF0000070471A
:1024900012F1610F01D1420202D14FF0FF307047BB
:1024A0004FF00000704700BF53B94AB9002908BF78
:1024B00000281CBF4FF0FF314FF0FF3000F06AB929
:1024C000ADF1080C6DE904CE00F006F8DDF804E08B
:1024D000DDE9022304B070472DE9F047089D0C4662
:1024E000002B4ED194468C458646B2FA82F262D9D0
:1024F0004AB1C2F12003914020FA03F30CFA02FC26
:10250000194300FA02FE4FEA1C471FFA8CF6B1FB92
:10251000F7F44FEA1E4307FB141143EA014304FB9F
:1025200006F199420AD91CEB030304F1FF3080F055
:102530001281994240F20F81023C6344591A1FFAFA
:102540008EF3B1FBF7F007FB101143EA014300FBE8
:1025500006F69E420AD91CEB030300F1FF3180F01E
:10256000FC809E4240F2F980634402389B1B40EAA3
:10257000044000211DB1D3400022C5E90032BDE86E
:10258000F0878B4205D90DB1C5E90001002108464D
:10259000F5E7B3FA83F1002946D1A34202D3904272
:1025A000C0F0F080861A64EB03030120002DE6D012
:1025B000C5E90063E3E7002A40F09080A1EB0C043A
:1025C0004FEA1C481FFA8CF70121B4FBF8F64FEADA
:1025D0001E4308FB164443EA044307FB06F09842F7
:1025E00008D91CEB030306F1FF3402D2984200F233
:1025F000CD8026461C1A1FFA8EF3B4FBF8F008FBB8
:10260000104443EA044300FB07F79F4208D91CEB40
:10261000030300F1FF3402D29F4200F2B080204653
:10262000DB1B40EA0640A5E7C1F120068B4022FAF9
:1026300006F71F4320FA06FC04FA01F343EA0C03F1
:10264000F44000FA01F8380C4FEA1349B4FBF0FEED
:102650001FFA87FC00FB1E4449EA04440EFB0CF9F8
:10266000A14502FA01F20AD93C190EF1FF3A80F0B5
:102670008480A14540F28180AEF1020E3C44A4EB7F
:1026800009041FFA83F9B4FBF0F300FB134449EA91
:10269000044403FB0CFCA44507D93C1903F1FF30AB
:1026A00067D2A44565D9023B3C4443EA0E40A0FBF7
:1026B0000293A4EB0C049C42CE469C4651D34ED0D0
:1026C00055B1B8EB0E0364EB0C0404FA06F6CB40EC
:1026D0001E43CC40C5E90064002150E7C2F120034D
:1026E00020FA03F10CFA02FC24FA03F394400C43A1
:1026F0004FEA1C4800FA02FE1FFA8CF7B3FBF8F011
:1027000008FB1031230C43EA014300FB07F1994217
:1027100008D91CEB030300F1FF362CD299422AD9C9
:10272000023863445B1AA4B2B3FBF8F108FB11331F
:1027300044EA034401FB07F3A34208D91CEB040459
:1027400001F1FF3613D2A34211D902396444E41ACD
:1027500041EA004139E70446F0E6084606E7C84585
:10276000AED2B9EB020E63EB070C0138A8E7314695
:10277000EDE7034699E73046D4E7D6467FE7634462
:1027800002384DE70646234608460FE7023E6344FB
:1027900030E700BF704700BF00487047001BB74BD1
:1027A00070B50C4601F024FA104E0546082130465B
:1027B00005F0A4FF012804D001F01AFA431BA3423C
:1027C00007D30821094805F099FF431E5842584194
:1027D00070BD72B60821304605F090FF012800D088
:1027E00030BF62B6BFF36F8FE0E700BF0004004860
:1027F00008B5002210214FF0904005F085FF0548F4
:102800000022202105F080FFBDE80840022001F0F1
:10281000F7B900BF0004004810B50C4C012210218C
:10282000204605F071FF052001F0EAF9204601225B
:10283000202105F069FF4FF090400122102105F0A2
:1028400063FFBDE81040022001F0DAB9000400483F
:1028500070B54FF090400C46164610210022144DE2
:1028600005F052FF00232B701248B3B222462146D6
:1028700007F03EF9D8B901F0BBF941F287360446BA
:102880002B783BB1BDE87040012210214FF0904001
:1028900005F03ABF01F0ACF9031BB342F2D872B6AF
:1028A0002B7803B930BF62B6BFF36F8FE8E770BD16
:1028B000CD07002030090020014B01221A7070471B
:1028C000CD07002000487047F85A030813B5114B94
:1028D0000446186800909B88ADF804300120FFF78B
:1028E0009BFF062269460120FFF7B2FF0120FFF798
:1028F0007FFF9DF80430112B08D19DF80520122A86
:1029000004D101202370627002B010BD00231A466A
:102910001846F7E7D01903080CB4F0B5ADB032ABE8
:1029200006AF53F8042B059305460E46384696210C
:102930002BF03EFD9528C1BF42F62E63ADF8AA30BC
:102940002E23ADF8AC3000F037F83C24042D4FF4C2
:102950007A7E1449B0FBFEFCB0FBF1F14EF6602329
:10296000B0FBF3F3B3FBF4F204FB1232BCFBF4F361
:1029700004FB13C30EFB1C049ABF0B48405D3F20B1
:10298000CDE90040CDE9026708482BF091FC084BE7
:102990001B6898682BF0B6FB2DB0BDE8F04002B084
:1029A000704700BF80EE3600565B0308345B0308B7
:1029B000D805002001F024B901F01AB91348144ACF
:1029C00008B54FF00043C0E9002304224261012210
:1029D0000023C2614FF480510722C0E90233C0E9ED
:1029E0000933C0E90C1203610383837680F8203039
:1029F00080F82C30826380F83C30C36404F0D6FD4C
:102A000018B1BDE8084000F097BB08BDD007002012
:102A1000002401400268084B9A4282B00AD14FF06C
:102A2000B0431A6E42F400721A661B6E03F4007310
:102A30000193019B02B07047002401400268054BDE
:102A40009A4201BF4FF0B042136E23F40073136635
:102A5000704700BF0024014030B585B00024054612
:102A6000CDE901440394FFF7A9FF144805F032F9BA
:102A700008B100F061FB1148039401A9CDE90154AC
:102A800004F0F2FE08B100F057FB0C4805F04CF8DA
:102A900008B100F051FB4FF0FF31084804F086FE0A
:102AA000064805F0F9F8054804F0DAFE0446034844
:102AB00005F09CF8204605B030BD00BFD0070020CF
:102AC000014B024A1A607047D007002000240140E1
:102AD00008B50948FFF7C0FF68B1084BB3F8AA3042
:102AE0004FF6FF72934216BF40F6E442044B534345
:102AF000B3FBF0F398B208BD002000B40075FF1FCF
:102B0000D8084C0013B50023ADF80630FFF7E0FFFE
:102B100004461948FFF7A0FF184BB3F8C820B3F8D4
:102B2000A8108A4204FB00F018D040F6E443B0FB42
:102B3000F3F364205B1A4343521A93FBF2F31E3300
:102B40001BB2ADF80630BDF806305BB21B02ADF823
:102B50000630BDF8060000B202B010BD4FF47A7224
:102B600040F6FF73B0FBF3F35343A3F53923A3F50A
:102B70000C6340F6C412E0E7001000B00075FF1FC0
:102B80004FF0B04382B09A6A22F480529A629A6CF3
:102B900042F480529A649B6C03F480530193019B2E
:102BA000002002B070474FF0B04307B59A6C42F076
:102BB00004029A649A6C02F004020192019A9A6CDF
:102BC00042F001029A649B6C002203F0010311465B
:102BD00000930B20009B05F01BF90B2005F04AF930
:102BE000002211460C2005F013F90C2005F042F9E3
:102BF000002211460D2005F00BF90D2005F03AF9E1
:102C0000002202210F2005F003F90F2005F032F910
:102C100000221146102005F0FBF8102005F02AF9DB
:102C200000221146112005F0F3F8112003B05DF8E1
:102C300004EB05F01FB9000008B505F05FFB10B10B
:102C40006FF0040008BD064B9A6942F040429A6159
:102C50004CF2FA321A6105F063FB0028F2D0EFE77C
:102C600000400058F0B585B000230D46009306469D
:102C7000A8B3FFF7E1FF044670BB05F03FFB88BB3C
:102C80001A481B4A02230193D0F8E01506F1784355
:102C900002EA8121B3FBF1F701FB1733DB0A029350
:102CA000D0F8E00505F178410139314402EA80228B
:102CB000B1FBF2F002FB1011C3EBD12301336946E3
:102CC00001A8039305F0ACFB20B1022814BF6FF0FC
:102CD0000104012405F024FB204605B0F0BD6FF08F
:102CE0000504F9E76FF00404F6E700BF0070FF1F6A
:102CF00000FCFF03014B18600020704734080020DF
:102D00002DE9F04FB0F1006F89B006460F469046AE
:102D1000C0F0C080DFF89091644DD9F8E03505EA45
:102D2000832303F10063013B984200F2B380002942
:102D300000F0B38040EA02035B0740F0AE80FFF78B
:102D40007BFF044690BB05F0D9FA002840F0A8802C
:102D5000D9F8E015009705EA812106F17842B2FB27
:102D6000F1F301FB132208F17843013B3344B3FB39
:102D7000F1F001FB1033DB0A01334FEAD22AA3EB57
:102D8000D222012A039388BFC6F30A050AF58037C9
:102D9000C6F108038CBFC5F500654546FF02B34682
:102DA0000693039B9A4505D305F0BAFA204609B06D
:102DB000BDE8F08FA6F10803069A1A4495421CD884
:102DC000009B04950193CDF814B04FF00009059BCA
:102DD00009EB0301049B99453DD3009BAB442B4475
:102DE000A8EB0505B5F5006F009328BF4FF400650B
:102DF0000AF1010A07F50067D3E753F8081F5A687C
:102E0000B2F1FF3F08BFB1F1FF3FD5D0284B1868A2
:102E100010B96FF00504C7E727B14FF400623946D7
:102E200011F08AFDDFF888900099D9F80030CBF3D3
:102E30000A001844AAB211F07FFD4FF40061384631
:102E4000FFF710FF00BBD9F8003001934FF4006387
:102E500005970493B9E7019B07914B440293012026
:102E6000D3E9002305F096FA88B90799019BD1E9C7
:102E7000000259F80310029B5B689A4208BF88421F
:102E800005D109F10809A2E76FF001048CE76FF0A2
:102E9000030489E74FF0FF3488E76FF0050485E706
:102EA0006FF0040482E700BF0070FF1F00FCFF0307
:102EB00034080020B1F1006F70B510D30B4BD3F87C
:102EC000E0650B4B03EA862303F10063013B994263
:102ED00005D838B192B211F02FFD002070BD4FF02F
:102EE000FF30FBE76FF00500F8E700BF0070FF1F41
:102EF00000FCFF03B0F1006F10B40DD3084BD3F802
:102F0000E045084B03EA842303F10063013B984248
:102F100002D810BCFFF7A6BE4FF0FF3010BC7047C0
:102F20000070FF1F00FCFF034FF0B04382B0DA6C6B
:102F30000243DA64DB6C03400193019B02B07047EB
:102F40002DE9F04186B01422002101A82BF04EFAA1
:102F50000220464EFFF7E8FF0420FFF7E5FF0120BF
:102F6000FFF7E2FF04213046002205F0CDFB0022EE
:102F700010214FF0904005F0C7FB042300240125E9
:102F800002270DEB03013046CDE901354FF0100863
:102F9000CDE9034705F092FA01A93046CDE9018554
:102FA000CDE9037405F08AFA202301A93046CDE962
:102FB0000135CDE9037405F081FA01A94FF0904085
:102FC000CDE90185CDE9034405F078FA08224FF4F4
:102FD000881301A93046CDE901234FF00308CDE95C
:102FE000034705F06BFA4FF4441301A94FF09040EA
:102FF000CDE90183CDE9035705F060FA4FF4405362
:1030000001A93046CDE90135CDE9034805F056FA6E
:103010004FF404134021CDE901131548039501A98C
:1030200005F04CFA22460F21062004F0F1FE06209E
:1030300004F020FF22460F21072004F0E9FE0720BC
:1030400004F018FF22462146092004F0E1FE092081
:1030500004F010FF22462146092004F0D9FE092081
:1030600004F008FF06B0BDE8F08100BF000400488E
:103070000008004800B59BB04822002108A82BF0AA
:10308000B5F91822002102A82BF0B0F905F056FB83
:103090004FF0B0420120D2F8903023F01803C2F86C
:1030A0009030D2F8003423F4C06343F40073C2F8C4
:1030B0000034D2F8003403F4C0630193019B24234D
:1030C000089381230B930023CDE91003B02208A8B5
:1030D000CDE9122305F0AAFC08B172B6FEE74F2332
:1030E000CDE90230CDE90400CDE90600022102A8B5
:1030F00005F036FF08B172B6FEE71BB05DF804FBC1
:1031000008B504F001FAFFF7B5FFFFF719FFFFF765
:103110004AFD00F0F5FF00F0A5FE00F087F8054835
:103120000122042105F0F0FA02F02CFC02F031FC3F
:10313000FCE700BF0004004872B6FEE700B58DB0A2
:103140002C22002101A82BF051F91748174B0360DE
:103150001F2383604FF080420023C0E90433C0E99D
:10316000072383614FF48073436206F09FF908B12F
:10317000FFF7E2FF0C4806F0C5FA08B1FFF7DCFFE5
:103180004FF0005300220793074808924FF48073D2
:1031900001A9029206920B9306F0E8F908B1FFF735
:1031A000CBFF0DB05DF804FB38080020002800407C
:1031B00010B5044690B03822002102A82BF016F971
:1031C0002268194B9A422CD14FF48033029302A803
:1031D0004FF480730F9305F0E7FF08B1FFF7ACFFE2
:1031E0004FF0B0430220D3F8902042F40042C3F8DD
:1031F00090209A6D42F480629A659B6D002203F4E0
:10320000806311460193019B04F002FE022004F04A
:1032100031FE00222A20114604F0FAFD2A2004F093
:1032200029FE10B010BD00BF002800401148124A0E
:1032300008B54FF48273C0E9002300234FF4E06225
:10324000C0E902324FF400712822C0E906120722B9
:10325000C0E90433C0E90833C0E90B2383620823C3
:10326000436306F0BFFB18B1BDE80840FFF764BF39
:1032700008BD00BF3009002000300140F0B5054610
:1032800089B01422002103A82BF0B0F82A68374B2C
:103290009A4269D14FF0B04302261A6E42F480522E
:1032A0001A661A6E02F480520292029ADA6C42F0A6
:1032B0000102DA64DA6C02F001020192019ADA6C1E
:1032C00042F00202DA64DB6C03F00203009305248F
:1032D000009B0327D02303A94FF09040CDE903368C
:1032E000CDE9067405F0EAF82023CDE903364FF066
:1032F0009040002603A90794CDE905671C4C05F012
:10330000DDF81C4826620723C4E900038023204619
:10331000C4E90266C4E90436C4E9066604F00AFE9C
:1033200008B1FFF709FF144AAC65A562134C0823E6
:10333000C4E900231021002380222046C4E902139F
:10334000C4E90423C4E90633236204F0F3FD08B1A1
:10335000FFF7F2FE002222206C651146A56204F000
:1033600057FD222004F086FD09B0F0BD0030014079
:10337000D00800201C0002403000024070080020ED
:103380007047000008B504F0D5F8044B0120C3F8DD
:103390008800BDE8084005F029BA00BF00040058C5
:1033A00008B504F0CEF800F0BBFFFFF7C9FDFFF74A
:1033B000FAFB00F057FDBDE80840FFF737BF08B53E
:1033C00004F0BFF8FFF7BCFDFFF7EDFBBDE80840D8
:1033D000FFF72CBF08B504F0ADF8BDE808400121A7
:1033E000002005F0B3B970477047FEE7FEE7FEE73F
:1033F000FEE7FEE77047704770477047014806F0E8
:10340000A7B900BF38080020024B0120187005F052
:1034100089B900BFF2180020024B012202201A7065
:1034200005F080B9F1180020082005F07BB90000F4
:10343000014804F0F5BE00BF9C0D0020014804F0D7
:10344000EFBE00BFD0080020014804F0E9BE00BF75
:103450007008002070470000014804F0E1BE00BF82
:10346000500E002070470000014806F02FBD00BF3D
:1034700030090020014807F067BE00BFB00E0020F1
:10348000014805F099BF00BF38080020014806F048
:10349000AEBF00BF880D00202DE9F04389B0804603
:1034A0000020109E0790894615461F46FCF7C0FE77
:1034B000F0B9104CCDE90090CDE9020407AB0E48FD
:1034C0000593142304933A46434629460068FCF7C3
:1034D00079FF2346324604F1140153F8044B42F8B5
:1034E000044B8B42F9D1079B337509B0BDE8F083DB
:1034F0000120FAE7AA090020E85A03087FB5124C18
:1035000000253C2302A86375CDE90255257500F01E
:1035100019FB042303AA009412210C48FFF7BCFFF7
:103520000B49142220462AF051FF0646B0FA80F0DB
:1035300040096075074B00902A462946022011F089
:10354000F5F8304604B070BD94090020925B030882
:103550005D1B0020745B0308034A044840F24B23C0
:10356000002107F067BC00BFC0090020FC0D00204F
:10357000132BF0B52DD81825102415FB0343194D36
:1035800000244FF0800C4CFA04F6A3F110073142EE
:1035900005EB470714BF4FF0240E4FF0140EA7F8A9
:1035A00006E0A3F10807304205EB470714BF4FF0D0
:1035B000240E4FF0140E0134324205EB4306A7F8F7
:1035C00006E00CBF14272427082CF78003F1010321
:1035D000D9D1054B1B781BB9BDE8F040FFF7BCBF44
:1035E000F0BD00BFC00900203819002010B500242C
:1035F0000022E3B2114610460134FFF7B9FF142C44
:10360000F6D110BD2DE9F0410646012090460F4647
:1036100000F0F6FA1C4A10254FF0800C2B460024CF
:103620004CFA04F1A3F110000F4202EB400014BF6A
:103630004FF0240E4FF0140EA0F806E0A3F108009E
:103640000E4202EB400014BF4FF0240E4FF0140E58
:10365000013418EA010F02EB4301A0F806E00CBFA9
:1036600014202420082CC88003F10103D8D1183578
:10367000B5F5F87FD2D1054B1B781BB9BDE8F041F9
:10368000FFF76ABFBDE8F081C009002038190020AB
:10369000002238B505460C4610461146FFF7B2FF2A
:1036A000082D30D8DFE805F005080C13171B1E2184
:1036B00023000022114601E000222146104602E0CC
:1036C000002211462046BDE83840FFF79BBF224646
:1036D00000210020F7E7002221462046F3E722469A
:1036E0000021EBE722462146F3E72246E2E7084DB8
:1036F000297849B1002211462046FFF783FF2B7835
:1037000083F001032B7038BD22460846F5E700BF61
:10371000BE090020024B1878024B1978FFF7B8BF9A
:1037200005000020000000207FB502AC204611F00B
:103730005FFA94E80300834C834D2378012B85E8DE
:10374000030009D081490B7833B1814A13781BB14A
:10375000804B1878052823D17F4B1A686AB92968ED
:1037600019607E49186808607D490A601B680093EB
:1037700011467C4B032010F0D9FF7B487B4D03782A
:10378000DBB20A2B32D8DFE813F02C004F005300D5
:10379000590062009900AC00B800C500C500C50022
:1037A0002078012806D1097821B9127812B91B783E
:1037B000052BE2D06A4B1A68002ADED1296819600D
:1037C0006B491868086064490A6018681B680968D2
:1037D0005B1ACDE900031146664B032010F0A6FFEB
:1037E000CBE7654B1B78DBB2644A13700378644EF9
:1037F000012B06D0634C227802F0FF03002A00F070
:103800008E805E4A002313702B703370FFF7EEFE3C
:10381000FFF780FF5C4A002313705C4A13705C4B17
:1038200001221A7004B070BD544B00221A70DDE7FB
:10383000584A1278012A08BF0123D5E7237813B923
:103840004E4B0122F2E72378012BCFD146E0444BC7
:10385000414A1B6812689B1A042BC7D923783C4A3B
:1038600053B93A4B1B78012B06D11378012BD9B2EF
:1038700002D1424B1970B9E72378012B05D0334BA5
:103880001B7813B11378002BB0D13C4B0221197077
:1038900041490C78032C03D104212970197008E0E8
:1038A0000C78012C01D10821F7E70C78022CE1B249
:1038B000F3D01278002A99D10822B7E7237833B9D8
:1038C000344B1B78012BDAB201D12C4BAEE72378B5
:1038D000012B03D02F4B1B78002B87D1274B0222C3
:1038E000A4E723781BB92D4B1B78002BA8D0237895
:1038F000012BF3D0294B1B78A6E723781BB9154B76
:103900001B78042B9CD02378012BE7D0114B1B781C
:10391000052B9AE70F4B1A78042AF8D190E7227802
:1039200012B9164B1B78DBB22B701D4B2878197817
:10393000FFF7AEFE237803B12B782B78DBB2337020
:1039400066E700BFD3180020D8180020F20000203E
:10395000F1000020D1180020EC180020E41800200D
:10396000E8180020A45B0308EE00002005000020FA
:10397000E0180020C75B03080400002006000020B8
:103980000100002038190020D6180020D51800208A
:10399000301900205C1B00205A0F0020D218002094
:1039A00000000020024803680021596307F0BCBAF8
:1039B000FC0D0020002270B50E4B1146022010F0C5
:1039C000B5FE01240A25294620461435FFF760FE7E
:1039D000EDB2322000F014F96E2DF4D10134E4B2CE
:1039E000092CEFD10022BDE87040034B11460220A4
:1039F00010F09CBEFE5B0308315C0308054808B567
:103A00000823036006F010FB18B1BDE80840FFF77B
:103A100093BB08BD880D00204FF0B04307B55A6E28
:103A200042F001025A665B6E002203F0010301932B
:103A300011463220019B04F0EBF9322003B05DF80F
:103A400004EB04F017BA00000CB407B5054A05AB47
:103A50001021019311F07AFA03B05DF804EB02B083
:103A6000704700BF675C030830B585B0044602A804
:103A70000D4611F097F8BDF90C30064A009310215D
:103A8000029B2046FFF7E0FF2046FDF7F1FC28806F
:103A900005B030BD675C03084FF0B04210B59368C5
:103AA00023F40043936011F005F9104B01241C70BE
:103AB00000F0ACF810F0D0FD0D4810F0E7FD0D4B14
:103AC0004FF400421A61022010F0E6FDFEF7F8FF05
:103AD00000F002F910F0DAFE2146204610F0F6FE62
:103AE00021462046BDE8104010F0DABE940D0020BB
:103AF000693A00080040005810F0FEBE08B5FEF715
:103B0000E7FF40F6B83398420CD8B0F5E16F0BD31D
:103B1000FE23A0F5E16058434FF49663B0FBF3F049
:103B2000C0B208BDFE20FCE70020FAE77FB568467A
:103B300000F0B6F80198FEF771FC00B207B05DF82E
:103B400004FB0000194A38B5D2F88035591C0446E8
:103B500019D103F0FDFC054603F006FD054403F012
:103B6000FDFC2B0EE3712B0CA3712B0A6371030E6A
:103B7000E370C0F30742C0F307232571C0B2A270FF
:103B80006370207038BD190AC3718171190C1B0E46
:103B900041710371D2F88435C370D2F88405C0F343
:103BA0000722C0F30743000EE9E700BF0070FF1FC4
:103BB00038B5094BD3F8803503600133054609D188
:103BC00003F0C6FC044603F0C9FC444003F0CCFCFF
:103BD00044402C6038BD00BF0070FF1F012102204F
:103BE00010F05EBE0021022010F05ABE0020704787
:103BF000024B187808B100F0BFB97047940D00204F
:103C000082B00190019802B000F052BAF0B5224A99
:103C1000224CD2F8903043F4804389B0C2F89030FF
:103C200003F0A8FC03F0AEFC03F0B4FC0123049302
:103C30000323069300254FF0B04305950795DA6CF2
:103C400042F00202DA64DA6C02F002020292029A94
:103C5000DA6C42F00202DA64DB6C03F002030193D7
:103C60004FF4805703A92046019B03974FF4005659
:103C700004F024FC03A92046039604F01FFC2A4606
:103C80003946204604F040FD2A463146204604F0DD
:103C90003BFD09B0F0BD00BF00080058000400481B
:103CA00010B50446FEF72EFF074BA36040F30F202C
:103CB000FEF784F9054B064A2360064B6060C4E9B1
:103CC0000323002010BD00BF0000484200007A44DA
:103CD0000D093E00AB03050000207047012070472E
:103CE00008B52AF0E5FB162303604FF0FF3008BD4E
:103CF00008B52AF0DDFB16230360FEE770B50D461C
:103D000014460E46731B9C4201DC204670BDAFF387
:103D1000008006F8010BF5E730B5104600234FF0A0
:103D20006042834200DB30BDD2F8804EE50707D504
:103D3000D2F8004EE40703D5CC5C156815B11470B9
:103D40000133EEE700BFF8E74FF0FF3070474FF464
:103D500000534B60002070470120704700207047DF
:103D60000B4A116810B5034609B90A491160106879
:103D700009490A4C0344091B8B4206D92AF098FBD7
:103D80000C2303604FF0FF3010BD1360FCE700BF51
:103D9000980D0020103B00200000012000080000CA
:103DA00037B5184B02689A42054628D14FF0B04308
:103DB000154C1A6E42F400621A661B6E134A03F425
:103DC00000630193019B1723C4E900231021002302
:103DD0008020C4E902134FF48073C4E904034FF454
:103DE000806C2023C4E906C320464FF400532362AD
:103DF00004F0A0F808B1FFF79FF96C62A56203B068
:103E000030BD00BF002C01409C0D00200800024086
:103E100010B5044686B01422002101A82AF0E6FA63
:103E200022680F4B9A4218D14FF0B04301A9DA6CC7
:103E300042F00102DA64DB6C03F00103009302221A
:103E4000009B4FF48073CDE901324FF09040012385
:103E5000CDE90332059304F031FB06B010BD00BF7D
:103E6000002C014010B58EB01022002103A82AF0CA
:103E7000BDFA00241C2221460DEB0200CDE90044CE
:103E800002942AF0B3FA1F481F4B8460C0E9003443
:103E90003B23C0E90334C0E9054406F011FD08B135
:103EA000FFF74AF94FF480531648039303A906F02D
:103EB00025FE08B1FFF740F9124806F031FD08B1C0
:103EC000FFF73AF900240F4802946946CDE900440F
:103ED00007F02CF808B1FFF72FF9602309480D947B
:103EE000002207A9CDE90734CDE90944CDE90B4407
:103EF00006F07EFD08B1FFF71FF90248FFF788FFC3
:103F00000EB010BDFC0D0020002C0140014B1868C4
:103F1000704700BF480E00200320704708B50146D7
:103F20004FF47A7200238002890DFEF7BDFA08BDB6
:103F30004FF47A73A0FB0303800A40EA8350704772
:103F4000034B98689A689042FBD1C043704700BF0A
:103F50000028004008B5FFF7F3FF014B186008BDCB
:103F6000480E002008B5FFF7EBFF024B1B68C01A94
:103F700008BD00BF480E0020024B187808B1FFF7BB
:103F8000DFBF70474C0E002010B5074B074C0122D5
:103F9000DA654FF48071204605F0D4F94FF0FF3315
:103FA0002363002010BD00BF002800403808002017
:103FB00002460021014805F0DCBB00BF38080020A4
:103FC00002460121014805F0D4BB00BF380800209B
:103FD00010B58CB02C220021044601A82AF006FA64
:103FE000FFF7D2FF0C4B0D481B681C4400230893BD
:103FF00006934FF00053E443079301224FF480737C
:1040000001A902940B9305F0B1FA08B1FFF794F8F7
:1040100000200CB010BD00BF480E00203808002062
:1040200038B50546FFF78CFF02210446074805F026
:10403000A7FBC4F309024FF47A71A2FB0121920A93
:10404000A30A2A8043EA805038BD00BF3808002008
:104050000148002105F094BB3808002001480121E7
:1040600005F08EBB38080020F8B50F4D2E78CEB97C
:104070000E4C4FF0FF372763FFF760F8FFF784FF20
:104080004FF48071204605F05DF92046276305F066
:104090001BFB32462046022105F06BFBFFF75AFF5F
:1040A00001232B700020F8BD4C0E002038080020A2
:1040B000014610B54FF47A7200238002890DFEF795
:1040C000F3F90146FFF73CFF0446FFF739FF031BF6
:1040D0008B4200D310BD00BFF7E710F0F3BE000025
:1040E00010B5064C0221204605F04AFB0221421C75
:1040F0002046BDE8104005F03CBB00BF380800205A
:104100001648174A08B54FF4E133C0E900230023ED
:104110000C22C0E90233C0E90523C0E90733C0E936
:104120000933036107F0F5FD08B1FFF705F80B4807
:10413000002107F066FF08B1FEF7FEFF07480021E7
:1041400007F07FFF08B1FEF7F7FF044807F039FFDB
:1041500018B1BDE80840FEF7EFBF08BDB00E002063
:104160000044004070B596B006461422002103A812
:104170002AF03CF93822002108A82AF037F93268E1
:10418000274B9A424AD10223089308A84FF44023B0
:104190000A9305F009F808B1FEF7CEFF4FF0B043DF
:1041A00000259A6D1F4C42F400329A659A6D02F414
:1041B00000320292029ADA6C42F00102DA64DB6C9D
:1041C00003F001030193019B0C220223CDE9032399
:1041D00003A907234FF090400793CDE9055504F05C
:1041E0006DF9114925621423C4E900131023C4E9B1
:1041F000023520468023C4E90435C4E9065503F09E
:1042000099FE08B1FEF798FF2520F46700220221ED
:10421000A66203F0FDFD252003F02CFE16B070BD54
:1042200000440040500E00208000024002680C4B09
:104230009A4210B5044612D14FF0B0420C21936D52
:1042400023F4003393654FF0904004F0E3F9E06FFE
:1042500003F0E2FEBDE81040252003F019BE10BDBA
:104260000044004008B50A460146024806F0D0FE68
:10427000002008BDB00E002013B5114B114C186082
:104280004FF40013009302AB13E90600204607F039
:104290003CFE2368DA69D103FCD4DA695202FCD50A
:1042A0009A68084842F480029A6007F074FE064952
:1042B0000448012207F0E2FD002002B010BD00BF5B
:1042C000440F0020B00E00204C0F002008B5074B13
:1042D0001860FEF768FCFFF713FF054AD2F880303C
:1042E00043F00063C2F88030002008BD480F002072
:1042F0000008005808B54FF0B04308489A6B42F4E4
:1043000000329A639A6B22F400329A63FFF78EFFB1
:10431000112003F0BDFD002008BD00BFB00E00203D
:1043200008B5074807F0F5FC08B1FEF705FF05489A
:1043300003F000FE18B1BDE80840FEF7FDBE08BD61
:10434000B00E0020500E00200268044B9A4203D1A8
:10435000034B00201B681847704700BF0044004013
:10436000480F002002680B4B9A4210B504460FD14B
:10437000094B1B682BB1D0F8902012B907480121D6
:10438000984720460549BDE81040012207F076BD58
:1043900010BD00BF00440040440F00204C0F00201F
:1043A0002DE9F04F9DB0FEF78DFA13F033FA024677
:1043B00040B90146644B022010F0B8F901201DB04D
:1043C000BDE8F08F012013F0CDFA11F0C9FF0446CB
:1043D000039040B9024601465C4B022010F0A6F95A
:1043E00013F08CFAEAE75A4D296812F009FC696863
:1043F000204612F01FFC297A204612F04FFC697A01
:10440000204612F07FFC6969204612F00BFDE86837
:10441000FEF72AF881B2204612F08EFC2969204668
:1044200012F056FCA97A204612F01EFC022120460A
:1044300012F0D0FC1021204612F00EFD039812F06D
:1044400017F80246049040B90146424B022010F092
:104450006DF903A811F0E4FFC2E703A811F0E0FF33
:10446000049812F06DFB024640B901463A4B022017
:1044700010F05CF904A812F019F9B1E7374EDFF833
:10448000E0A0DFF8E0B0002333604FF002080498AA
:1044900005AB0A2208A912F045F9054628BB0246D9
:1044A0000146314B022010F041F930682C49FDF7EC
:1044B000D9FD4FF07C51FDF7D5FD3060049812F026
:1044C0006FFB044604A812F0F1F813F017FA002C61
:1044D0003FF474AF002D3FF471AF0022234B11461F
:1044E000032010F023F9002069E731680998FDF7EF
:1044F000B1FCBDF81890306000221D4BCDF8009043
:104500001146022010F012F908AC0027BBB2994501
:1045100004F1080405D8B8F1010FC6D04FF0010826
:10452000B5E754F8040C5146FDF79CFDFDF79CFFE0
:10453000019034F8083C009300225B4611460220AB
:1045400010F0F4F80137E1E7C05C0308D85C030819
:10455000080000200D5D0308345D0308F4180020F6
:1045600000007A44975D03085D5D0308AE5D0308B3
:10457000865D030830B5044685B0084614491546E3
:10458000FDF770FDFDF74AFFCCB1114902902846B6
:10459000FDF768FDFDF742FF0E4901902846FDF743
:1045A00057FC0D49FDF712FEFDF75EFF002200905B
:1045B0000A4B1146032010F0B9F805B030BD009049
:1045C000074B22462146032010F0B0F8F5E700BF64
:1045D00000007A44CDCC4C3FCDCCCC3EC75D030827
:1045E000F45D03082DE9F04FADF2344D4FF4007245
:1045F00000210CA829F0FAFE4FF4007200218CA8CB
:10460000B34E29F0F3FE002537464FF000082C4644
:10461000B9682046FDF71EFC796804462846FDF778
:1046200019FC08F10408B8F5007F054607F11007EA
:10463000EED14FF070512046FDF714FD4FF0705150
:1046400004462846FDF70EFD0025DFF88482074664
:104650004FF00009AA46D8F808002146FDF7F8FBFC
:104660000146FDF7FFFC01465046FDF7F3FB3946D6
:104670008246D8F80400FDF7EBFB0146FDF7F2FC9B
:1046800001462846FDF7E6FB09F10409B9F5007F6C
:10469000054608F11008DED14FF070515046FDF785
:1046A000E1FC4FF070510A902846FDF7DBFC824692
:1046B0000A98FDF749F8874B00222BF00DFECDE953
:1046C00004015046FDF740F8824B00222BF004FE17
:1046D000FDF76AFB0DF130090546C84600234FF08F
:1046E000000BB168B0690693FDF7B2FBFDF796FECB
:1046F0000028B8BF4042FDF761FC48F8040B0146B2
:104700005846FDF7A7FB069B0433B3F5FE7F8346AF
:1047100006F11006E5D17049FDF758FD0DF130089E
:10472000064600234FF0000B314658F8040B069361
:10473000FDF78EFB0146FDF795FC069B01461846EA
:10474000FDF788FB0BF1010B1FFA8BFBBBF17F0F11
:104750000346E9D16049FDF739FDFCF7F5FF5D4BF4
:1047600000222BF0B9FDCDE906010DF50C78C3460A
:10477000002200234846D9F8001040680B930892A5
:10478000FDF766FBFDF74AFE0028B8BF4042FDF783
:1047900015FC089A4BF8040B01461046FDF75AFB2E
:1047A0000B9B01339BB27E2B09F104090246E1D138
:1047B0004A49FDF70BFD4FF0000B814600234946A7
:1047C00058F8040B0893FDF743FB0146FDF74AFC3C
:1047D000089B01461846FDF73DFB0BF1010B1FFA44
:1047E0008BFBBBF17E0F0346E9D13C49FDF7EEFCA4
:1047F000FCF7AAFF374B00222BF06EFDCDE9080134
:1048000037492846FDF72EFCFDF708FE3449029093
:104810005046FDF727FCFDF701FE3149019038466F
:10482000FDF720FCFDF7FAFD002211462D4B00900C
:1048300002200FF07BFF2C492C4F2846FDF7BAFDD4
:1048400008B105233B702A4B1A782A4B1B889BB270
:104850009A4280F08C80284B1A78284B1B889BB298
:104860009A4206D226492046FDF7B8FD08B1012339
:104870003B70244FDFF890A03B880A9A01339BB22B
:104880003B803B889BB20A2B04BF00233B803B88C4
:104890004FF01C0B9BB20BFB03F3DDE904014AF85C
:1048A00003403B889BB20BFB03A35A603B889BB23F
:1048B0000BFB03A8FDF778FA3B88C8F808009BB209
:1048C0000BFB03A34FF08641DD603D8830461DE0C1
:1048D000741000200000E03F0000FE420000FC4297
:1048E00000007A440A5E030800007A435A0F002051
:1048F0008B030020520F00208A030020500F00205D
:10490000CDCC4C3F741800205C0F0020FDF7AAFBB3
:10491000ADB20BFB05A528613D88DDE90601FDF779
:1049200043FA4FF08641FDF79DFBADB23B880BFB90
:1049300005A59BB26861324D0BFB03AA2A788AF861
:104940001820DDE90801FDF72FFA4FF08641FDF749
:1049500089FBFDF789FD2B4BC0B218802B78012B0A
:1049600005D10022284B114602200FF0DFFE274F11
:10497000234D3B78DFF89880012B24D1DFF8949009
:10498000254EB9F80030B9F800204FF01C0A9BB250
:1049900092B20AFB03F30AFB0262F0589168FDF73A
:1049A00059FA2146FDF71AFDB0B102232B702B787E
:1049B000022BD8B204D10022184B11460FF0B6FEDC
:1049C0002B78DBB23B702B78DBB23B70C8F8004031
:1049D0000DF2344DBDE8F08FB9F80030D8F80090F2
:1049E0009BB20AFB03662046B168FDF733FA4946DD
:1049F000FDF7F4FC10B103232B70E4E72870E2E725
:104A00005A0F00204E0F0020505E0308580F002060
:104A1000540F0020741800205C0F0020955E0308DE
:104A20002DE9F04F9FB0FDF74DFF12F0F3FE024667
:104A300040B90146A84B03200FF078FE01201FB0BB
:104A4000BDE8F08F012012F08DFF10F0A1FB0446AD
:104A50000D9040B902460146A04B03200FF066FEC0
:104A600012F04CFFEAE79E4F3B78012BDDB252D0AB
:104A7000022D6FD0002D39D1042110F04FFF0121FC
:104A8000204610F079FE9749204610F0A9FE96497D
:104A9000204610F08BFE9549204610F039FE9449CF
:104AA000204610F04FFE0221204610F06BFF914986
:104AB000204610F04DFF214606A810F0ABFE8E4AAE
:104AC00019928E4A1A924FF07C53002218A9204660
:104AD00018931B921C921D9310F0C8FE2946204685
:104AE00010F0E8FE0321204610F0FEFE0D98002491
:104AF0003C7010F0E3FB02460E9000286DD1804B15
:104B0000014603200FF012FE0DA810F0AFFB0EA817
:104B100010F062FCA4E77B4E294610F02DFE71498F
:104B2000204610F05DFEB168204610F0F1FDF168FE
:104B3000204610F007FE716A204610F037FEF16C37
:104B4000204610F005FF704B0022114601200FF0A7
:104B5000EDFDCBE76B4D012110F00EFEE96920461B
:104B600010F03EFE696A204610F020FEA96820463B
:104B700010F0CEFDE968204610F0E4FDA86CFDF7CA
:104B800073FC81B2204610F0FDFEE96C204610F067
:104B9000DFFE214606A810F03DFE2B6B18936B6BD1
:104BA0001993AB6B1A93EB6B1B932B6C1C9318A98B
:104BB0006B6C1D93204610F059FEA86AFDF754FC5B
:104BC000C1B2204610F076FE286AFDF74DFCC1B256
:104BD000204610F0F1FE4D4BB6E710F093FC38B9CB
:104BE00000224B4B114603200FF0A0FD002026E7CA
:104BF0001422214613A829F0F9FB0026DFF8EC80E7
:104C0000DFF81091DFF810A1212537460E980FA983
:104C100010F0D0FC0246002840F08A8001463F4B4D
:104C200003200FF083FDDFF8F8800E9810F08AFC67
:104C3000B8F8003000229BB2114600930320394B94
:104C40000FF074FD0D9D0121284610F095FD042103
:104C5000284610F063FE2349284610F0C1FD224982
:104C6000284610F0A3FD2149284610F051FD2049A7
:104C7000284610F067FD0221284610F083FE1D49EA
:104C8000284610F065FE294606A810F0C3FD1A4A12
:104C90001992254A1B924FF07C534FF07E5218A96F
:104CA00028461C9218931A931D9310F0DFFD0021E3
:104CB000284610F0FFFD0321284610F015FE0D993F
:104CC0000EA810F0B3FB0246002840F08480014695
:104CD000164B022016E700BFC05C0308DA5E03082B
:104CE000F0180020000082429A99993FCDCC4C3FA9
:104CF000000020406666263F000020410AD7233C82
:104D00005C5F030878180020FA5E03082A5F030836
:104D1000775F0308CDCCCC3E88030020955F030865
:104D200076180020BE5F0308CDCC4C3EF35F03082D
:104D3000119A10999DF83C00FFF71CFC9DF83C303F
:104D4000FBB1DDF844B038465946FDF783F81099B9
:104D500007463046FDF77EF8414606465846FDF7C1
:104D600077F84946FDF732FAFDF77EFB1EAB80B2BD
:104D700003EB4000013430F82C3C0133E4B220F85E
:104D80002C3C9AF80030012B1ED1DFF818B2864A6D
:104D9000BBF8003011999BB202EB03139960BBF88A
:104DA00000309BB202EB0312109B5360BBF8003043
:104DB0009BB25A1C92B2802BABF8002004D1FFF7B3
:104DC00011FC0023ABF800300F20FDF7F3FD013D8F
:104DD0007FF41CAF27E70E9810F094FB00283FF4F7
:104DE000FFAE0DA810F042FADFF8C0B14FF0210974
:104DF0000E980FA910F0DEFB054600287CD1024674
:104E000001466B4B03200FF091FCB8F80030DFF83F
:104E1000A491DFF8A4B100229BB2114600930320B5
:104E2000664B0FF083FC012C94BF0023012389F80B
:104E3000003099F800300022CDE900431146604B64
:104E400003200FF073FC0DF14C084FF0000A38F806
:104E5000022B3AB1CDE900A200225B4611460120A7
:104E60000FF064FC0AF1010ABAF10A0FEFD15549BB
:104E70003846FDF7F7F807462046FDF79FF88046CD
:104E800001463846FDF7A2F94E4907463046FDF780
:104E9000E9F84146FDF79AF94B4B1F604B4B002157
:104EA00018608046FDF772FA0646A8B942234046CC
:104EB00099F80090CDE90343FDF7B0FA0290384627
:104EC000FDF7ACFA5FFA89F9CDE90090404B324624
:104ED000314603200FF02AFC0E9810F033FB0446F5
:104EE0000EA810F079FA12F009FD002C3FF4A6ADDF
:104EF00085F00100C0B2A2E5119A10999DF83C001E
:104F0000FFF738FB9DF84930002B43D19DF83C302A
:104F1000FBB1DDF844A038465146FCF79BFF1099E1
:104F200007463046FCF796FF2A4906465046FCF7EE
:104F30008FFF5946FDF74AF9FDF796FA1EAB80B28E
:104F400003EB4000013430F82C3C0133E4B220F88C
:104F50002C3C214B1B78012B1CD1B8F80030124A95
:104F600011999BB202EB03139960B8F800309BB221
:104F700002EB0312109B5360B8F800309BB25A1C2E
:104F800092B2802BA8F8002004D1FFF72BFB00235E
:104F9000A8F800300F20FDF70DFDB9F101097FF4ED
:104FA00027AF32E77618002074100020CDCCCC3E1D
:104FB000955F0308D318002072600308136003088C
:104FC0003E60030800007A44CC180020C818002076
:104FD00092600308CDCC4C3F880300202DE9F043BC
:104FE000ADB014230DF10E0204A9ADF80E3012F08D
:104FF00099FE044648B902460146194B03200FF0BA
:1050000095FB20462DB0BDE8F0830022154B164FCE
:10501000DFF85880DFF85890114603200FF086FB28
:105020000025BDF80E30AAB29342EAD9AAB22CAB41
:1050300003EBC202032012F89C6C52F8A03C002E35
:1050400014BF3A464246CDE9003200224B46114693
:105050000FF06CFB002E05F1010508BF3446E0E7B8
:10506000EC6003080F610308E2600308E7600308CF
:105070003361030830B5102289B000252946044663
:105080000DEB0200039529F0B1F914F0F5F92A4669
:10509000A34B0090294603200FF048FBFDF712FCBC
:1050A00012F0B8FB8DF80C0012F05EFC431B18BF29
:1050B000012301218DF80D30029012F073FC02984B
:1050C00012F012FE029812F087FC0298FFF786FF9A
:1050D000002840F0008102A812F056FC12F00EFCED
:1050E000029812F095FC029812F0AEFC0298FFF7BD
:1050F00075FF002840F0F38002A812F045FC12F082
:10510000FDFB029812F0BCFC0022864B11460320E6
:105110000FF00CFB029812F0CFFC0298FFF75EFF35
:10512000002840F0E08002A812F02EFC12F0E6FB0E
:10513000029812F0DDFC002211467B4B03200FF099
:10514000F5FA0022794B114603200FF0EFFA02988E
:1051500012F05AFD0298FFF741FF002840F0C78087
:1051600002A812F011FC12F0C9FB029812F068FDBF
:10517000002211466E4B03200FF0D8FA00226D4B2F
:10518000114603200FF0D2FA029812F075FD029832
:10519000FFF724FF002840F0AE8002A812F0F4FBD5
:1051A00012F0ACFB029812F083FD00221146624B14
:1051B00003200FF0BBFA0022604B114603200FF0D2
:1051C000B5FA029812F0B0FC0298FFF707FF00282A
:1051D00040F0958002A812F0D7FB12F08FFB0298E6
:1051E00012F0BEFC00221146554B03200FF09EFA30
:1051F0000022544B114603200FF098FA029812F047
:10520000CBFC0298FFF7EAFE00287CD102A812F03E
:10521000BBFB12F073FB029812F0DAFC002211467D
:10522000494B03200FF082FA0022404B1146032025
:105230000FF07CFA029812F0E7FC0298FFF7CEFE1E
:10524000002864D102A812F09FFB12F057FB0298CD
:1052500012F0F6FC00221146354B03200FF066FADF
:105260000022344B114603200FF060FA029812F02E
:1052700003FD0298FFF7B2FE00284CD102A812F0FD
:1052800083FB12F03BFB029812F012FD0022114644
:10529000294B03200FF04AFA002211462B4B032022
:1052A0000FF044FA01238DF8173003AB03CB002233
:1052B0002060186861600C23A060114600930320F1
:1052C000234B0FF033FA02A812F05EFB12F016FB2C
:1052D000002009B030BD01238DF80E3000E7012316
:1052E0008DF80F300DE701238DF8103020E70123F2
:1052F0008DF8113039E701238DF8123052E7012380
:105300008DF813306BE701238DF8143083E7012308
:105310008DF815309BE701238DF81630B3E700BFF9
:105320004961030872610308A5610308D661030897
:105330000562030832620308676203089A62030881
:10534000CD620308FE6203082E6303085C63030852
:105350008963030802480122102103F0D5B900BF78
:105360000004004802480022102103F0CDB900BF1C
:105370000004004813B5134C23785BB9E37C03F0B9
:10538000FF023BB9104B1146022002B0BDE81040AD
:105390000FF0CCB9FEF7B2F800380C4B18BF012063
:1053A000400018701A78022A02BF00222270E274AC
:1053B0001B7800930022064B114603200FF0B6F92C
:1053C00002B010BD5D1B0020A8630308381900203F
:1053D000C463030838B5184C23785BBBE37C03F047
:1053E000FF023BBB154D2B68012B0CD92B68042BFE
:1053F00009D81146124B02200FF098F9114A0421E6
:10540000012000F0F7FE2B68042B13D900220E4B6D
:10541000114602200FF08AF9FEF770F800380B4BA6
:1054200018BF0120400018701B78022B02BF002318
:105430002370E37438BD00BF5D1B002034190020C9
:10544000DB630308006403080564030838190020BF
:1054500010B501214FF0904003F050F90C4B0D4A6C
:105460001870002414701B780B4ADBB202214FF035
:105470009040137003F042F9084B094A18701470F9
:105480001B78084ADBB21370BDE81040FEF74CB938
:10549000F2000020F2180020F0000020F1000020AF
:1054A000F1180020EF00002010B5FEF733F9164B7D
:1054B0001A78022A26D91B78072B23D8FFF7B0FACF
:1054C0001248134A037811785B1A124918BF012356
:1054D0000B7003781048DBB21370104B104A1C7825
:1054E0000378E31A18BF012313700E4B04701B7866
:1054F00023B100230B700C490B701370BDE81040F2
:10550000FEF712B910BD00BFEE000020D318002036
:10551000D0180020D4180020580F00205A0F002067
:10552000590F002038190020D618002070470000BD
:1055300038B5324D324C287BFCF73CFD3149FCF745
:1055400091FDA060687BFCF735FD2E49FCF78AFDD4
:10555000E060A87BFCF72EFD2A49FCF783FD606222
:10556000E87BFCF727FD2849FCF77CFD274BE0642E
:105570002361287CFCF71EFD6060687CFCF71AFD47
:10558000A061A87CFCF716FDE061E87CFCF712FD49
:105590002062287DFCF70EFDA062687DFCF70EFD01
:1055A0001849FCF75FFD2063A87DFCF703FD6063ED
:1055B000E87DFCF703FD1449FCF754FDA063287E49
:1055C000FCF7F8FCE063687EFCF7F8FC0D49FCF79B
:1055D00049FD2064A87EFCF7F1FC0A49FCF742FD76
:1055E0006064E87EFCF7E6FCA064287FFCF7E2FC40
:1055F000074BE06202221A7038BD00BF4003002052
:1056000078180020CDCCCC3D0AD7233CCDCCCC3E65
:10561000F018002038B5114D114C287BFCF7CEFC5A
:105620001049FCF71FFDA060687BFCF7C7FC0D4923
:10563000FCF718FDE060A87BFCF7C0FC0949FCF70B
:1056400011FD6062E87BFCF7B9FC0749FCF70AFD35
:10565000064BE06401221A7038BD00BF40030020F1
:1056600078180020CDCCCC3D0AD7233CF018002080
:105670007FB5434E434D33780370434B1B784370E3
:10568000044601214FF0904003F038F82B78A070C9
:10569000E37002214FF0904003F030F83B4B207153
:1056A0001B78637100223A4B114602200FF03EF83E
:1056B0002B78012B5AD100221146364B02200FF0D5
:1056C00035F8354B1868FCF7CFFE344BE08018688E
:1056D000FCF7CAFE80B2324BA0831B7884F82430DA
:1056E000191F4A424A41A2779BB12E4A03EB83031A
:1056F00002EB83030022009311462B4B02200FF094
:1057000015F82A4B1B8884F82530294B1B8884F810
:10571000263002A80FF06CFA264B1A780AB3264AF4
:105720001168F1B11268254A1568254A12681B787C
:10573000AD1AC3EB0313B5EB830F12D90022214B33
:10574000114602200EF0F2FF1F4B258501221A7030
:105750001B781E4A84F82730082313703370FDF736
:10576000D9FF1B4B01221A7004B070BD0022194BE7
:10577000114602200EF0DAFF0020E080ABE700BF08
:1057800005000020D3180020EE000020D2180020D1
:10579000386403085F640308CC180020C818002090
:1057A0005A0F002026000020AB640308520F00208F
:1057B0004E0F002089030020EC180020E418002080
:1057C000E0180020E46403085B1B002006000020B2
:1057D0003019002087640308024B012200210320B6
:1057E0000EF0A4BF04650308024B01220021032030
:1057F0000EF09CBF3A65030808B50122074B002153
:1058000003200EF093FFFFF7A5FDFFF791FE044A7A
:1058100000231370034A137008BD00BF806503089E
:10582000F0180020591B002010B5104B0122002158
:1058300002200EF07BFF0E4B04225A7063210122DE
:1058400000241A7083F82A1083F82B201C635C63F1
:1058500083F827401C85FFF77DFDFFF7C5FFFFF7A5
:10586000BBFFFFF7C9FF034B1C7010BDB6650308F3
:10587000F8180020591B00201FB5114B11491C6856
:1058800058681A7A5B7ACDE90223FCF7EBFBFCF748
:10589000EBFD0C4901902046FCF7E4FBFCF7E4FD2E
:1058A0000022094B0090114603200EF03FFFFEF747
:1058B00077FD642004B0BDE81040FEF7A1B900BF39
:1058C0000800002000007A44ED65030870B586B03A
:1058D0000D460446FFF73EFD01F016FEFDF730FBD6
:1058E0009620FEF78DF90026AE420AD101AB03CB1C
:1058F0001B882381094B2060002261601A7006B06A
:1059000070BDFEF757F801A8FFF7B4FB41F28830ED
:10591000FEF776F90136FFF7AFFFE5E7591B0020E8
:1059200030B585B00446002503A8ADF80C50FCF74F
:10593000CDFF70B19DF80C309DF80D202370627082
:105940002946CDE900320320034B2A460EF0EEFE35
:10595000012005B030BD00BF22660308022801D82F
:10596000FFF7F8BC7047022801D8FFF7FBBC70476F
:10597000022803D80248102102F0CBBE704700BFB6
:105980000004004808B5FEF787F8BDE8084000F0BD
:1059900069BE4FF0FF300FF013B87047704700003A
:1059A000014BD870704700BF00010020014B1874F4
:1059B000704700BF0001002007B5064B00221B5CAA
:1059C00000931146044B02200EF0B0FE03B05DF8C8
:1059D00004FB00BF616603084766030808B50021A1
:1059E00002200EF0B5FF0A4B1B7803F0FF014BB904
:1059F000084B1A68042A05D81A68102001321A6068
:105A00000EF0A6FFBDE8084003480FF009BA00BF3A
:105A10005D1B002034190020C01A00200021012045
:105A20000EF096BF13B5104A104C42F210730028C6
:105A300018BF03460E48236013600FF0A3F92168D6
:105A40000B480FF027FA0A480FF0EAF923684FF4E1
:105A50007A72B3FBF2F3002200931146054B01204A
:105A60000EF064FE02B010BD80030020FC00002098
:105A7000C01A00206566030813B50D4C206023682A
:105A80000BB90C4B23600C480FF07CF921680A48D5
:105A90000FF000FA08480FF0C3F9236800930022C2
:105AA000064B114603200EF041FE02B010BD00BFB0
:105AB00080030020A08601003C19002091660308A5
:105AC00037B5044600283AD090F90650002D40D151
:105AD00023480FF057F92A462946224B02200EF0A0
:105AE00025FEE379012B0CBF1F4B204B2A4629468C
:105AF00002201F4D0EF01AFEE3792B701D4B186823
:105B0000FFF7BAFF1C4B1868FFF78CFF29781B4A78
:105B10001B4B012908BF1346002200931146194B65
:105B200001200EF003FE94F90530019394F904303E
:105B300000930022144B114603200EF0F7FD134B87
:105B40000122002102201A7003B0BDE830400EF09F
:105B5000FFBE00220E4B114602200EF0E7FDE2E7E9
:105B60006C190020D6660308EB6603080867030873
:105B70005A1B002080030020FC000020CD66030893
:105B8000D1660308256703085D670308581B0020DA
:105B9000446703080A460149FDF78CB900F0030881
:105BA00070B516480FF0EEF806F0ACFE044650B1A2
:105BB0000022134B114602200EF0B8FDBDE87040E4
:105BC00010480FF02DB9104D104B0246014602202F
:105BD0000EF0ACFD01260E4B2E702246214602200F
:105BE0000EF0A4FD0B4806F021FD2878314606F0A2
:105BF00075FA02480FF014F9E0E700BFC01A002060
:105C000086670308A81A002064010020A46703081F
:105C1000B867030800010020F0B599B0FDF76EFFEA
:105C2000054606F055FB0746002860D1834C0AA8BC
:105C3000FFF71EFD13232370814B1A7802F0FF0635
:105C4000002A65D01F70142323707E4B62681B7876
:105C500063F07F03137062682BB203EB4303FE21F2
:105C600003EB43130220B3FBF1F339465370764B39
:105C70003A460EF05BFD0223744A754D1278012AF4
:105C800094BF1A4600226270CDE9012300222378D6
:105C9000009311466F4B01200EF048FD6B7A63B103
:105CA00006F002FB0128044607D128460FF06AF8E7
:105CB00069482246042102F027FD684B5F48D978E5
:105CC000002206F01BFB0446002840F0A280624838
:105CD0000122042102F018FD012221461046604BEA
:105CE0000EF024FD5C482246042102F00DFD002444
:105CF0005C480FF047F85C4B5A481968A14238BF1E
:105D000021460FF0C7F857480FF08AF819B0F0BDD8
:105D1000564D2A7802F0FF03002AADD0544B32468C
:105D2000314602200EF002FD464B62681B782E7051
:105D300063F07F03137063689DF828205A706168D0
:105D40009DF829308B7061689DF82A00C8706168E1
:105D50009DF82B00087161689DF82C0048716168FE
:105D60009DF82D008871BDF82E106068090AC17178
:105D70006068BDF82E100172BDF84410090A417226
:105D8000BDF8441081729DF84610C1729DF84C1008
:105D900001739DF84F104173BDF85010090A8173CB
:105DA000BDF85010C17303EB8303324903EB830347
:105DB0000B440193304B02EB820203EB420300934E
:105DC00032462E4B314601200EF0B0FC9DF84C308F
:105DD0000893BDF84A3007939DF846300693BDF806
:105DE00044300593BDF82E3004939DF82D30039375
:105DF0009DF82C3002939DF82B3001939DF82A30AA
:105E0000009332461E4B314601200EF08FFC1023CA
:105E100032E706347FF46BAF06F040FA0446002800
:105E20003FF465AF01224FF47A730021B0FBF3F326
:105E300010460093134B0EF079FC59E7F400002054
:105E4000581B0020B4190020D76703083819002018
:105E50006C19002078690308000400480001002044
:105E6000C0690308C01A0020FC000020301900207F
:105E7000FD67030865010020DC0200202A68030892
:105E800067680308CF69030800B503468DB0002892
:105E90002CD0407802280AD003282AD0164B0022A2
:105EA000114602200DB05DF804EB0EF03FBC1A7FE6
:105EB0000B92DA7E0A929A7E09925A7E08921A7E94
:105EC0000792DA7D06929A7D05925A680492DA6802
:105ED000039293F914200292B3F9122001921B7CD1
:105EE00000930022054B11460EF020FC0DB05DF82A
:105EF00004FB034BD3E700BFED690308046A030802
:105F0000766A030801284FF000020CBF024B034BD6
:105F1000114602200EF00ABC956A0308A76A03081E
:105F20001FB50446002831D00378002B2ED01D4821
:105F30000EF076FF002211461B4B02200EF0F6FBFE
:105F400094F91830039394F90A300293237C019357
:105F5000E368009300221146144B02200EF0E6FB8A
:105F60000022134B114602200EF0E0FB237A012B96
:105F70000ED1617A0F4A104B002918BF1346002238
:105F8000009311460D4B02200EF0D0FB04B010BD63
:105F900000220B4B1146022004B0BDE810400EF069
:105FA000C5BB00BF9C190020C06A0308F16A030842
:105FB000226B0308BC6A0308BB6A03082F6B030843
:105FC000406B030808B5104B0122002102201A7013
:105FD0000EF0BEFC0D480EF023FF0D4B1B788BB16D
:105FE0000C4B1A7872B9DB7C63B90B4B1A68042A24
:105FF0009EBF1A6801321A600021BDE808401020D7
:106000000EF0A6BC08BD00BF581B00203C190020A4
:106010005A1B00205D1B00203419002008B5002108
:1060200040200EF095FC074B1B7853B1064B1A78B5
:10603000012A06D100211970BDE8084002200EF0A7
:1060400087BC08BD5A1B0020D4180020044B1B78C5
:10605000022B03D1002108200EF07ABC704700BF4C
:1060600064010020044B1B78012B03D00021802009
:106070000EF06EBC704700BFEE00002008B506F0C1
:106080004AFC80B906F010F901280CD1BFF34F8FFC
:106090000549064BCA6802F4E0621343CB60BFF3C4
:1060A0004F8F00BFFDE708BD00ED00E00400FA05DA
:1060B00038B504460D4607484FF40061FCF71AFF57
:1060C00030B92A4621460348BDE83840FCF718BEDF
:1060D00038BD00BF00F0030810B506F0B1FC10F1A8
:1060E000080F07D1064B0022BDE8104011460220E0
:1060F0000EF01CBB013001D1024BF4E710BD00BF14
:106100004E6B0308646B030870470000022837B524
:10611000044634D0402853D0012854D12B4B1B784F
:10612000002B50D0FA20FDF76BFD21464FF0904038
:1061300002F0E4FA264B214618704FF0904002F02E
:10614000DDFA214605464FF0904002F0D7FA214B88
:10615000214A002808BF1346CDE900531F4B0022F7
:10616000114602200EF0E2FA002120200EF0F0FB92
:106170000021022003B0BDE830400EF0E9BB184B0F
:106180001B7803B3FA20FDF73BFD21464FF090400A
:1061900002F0B4FA134B214618704FF0904002F011
:1061A000ADFA214605464FF0904002F0A7FA0E4B9B
:1061B0000E4A002808BF1346CDE900530C4BCEE72A
:1061C00000210420D6E703B030BD00BFF218002044
:1061D00003000020886B03087C6B0308AE6B030888
:1061E000F118002002000020A16B0308946B030843
:1061F000D46B030873B505460C46164606F068F8DE
:106200000346002840D000242A480EF0BBFD2A4B4C
:1062100028481968A14238BF21460EF03BFE2548A8
:1062200002B0BDE870400EF0FBBD4A68F05CD0548F
:106230000133DAB29442F8D8204B0D701A781B78EB
:10624000012A88BF00244C700022CDE900341C4C88
:106250001C4B114601200EF069FA637A33B106F047
:1062600023F8012802D120460EF08CFD164B17486A
:10627000D978002206F042F8014638B9144B0122C1
:1062800003200EF053FABEE71049D2E70631BAD127
:1062900006F004F804460028B6D04FF47A730122C1
:1062A000B0FBF3F30021009303200A4B0EF03EFAFB
:1062B000AAE700BFC01A0020FC0000203819002007
:1062C0006C190020F96B030800010020F400002085
:1062D000C0690308CF690308044B1B7823B9044A3B
:1062E00005210120FFF786BF704700BF3819002045
:1062F0002A6C030810B5002490B03C22214601A866
:10630000009428F073F8354B2022DA7219788DF852
:10631000001059788DF8011099788DF80210D9780D
:106320008DF8031019798DF8041059798DF805103E
:1063300099798DF80610D9798DF80710197A8DF8AA
:106340000810597A8DF80910997A8DF80A108DF88D
:106350000B2021460DF10B0258180131007B02F889
:10636000010F1C29F8D193F828208DF8282093F8E4
:1063700029208DF8292093F82A208DF82A2093F8D7
:106380002B2093F828108DF82B20154A19BB93F871
:10639000291001F0FF00F1B9107093F82C206AB1B8
:1063A00093F83F2052B10DF12B01002298180132D1
:1063B00090F82C0001F8010F142AF7D109484FF486
:1063C0000061FCF797FD20B9064840226946FCF7BA
:1063D00097FC10B010BD01211170DEE740030020D2
:1063E0008803002000F8030810B500220446114677
:1063F000054B02200EF09AF920460449BDE81040F2
:1064000040220EF099BA00BF306C030800F8030870
:1064100073B54B4C207963794D2BC0B25ED1C0EB84
:10642000001080000A2838BF0A204FF47A735843BE
:10643000444B1860A379E2794D2ADBB256D1C3EB05
:1064400003139B004FF47A7202FB03F594F82C308F
:10645000002B53D194F83F30002B4FD142F21070F3
:10646000FFF7E0FA384B1868FFF706FB237A374A44
:106470003749DBB21370374B01221A70637A364A00
:10648000DBB2137094F82830344A03EB83035B00CB
:10649000DBB2137094F82930314A03EB83035B00BD
:1064A000DBB2137094F82B302E4A03EB83035B00AE
:1064B000DBB213700023E21892F82C20D2B2CA5437
:1064C0000133142BF7D1A378012B37D1E37A202B9A
:1064D00034D102B0BDE87040FFF7A6B96379482B0C
:1064E0000ABF4FF46163637958439BE7E279482A16
:1064F0000ABF4FF46162E2795343A3E71A4EFFF7F4
:1065000091FA3560336813B942F21073336017485B
:106510000EF038FC316815480EF0BCFC13480EF044
:106520007FFC33684FF47A72B3FBF2F300220093DE
:1065300011460F4B01200EF0F9F897E702B070BD3D
:1065400040030020FC00002080030020EE0000201B
:106550005D1B002005000020381900208B0300205F
:106560008A0300208903002084030020541900209E
:10657000446C030810B590B000213C2201A80091A2
:1065800027F034FF4022344968460EF0D5F99DF8D3
:1065900000203AB99DF80100102803D19DF802109F
:1065A00001290FD000222D4B114602200EF0BEF81B
:1065B000FFF7A0FE4FF47A70FDF722FBFFF728FFEC
:1065C00010B010BD264B1A70587099709DF80310CA
:1065D000D9709DF8041019719DF8051059719DF836
:1065E000061099719DF80710D9719DF8081019725D
:1065F0009DF8091059729DF80A1099729DF80B10B8
:1066000001F03F01D972D87AD1B288421BD89DF8E7
:10661000282083F828209DF8292083F829209DF838
:106620002A2083F82A209DF82B2083F82B200DF1B7
:106630002B0100229818013211F8014F80F82C40EC
:10664000142AF7D1BAE701F140006844194410F860
:10665000340C08730132D6E700F803087D6C030898
:1066600040030020F0B50C238BB005260024012543
:10667000CDE9056318221023CDE903322146694B89
:10668000029422460327CDE90055022009940EF01A
:106690004DF8654B029422462146CDE90057022071
:1066A0000EF044F8CDE901640226604B00962246C4
:1066B000214630460EF03AF85D4B009522462146C1
:1066C000CDE9017430460EF031F809A9204606F0F4
:1066D00007F9099BC3F307220292C3F307421B0E7B
:1066E000019200932246534B214630460EF01EF88D
:1066F00009A9284606F0F4F8099BDAB20392C3F31D
:1067000007220292C3F307421B0E01920093224616
:10671000494B214630460EF009F8484B4848009452
:1067200022464FF4FA710EF0CFFA464B46480094D9
:1067300022464FF4FA710EF0C7FA444B44480094D5
:106740002A464FF4FA710EF0BFFA2046FCF7D2FA4F
:1067500008B1FCF7F1FC3F4B009400224FF4FA61C2
:106760003D480EF0B1FA3D4A002101200EF0ACF98F
:106770003B4A002102200EF0A7F93A4A00210420EA
:106780000EF0A2F9384A002108200EF09DF900F021
:1067900015FE3649364806F059F8364805F046FFEA
:1067A0002B480EF03DFB344B0021187805F096FC89
:1067B00032490094324B0968324800220EF084FAC4
:1067C00030480EF02DFBFFF7D5FE2F4A0021102098
:1067D0000EF07AF92D4A002120200EF075F92C4A8E
:1067E000002140200EF070F92A4A002180200EF08E
:1067F0006BF9294B29481968294B009401220EF0A6
:1068000063FA26480EF00CFB264B27481968274BE5
:10681000009401220EF058FA23480EF001FB0BB051
:10682000F0BD00BFBD6C0308FD6C03081E6D0308BE
:106830003F6D0308606D0308816D03089B590008D4
:106840009C19002009610008841900206560000877
:106850006C1900204D600008A81A002031C40008FF
:10686000195C0008D9600008A15B00080000030162
:10687000180100200001002064010020FC0000201D
:10688000DD590008C01A0020D553000851540008F3
:10689000A95400082D550008840300205419002035
:1068A0001D600008800300203C190020C55F00081F
:1068B00073B50D4D00262E60FEF7DEFFC820FDF7F4
:1068C0009FF928683146FBF761FD04460028F3D1A3
:1068D0002868FBF7A3FD054B0090224621460120C6
:1068E0000DF024FF02B070BDF4180020A56D030860
:1068F00030B50024A5B07C22214605A8049427F0D9
:1069000075FD53238DF8103001254FF48873ADF8D1
:106910001230ADF800408DF81450FDF7EFF8FE236B
:10692000B0FBF3F000EB400000EB40103A4B8DF869
:1069300015002246214603200DF0F8FE6846FEF7BA
:10694000EFFF9DF800309DF80120134314D1582328
:106950008DF81630072480220021304827F046FDAC
:10696000224604A92D4827F0D7FD2C4A21460120B4
:10697000FFF740FC25B030BD0E23294601A8CDE924
:1069800001448DF81630ADF80C40FEF79FFF01ABC7
:1069900003CB234C1B88CDF81B10ADF81F30CDF86E
:1069A0001700FEF769FF2068FBF75EFD0A254FF42C
:1069B0007A7380B2B0FBF3F0B0FBF5F305FB130084
:1069C00030308DF821002068FBF74EFD642380B243
:1069D000B0FBF3F0B0FBF5F305FB130030308DF89E
:1069E00022002068FBF740FD80B2B0FBF5F0B0FB61
:1069F000F5F305FB130030308DF823002068FBF71A
:106A000033FD80B2B0FBF5F305FB130030308DF899
:106A1000240015249FE700BFD86D0308D81A002072
:106A2000F41800202DE9F047044694B0BD480D4607
:106A3000802200210DF08AFF2378592B40F04082FC
:106A4000052D5ED86378443B162B5AD8DFE813F047
:106A50007C01590059015900610159005900590040
:106A60005900BD0059004401590059005900D7018F
:106A700059005900E7005900590059001700A6783D
:106A8000482E17D1A84A14210120FFF7B3FB41F289
:106A90008830FDF7B5F80022A44B114603200DF015
:106AA00045FE40F6B830FDF7ABF814B0BDE8F0474E
:106AB000FFF7E4BA532E0DD1FFF71AFF41F28830E9
:106AC000FDF79EF8974A1521012014B0BDE8F04764
:106AD000FFF790BB432E17D1002404A88DF8104077
:106AE00005F01CFD8F4A4C231370102393709DF802
:106AF0001030547001204133D07013710521FFF71D
:106B000079FB14B0BDE8F087442EFAD1854C884D4E
:106B1000A670592323705A236370FFF7C9FE2868B3
:106B2000FBF77CFC0022834B0090114603200DF004
:106B3000FDFD7F220021601C27F058FC10232670E9
:106B40000126A370E6702671FCF7D8FFFE23B0FB88
:106B5000F3F000EB4000042300EB40106071A371E0
:106B60002868FBF781FC0A274FF47A7380B2B0FBE8
:106B7000F3F0B0FBF7F307FB13003030E071286847
:106B8000FBF772FC642380B2B0FBF3F0B0FBF7F3C9
:106B900007FB1300303020722868FBF765FC80B2D9
:106BA000B0FBF7F0B0FBF7F307FB13003030607277
:106BB0002868FBF759FC80B2B0FBF7F307FB130022
:106BC0003030A07222460B217EE7A378303BDBB247
:106BD000092B96D8584C594A23702378DBB253724C
:106BE000504A592313704D235370237803213033B7
:106BF00001209370FFF7FEFA237800930022504B98
:106C0000114601200DF092FDFFF774FB23780BB1C4
:106C1000FCF7ECFC14B0BDE8F047FCF785BDA578A7
:106C2000482D1BD13F4C562323701023A3701823EB
:106C30006371052301200025A37122460C2308213E
:106C4000E3716570E0702071FFF7D4FA3D4B00945A
:106C50002A46114602200DF069FD52E7432D7FF4CC
:106C600050AF00213C2205A82E4C049127F0BEFB1A
:106C700004A8FFF7B9FB9DF8103063709DF8113040
:106C8000A3709DF81230E3709DF8133023719DF8C6
:106C9000143063719DF81530A3719DF81630E371BF
:106CA0009DF81730257023729DF81B509DF8183001
:106CB00063729DF81930A3722A469DF81A30E37268
:106CC00007A904F10D00257327F026FC05F10D013D
:106CD0002246C9B2012012E7A07839280CD83038F2
:106CE000C0B2FEF73BFE0F4A2378137063785370EF
:106CF000A37893700321E7E614B0BDE8F047FFF7EF
:106D0000EBBAA0783928F7D83038C0B2FEF72BFE9E
:106D1000E9E7A0783928EFD83038C0B2FEF728FE6E
:106D2000E1E700BFD81A0020F16D0308066E0308E2
:106D3000F4180020286E03083819002040030020B2
:106D40004B6E0308746E0308A378303BDAB2092A4D
:106D5000D2D8E578303DEAB2092ACDD82179A1F11F
:106D60004802D2B20B2AC7D87A4840FA02F2D007BA
:106D7000C2D40A224D2902FB03553BD13C235D437B
:106D8000754B4FF47A7068431860744B1860FEF7C7
:106D900049FE734A2378137063785370A378937015
:106DA000E378D3700521237913710120FFF722FACC
:106DB0006C4B002610221E705A7001229A70DA70F5
:106DC000A178303901EB8100E178303901EB4001E5
:106DD000C9B2197122795A71634A1278D2B21A7201
:106DE000624A1278D2B25A72FFF784FA604B009569
:106DF00032462EE74829C3D14FF46163BFE7A37839
:106E0000303BDAB2092A3FF677AFE578303DEAB297
:106E1000092A3FF671AF2179A1F14802D2B20B2ABB
:106E20003FF66AAF4B4840FA02F2D2073FF564AF33
:106E30000A224D2902FB03553DD13C235D43474BBC
:106E40004FF47A7606FB05F21A601868FEF714FE16
:106E5000434A2378137063785370A3789370E37870
:106E6000D3700521237913710120FFF7C3F93D4B3E
:106E7000002710221F705A7001229A70DA70A178D0
:106E8000303901EB8102E178303901EB4201C9B2BE
:106E900099712279DA71344A1278D2B21A72334A6D
:106EA0001278D2B25A72FFF725FAB5FBF6F5314BDC
:106EB00000953A46CDE64829C1D14FF46163BDE75C
:106EC000502B40F0A881022D7FF61BAE6178A1F116
:106ED0003003012B3FF615AEA378312B7FF411AEB2
:106EE000052D4FD1E378302B40F0C4801E4D224E4B
:106EF00000232B702B7803F0FF0253B92379303B2A
:106F0000DBB233703378009311461C4B02200DF036
:106F10000DFC16491A4A00230B703378DBB213704C
:106F20002B78104ADBB213720B78DBB25372FFF787
:106F3000E1F90B4B22781A7062785A70A2789A7035
:106F4000E278DA7022791A71FCF7EEFB0521044A27
:106F5000BAE500BFDEF7FFFFFC0000208003002041
:106F6000D81A002040030020EE000020381900202D
:106F70009E6E0308D56E0308040000201F6F0308EF
:106F800005000020082D69D1E378462B40F0EC8005
:106F90002579A5F13000C0B2092800F23A81617963
:106FA000A1F13003092B00F23481A279A2F1300360
:106FB000092B00F22E81E379A3F13006092E00F2AD
:106FC000288105EB85067600B04D203601EB810166
:106FD000F6B249002E702031AD4E263AC9B2D2B277
:106FE000317002EB8202AB4903EB830352005B007A
:106FF0000A802033A84ADBB21370A84A82F828001E
:107000006379303BDBB282F82930A379263BDBB2CF
:1070100082F82A30E379303BDBB282F82B302B78D0
:107020002BB9337803F0FF020BB99D4B1A70FFF7B1
:1070300061F99C4B22781A7062785A70A2789A7023
:10704000E278DA7022791A7162795A71A2799A71AA
:10705000E279DA71FCF768FB082178E7042D2FD17B
:10706000E278A2F13003DBB2092B11D9A2F141037E
:10707000192B0AD9FFF730F900228B4B114601205A
:1070800014B0BDE8F0470DF051BBA2F13703DBB2FD
:1070900086480370834B207859703121187099709D
:1070A000DA70824B7D4A1B78DBB21372804B1B78FF
:1070B000DBB25372FFF71EF9FCF736FB042146E7FB
:1070C0001D2D4FD9A61C0025DFF8D091DFF8E4A1D3
:1070D0003746A84617F8012F303AD2B2092A3ED8CF
:1070E00009EB050303201A731B7BCDE902533B78A0
:1070F0000022CDE90053114653460DF017FB013530
:107100001E2DE7D1B8F1000FB4D1FEF711FA654B8F
:1071100050221A7000225A7010229A700122DA70DE
:1071200003F8042F203416F8012F03F8012FB4427E
:10713000F9D15A4B00221A7010225A7001229A700B
:10714000DA705A4A1278D2B21A72594A1278D2B206
:107150005A721E22DA72FFF7CDF82321F7E64FF0BC
:107160000108CCE7072D85D900254C4FDFF8448175
:1071700002342E4614F8012F303AD2B2092A46D8EA
:10718000791903200A730B7BCDE90253237800227F
:10719000CDE90053114643460DF0C8FA0135082DDC
:1071A000E8D1002E7FF466AFFEF734FA3D4B3B4C3E
:1071B00050221A7010229A70002501225D70DA7038
:1071C00003F8042F62190135127B082D02F13002F9
:1071D00003F8012FF6D1002250231146009301201D
:1071E000354B0DF0A3FA00232370102363700123A5
:1071F000A370E3702D4B1B78DBB223722C4B1B78F2
:10720000DBB26372E572FFF775F80D219FE6012688
:10721000C4E700219BE6412B7FF473AC6378432BDA
:107220007FF46FAC162D7FF46CAC244D621C0023F0
:1072300012F8011FE9540133142BF9D1FEF79AF823
:107240001F4B5B7D012B1DD114490023EA5CC8183C
:107250000133D2B2142B80F82C20F7D1144B00222A
:107260001A701B78DBB24B72FFF744F80D4A631EAD
:10727000153413F8011F02F8011B9C42F9D1094A89
:10728000162121E40A4B02221A70EFE78B0300203B
:107290008A030020240000208903002040030020EE
:1072A00088030020D81A00207E6F0308EE0000201B
:1072B000381900203B6F0308636F03085D1B002033
:1072C0009409002070B5054688B00C46002951D0BD
:1072D00033480DF0A5FD26789EB3002D5ED068687A
:1072E0002E7870B3032E0BD0132E45D0022E28D14A
:1072F0006978012925D00B0623D4FFF793FB20E002
:107300006B78012B07D10078012802D0022800D029
:1073100008B905F0BDF800250DF11F008DF81F50CC
:1073200005F0FCF81F4A4C231370102393709DF84E
:107330001F305570012041330521D0701371FEF7C5
:1073400059FF237C052B15D894F90A20059294F94E
:1073500009200492144A52F82330039394F9083018
:10736000CDE901630022E368009311460F4B03202F
:107370000DF0DCF908B070BD6B78012BE1D102781B
:107380000B4B02F001021A702AB90A4B1146032076
:107390000DF0CCF9D5E7084B0022F7E72E46D0E7F1
:1073A00084190020D81A002008700308B66F03085B
:1073B000B4190020A36F0308AD6F0308034B00222C
:1073C000C3E902220122C3E900227047741B002096
:1073D00000487047741B00204FF0B04382B0DA6C55
:1073E0000243DA64DB6C03400193019B02B07047F7
:1073F0002DE9F04186B000240220154D0594FFF7D9
:10740000EBFF0420FFF7E8FF124F03944FF4807660
:1074100001230DEB0001CDE901632846032304930A
:107420004FF4005801F04AF801A93846CDF804801D
:1074300001F044F822464146384601F065F92846F5
:107440002246314601F060F9204606B0BDE8F081E1
:107450000004004800080048032810B50ED8012891
:1074600010D868B902460B484FF4807101F04CF90E
:10747000002209484FF4005101F046F9002010BDE8
:107480000122F0E7002203484FF4807101F03CF93B
:107490000122EEE70004004800080048022070477F
:1074A0000020704701207047002814BF16200F20CD
:1074B000704700000D48854600F025F80C480D493E
:1074C0000D4A002302E0D458C4500433C4188C423F
:1074D000F9D30A4A0A4C002301E013600432A242A5
:1074E000FBD326F0EBFFFBF70BFEFEE700000120CD
:1074F00000000020B0070020E8D50308B0070020F6
:10750000103B0020FEE7704710B5032000F06EFC32
:1075100001F07CFA064B18600F20FCF767FB04466D
:1075200018B9FBF761FF204610BD0124FBE700BF3F
:107530008C0300204FF0E022136923F00203136153
:1075400070474FF0E022136943F002031361704764
:10755000014BD3F8900570470070FF1F014BD3F823
:10756000940570470070FF1F014BD3F898057047D2
:107570000070FF1F024A536843F0010353607047D5
:10758000002004E0024A536843F00203536070474E
:10759000002004E0024A536843F00403536070473C
:1075A000002004E08068C0F380007047F7B5002336
:1075B00001930446002800F0E980856D25B9FBF7AA
:1075C00029FAE56584F8545023689A68D00040F1A0
:1075D000A1809A68D10000F1B480A26D42F010023F
:1075E000A265E26D42F00102E26501251846FFF74F
:1075F000D9FFA26D02F01002024340F0C980A26DD3
:10760000206922F4817242F00202A2659A68D207D0
:107610005DD4226BA67E94F82CC0003A18BF0122DC
:107620001703D4E902120A43217E42EA8132617EC5
:1076300042EAC13242EA4632002842EA4C02B4BF72
:1076400020F000414FF400113A430A4394F820100F
:10765000012903D1002E76D142F48032616A21B132
:10766000A66A01F4E07131430A43D968E66C21F45B
:10767000FE3121F4FF711143D96094F83C20616818
:10768000012A01F0404C4CEA060609D1D4E9102742
:107690003A433243A66C324342EA0C0242F00106FE
:1076A0001F693E4A3A4032431A6121F00042B2F16A
:1076B000804F0CD0B1F1004F09D0394ED6F80827D1
:1076C00001F4701122F470120A43C6F808275A69AF
:1076D000666BA16B22F0070232435A615A6922F0AD
:1076E000700242EA01125A61002835D19A6A62F0AA
:1076F0000F029A625B6903F007039E423CD10023AC
:10770000E365A36D23F0030343F00103A36528465B
:1077100003B0F0BD9A68234922F0104222F017020C
:1077200042F080529A60204A1268B2FBF1F20132B4
:1077300052000192019A002A3FF44BAF019A013A9C
:10774000F7E7002552E7A16D41F02001A165E16D49
:1077500041F00101E16581E7B0F5001FCAD19A6AE5
:10776000E269013A92006FF00F0102F01C0201FA87
:1077700002F2216E0A43BCE7A36D23F0120343F02B
:107780001003A365E36D43F00103E3650125BEE744
:10779000A36D43F01003A365F8E700BF02FCFF1FD1
:1077A00000200140400D03008C030020F8B545691E
:1077B000082D04460E460AD00368DB68D80705D5B5
:1077C000A36D43F02003A3650120F8BD0425FCF759
:1077D0000FFA074623681A682A4220D0A26D42F4A5
:1077E0000072A265DA6812F4406F14D1A27E92B9D9
:1077F0001A6812070FD51846FFF7D4FE20BB5A6847
:1078000022F00C025A60A26D22F4807222F0010272
:1078100042F00102A265227EFAB10020D5E7711C78
:10782000D9D0FCF7E5F9C01BB04201D8002ED1D168
:1078300023681B682B40CDD1A26D84F8543042F0F0
:107840000402A2650320C0E7A26D42F02002A265F7
:10785000E26D42F00102E265DDE70C221A60DCE72E
:107860000368186C70470000F7B50023019390F887
:107870005430012B044600F0C080056802690123E2
:1078800080F854302846FFF78DFE002840F0AF8086
:10789000D1E90030022822F004027ED0B2F1004F7C
:1078A000C3F3110E35D1AA6A42EA0E02AA628A68AF
:1078B000686902EA032222F07C4222F0FF0220EAF9
:1078C00003210A43002B6A611DDA4D4A4D4DD2F85F
:1078D0000817AB4201F0E07043D10D0213D4D2F887
:1078E000083723F0E073034343F40003C2F808377A
:1078F000454B1A68454BB2FBF3F20C2302FB0333F2
:107900000193019B53BB0020002384F8543003B043
:10791000F0BD226E00F01F074FF00F0C0CFA07FCB1
:107920006FEA0C0622EA0C0CBEF1000F11D1C3F372
:107930008462BA4042EA0C0222668008E2690130A1
:107940009042B4D8A86AC3F38362BA400640324377
:10795000ACE793FAA3F2B2FA82F2EAE7019B013BA9
:10796000CEE72B4DAB420BD1C901CCD4D2F80837AE
:1079700023F0E073034343F08073C2F80837C2E793
:10798000244DAB42BFD14B02BDD4D2F8083723F00F
:10799000E073034343F48003EFE7B2F1004F01BF0C
:1079A000AA6AC3F311018A43AA62002BABDA154815
:1079B00013498342D1F8082709D1D1F8083702F0DA
:1079C000A07223F0E0731A43C1F808279BE7104820
:1079D000834204D1D1F8083702F44002F1E70D48A0
:1079E000834290D1D1F8083702F0C072E9E7A26D66
:1079F00042F02002A265184686E7022087E700BF12
:107A000000200140001000B08C030020400D030056
:107A1000004000B8002000B4026838B504461046A3
:107A2000FFF7C0FD08B9002038BD9368990707D457
:107A3000936823F0004323F0170343F0100393608F
:107A4000FCF7D6F8054623689B685B07EBD5FCF787
:107A5000CFF8401B0228F6D923689B685A07F2D555
:107A6000A36D43F01003A365E36D43F00103E365E9
:107A70000120D9E773B50023026801939368DD07FD
:107A8000044602D5002002B070BD9168214B194216
:107A900009D0A36D43F01003A365E36D43F0010328
:107AA000E3650120EFE7936823F0004323F0170319
:107AB00043F001039360184BD3F8083718021CD425
:107AC000637E012BDED0FCF793F8144E0546226846
:107AD0001368DB07D6D49368D9075FBF9368334038
:107AE00043F001039360FCF783F8401B0228EED9B2
:107AF00023681B68DA07EAD4CBE7094B094A1B68FD
:107B0000B3FBF2F301330193019B002BD8D0019B0F
:107B1000013BF8E71700008000200140E8FFFF7FED
:107B20008C030020400D030038B504460068FFF7C1
:107B300039FD054620BB94F85430012B20D0012399
:107B400084F854302046FFF795FFB0B9A36D226842
:107B500023F4706323F0010343F48073A3651C23B3
:107B6000E065136084F85400936823F0004323F029
:107B7000170343F00403936038BD84F85450FBE7C7
:107B80000220F9E7026838B5936891680446C8078F
:107B900001D4002038BD9907FBD4936803F0050396
:107BA000012B19D1936823F0004323F0170343F00E
:107BB0000203936003231360FCF71AF80546236859
:107BC0009B68DB07E5D5FCF713F8401B0228F6D9C4
:107BD00023689B68DA07F2D5A36D43F01003A36511
:107BE000E36D43F00103E3650120D3E770B504467C
:107BF00000284BD0836D43F002038365FFF70CFF31
:107C0000054668B92046FFF7BDFF054608B90123C0
:107C1000A3652268936823F0104323F01703936051
:107C200023685A6822F4677222F003025A6040F215
:107C30009F321A60D968164A0A40DA601A6922F03F
:107C400040421A615A6922F007025A611A6A02F028
:107C5000F0221A625A6A02F0F0225A62DA6A02F0DC
:107C6000F022DA629A6A0B4A00269E62D2F808373E
:107C700023F0FE73C2F808372046FAF7DFFEE66508
:107C80002666A66584F85460284670BD0125FBE78A
:107C900000023E830020014010B590F85430012BC3
:107CA000044615D0012380F85430FFF7B5FE58B9CB
:107CB0002046FFF767FF38B9A36D23F4807323F0E4
:107CC000010343F00103A365002384F8543010BD81
:107CD0000220FCE7F7B50023019390F85430012B04
:107CE00004467FD0012380F85430FFF74BFF236810
:107CF0009A6812F00102054607D0A36D43F0100305
:107D0000A365002384F854302DE0A16D364F21F493
:107D1000817141F00201A165DE68D96826F4FF4651
:107D200026F07C0621F40041360421F00301360CD4
:107D3000D96008209968394041F0004199609968FC
:107D4000002913DA0199013101910199B1F52E3F12
:107D5000F5D3A36D23F0120343F01003A3650023B2
:107D600084F854300125284603B0F0BDD3F8B41090
:107D7000013801F07F010A44DCD199681A480140BA
:107D800041F001019960D3F8B41021F07F0141EA7C
:107D9000D202C3F8B4209A68024042F002029A600C
:107DA000FBF726FF074623689A68D20708D4DA68EB
:107DB0003243DA60A36D23F0030343F001039FE72E
:107DC000FBF716FFC01B0228EDD923689B68D90773
:107DD000E9D5A36D43F01003A365E36D43F0010300
:107DE000E365BFE70225BEE7E8FFFF7F0749CA68F2
:107DF00022F4E0620302120403F4E063120C134362
:107E000043F0BF6343F40033CB60704700ED00E004
:107E1000164B30B5DC68C4F30224C4F10703251DFA
:107E2000042B28BF0423062D4FF0FF358CBF033CE5
:107E3000002405FA03F321EA0303A54022EA050220
:107E4000A340002843EA0203ACBF00F16040084AA7
:107E50004FEA0313B8BF00F00F00DBB2AABF00F572
:107E60006140135480F8003330BD00BF00ED00E0E6
:107E700014ED00E0002807DB044A4109012300F06B
:107E80001F00834042F82130704700BF00E100E04E
:107E900000280CDB4309064900F01F0020330122B3
:107EA000824041F82320BFF34F8FBFF36F8F70479D
:107EB00000E100E070B5D0E913456560446D14B190
:107EC000D0E916456560D0E9105404F01C06012481
:107ED000B4406C60046863608368102B0BBFA260C1
:107EE000A160E160E26070BD0268416CD3B210B580
:107EF000083B1424B3FBF4F30B4CA24288BF0B4A9B
:107F000021F0030199BF01F1804202F502325218BB
:107F100007338264064AC26403F01F03012202FA97
:107F200003F3036510BD00BF070402401C080240B4
:107F30008008024038B500285CD002682E4B9A4277
:107F40004FF014014AD82D4B1344B3FBF1F32C49E5
:107F50009B00C0E91013022380F8253013680569DF
:107F600023F4FF4323F070031360D0E9024323435B
:107F70002B43456911682B4385692B43C5692B4306
:107F8000056A2B430B431360FFF7AEFFB4F5804F38
:107F900004BF002343604368816C03F07F020A60E2
:107FA000D0E91314013B032B4C601ED8154B164926
:107FB000816513449B000121013A01FA02F200217C
:107FC0004365C2651960114B5A6400230122C363E3
:107FD00080F8243080F82520184638BD0C4B134417
:107FE000B3FBF1F30B499B00B3E70023C0E9153362
:107FF000C365EAE70120F0E707040240F8FFFDBF90
:10800000000002403F820010400902400009024087
:10801000F8FBFDBF0004024038B5002841D00268DB
:10802000136823F0010313601F4B9A424FF01401B1
:1080300030D81E4B1344B3FBF1F31D499B00C0E93C
:108040001013012403F01C0304FA03F30025156048
:108050004B60FFF749FF836C41681D60D0E9133224
:108060005A604A1E032A06D8124B0B449B009440C8
:108070001D60114B5C640023C363C0E91533C0E984
:108080000B33C0E90D33C36580F8253080F8243008
:10809000184638BD094B1344B3FBF1F308499B0064
:1080A000CDE70120F5E700BF07040240F8FFFDBF60
:1080B000000002403F82001000090240F8FBFDBFB3
:1080C0000004024070B590F82450012D04463BD0C6
:1080D00090F825600125AE4280F824504FF000064C
:1080E0002CD1022580F825500568C6632E6826F03D
:1080F00001062E60FFF7DEFE036BBBB12B6843F079
:108100000E032B60A36C1A68D20342BF1A6842F4B4
:1081100080721A60636D1BB11A6842F480721A6033
:108120002B6843F001032B60002070BD2B6823F007
:1081300004032B602B6843F00A03E2E78023C36348
:1081400080F824602846F0E70220EEE7034640B1BD
:1081500090F82520022A06D00422C263002280F86B
:108160002420012070470268806C116821F00E0104
:108170001160016821F480710160116821F0010132
:108180001160D3E9100202F01C0101228A40426012
:10819000D3E9132151605A6D32B1116821F4807115
:1081A0001160D3E9162151600122002083F82520B7
:1081B00083F82400704708B590F82530022B03D0CF
:1081C0000423C363012008BD03681A6822F00E026D
:1081D0001A601A6822F001021A60826C136823F494
:1081E00080731360D0E9101303F01C020123934045
:1081F0004B60D0E913325A60436D33B11A6822F4F0
:1082000080721A60D0E916325A60012380F8253056
:10821000002380F82430836B03B198470020D2E715
:1082200070B4426C046C036826681D6802F01C027E
:108230000421914031420FD015F0040F0CD01A6880
:1082400092065EBF1A6822F004021A60036B616036
:10825000002B33D070BC184702219140314217D017
:1082600015F0020F14D01A68940606D41A6822F08A
:108270000A021A60012280F82520114A93428CBF1D
:10828000104B114B5960002380F82430C36ADFE79C
:1082900008219140314211D029070FD5196821F0EA
:1082A0000E011960012303FA02F26260C36380F8D1
:1082B0002530002380F82430436BC9E770BC704739
:1082C0008000024000040240000002400A4A536954
:1082D00043F4802330B55361EFF3108472B600236A
:1082E000CD58C5500433B3F5807FF9D11369DB0352
:1082F000FCD484F3108830BD00400058064B5A6906
:10830000002ABFBF054A9A6002F188329A60BABF5C
:108310005869C00F0020704700400058230167458E
:10832000044B5A6942F000425A615869C043C00F79
:10833000704700BF0040005870B50546FBF758FC79
:10834000124E04463369D90313D43369DA0744BFA4
:10835000012232614CF2FA32134011D10B4E3069D6
:1083600010F480200BD0FBF743FC001BA842F6D38F
:1083700004E0FBF73DFC001BA842E3D3032070BDE3
:10838000024A1361024A01205360F8E70040005896
:10839000841B00202DE9F041184D98462B78012BC5
:1083A00006460C46174626D001232B704FF47A70F0
:1083B00000236B60FFF7C0FFA0B9012E16D1104A51
:1083C000536943F0010353612760BFF36F8FC4F813
:1083D00004804FF47A70FFF7AFFF094A536923EA2C
:1083E0000603536100232B70BDE8F0813946204617
:1083F000FFF76CFFEDE70220F6E700BF841B0020CB
:1084000000400058054A536923F47E7343EAC000D4
:1084100040F4803040F00200506170470040005846
:108420002DE9F041234F3B78012B054688463FD08C
:1084300001233B704FF47A7000237B60FFF77CFFD1
:10844000044688B92B68042B13D11B4A536943F4A3
:10845000803343F0040353614FF47A70FFF76CFFED
:108460000446154B1A681B6800233B702046BDE884
:10847000F0814FF0FF33C8F800306E68D5E9013263
:108480001344B3420AD93046FFF7BCFF4FF47A7069
:10849000FFF752FF50B1C8F800600446064A53691E
:1084A00023F47E7323F002035361DAE70136E5E734
:1084B0000224DBE7841B0020004000582DE9F04F28
:1084C000524C00234FF00F090A6832FA03F501D12C
:1084D000BDE8F08F012505FA03F818EA020200F062
:1084E0008E804E68032706F003054FEA430E07FA15
:1084F0000EFC6F1E012F6FEA0C0C32D8876807EA5A
:108500000C0ACF6807FA0EF747EA0A078760476840
:1085100027EA0808C6F300179F4047EA08074760A4
:10852000C76807EA0C088F6807FA0EF747EA0807DA
:10853000022DC76017D14FEAD30800EB880803F07B
:10854000070AD8F820704FEA8A0A09FA0AFB27EAD4
:108550000B0B0F6907FA0AF747EA0B07C8F82070F8
:1085600001E0032DDCD1076805FA0EF507EA0C07D8
:108570003D4316F4403F056041D023F0030707F167
:10858000804707F5803703F0030CBD684FEA8C0C79
:108590004FF0070E0EFA0CFEB0F1904F25EA0E0ECA
:1085A0002FD01B4DA8422ED005F58065A84214BFE0
:1085B0000725022505FA0CF545EA0E05BD6025687C
:1085C000D74316F4801F0CBF3D40154325606568F6
:1085D00016F4001F0CBF3D4015436560D4F8805071
:1085E00016F4803F0CBF3D401543C4F88050D4F8CA
:1085F0008450B60354BF3D401543C4F88450013342
:1086000062E70025D6E70125D4E700BF000800583F
:1086100000040048374A2DE9F04F00234FF0010ACB
:108620004FF0070B4FF00F0931FA03F401D1BDE809
:10863000F08F0AFA03FC1CEA010654D023F003046D
:1086400004F1804404F5803403F00307A568BF00FB
:108650000BFA07F8B0F1904F08EA050E45D0264D09
:10866000A84244D005F58065A8420CBF0225072525
:10867000BD40754517D1D2F8805025EA0605C2F8ED
:108680008050D2F8845025EA0605C2F88450156857
:1086900025EA06051560556825EA06055560A568B2
:1086A00025EA0805A560056803265C0006FA04F4BF
:1086B00023FA06F6254300EB8606056003F007055E
:1086C000376AAD0009FA05F527EA050737628568BC
:1086D00025EA04058560456825EA0C054560C568FE
:1086E00025EA0404C46001339EE70025C0E70125A4
:1086F000BEE700BF000800580004004803691942A3
:1087000014BF0120002070470AB181617047816267
:108710007047436901EA030221EA030141EA024189
:1087200081617047044AD168014208B502D0D06027
:10873000FDF7ECFC08BD00BF00080058024A1368B2
:1087400043F4807313607047000400580D4B10B55C
:108750005B690C4628B99A0507D500F027F820B1C7
:1087600010BD9B0501D400F019F8074A1369012CCC
:1087700023F00403136101D130BFF1E740BF20BFF4
:1087800020BFEDE70004005800ED00E0024B186840
:1087900000F4C060704700BF00040058024A13682C
:1087A00043F4804313607047000400580C4A136878
:1087B00023F4804313600B4B1B6832214B430A495F
:1087C000B3FBF1F35169890500D533B9536913F44B
:1087D000007F14BF032000207047013BF2E700BF79
:1087E000000400588C03002040420F000B4A13681D
:1087F00023F0070343F002031360094B1A690128B1
:1088000042F004021A6105D130BF1A6922F0040255
:108810001A61704740BF20BF20BFF6E70004005830
:1088200000ED00E04FF0B0431868C0F340407047DF
:108830004FF0B0431868C0F3400070474FF0B042AB
:10884000536823F47F4343EA0023536070474FF09B
:10885000B0431868C0F34060704700007FB54FF028
:10886000B0432C4AD3F80831C0F3031003F00F03D0
:1088700052F82040284A52F82330B4FBF3F4FFF7B3
:1088800085FF264B054693E80700B5F5007F04AB4E
:1088900003E9070010D0224B9C4218D303F5B7031D
:1088A00003F67F539C4229D903F5741303F5106333
:1088B0009C4225D802230BE01A4B9C4207D91A4B45
:1088C0009C421BD903F5370303F5D853F0E7002387
:1088D00004AA02EB830353F80C4C144D2B6823F0CD
:1088E000070323432B60FBF783F906462B6803F04D
:1088F00007039C4206D1002004B070BD0123E7E7C6
:108900000024EAE7FBF774F9801B0228EED9032064
:10891000F2E700BF2070030880700308D81903082D
:10892000C0CF6A00BFEA21013F93340200400058E3
:108930004FF0B04310B59A68D96812F00C0205D018
:108940000C2A4AD101F00303012B51D14FF0B04161
:108950002B480B6813F0080306D00B6813F00803CC
:1089600037D1D1F8941007E00C68240756BFD1F82E
:1089700094300968C3F3032350F82330002A0CBF56
:10898000184600204FF0B0418A6802F00C020C2A11
:108990001ED1CA6802F00302022A2ED0032A06D191
:1089A0000B68184A13F4801F174B18BF13464FF07B
:1089B000B042D068D168D268C0F306205843C1F3F2
:1089C00002130133B0FBF3F0530F0133B0FBF3F0AC
:1089D00010BD0B68C3F30313CEE7042A05D0082AA1
:1089E00006D11B6813F4801305D006480023C9E79D
:1089F00000231846C6E70448C4E7024BD7E700BF88
:108A0000207003080024F4000048E80108B5FFF7CF
:108A10008FFF4FF0B043044A9B68C3F3031352F82F
:108A20002330B0FBF3F008BD807003082DE9F0415E
:108A30000446002853D04FF0B0439D68DE680368B9
:108A40009B0605F00C0506F0030668D5026A1DB109
:108A50000C2D46D1012E44D1002A40D04FF0B04316
:108A6000A16A1A68170756BFD3F894301B681B0910
:108A700003F0F00399421FD90846FFF7EFFE0028E4
:108A80002DD14FF0B042136843F008031360136810
:108A9000A16A23F0F0030B431360606AFFF7CEFE78
:108AA000FFF7B4FFAB4B1860AB4B1868FBF79EF8B1
:108AB000002834D0BDE8F0814FF0B042136843F095
:108AC00008031360136823F0F0030B431360606A1C
:108AD000FFF7B4FE0846FFF7C1FE0028E0D00120F2
:108AE000E8E74FF0B043002A54D01A6842F0010280
:108AF0001A60FBF77DF80746FFF79AFE002842D080
:108B00004FF0B042136843F0080313601368A16A82
:108B100023F0F0030B431360606AFFF78FFE2368B6
:108B2000D80748D42368990700F18C8023681E0772
:108B300040F1FA80A3694FF0B046002B00F0E180CD
:108B4000D6F89430E16903F01002914200F0C4803D
:108B500003F00302022AC2D0D80740F1B380D6F84E
:108B6000943023F00103C6F89430FBF741F8074630
:108B7000D6F89430990740F1A580FBF739F8C31B6C
:108B8000112BF5D904E0FBF733F8C01B0228B3D949
:108B900003208FE71A6822F001021A60FBF728F819
:108BA0000746FFF745FE0028B9D0FBF721F8C01BA8
:108BB0000228F6D9ECE7082D03D00C2D05D1032EA1
:108BC00003D16368002BADD189E74FF0B043A168B2
:108BD0001A6822F480120A431A606268B2F5803F74
:108BE00010D11A6842F480321A60FBF701F8074688
:108BF000FFF718FE002895D1FAF7FAFFC01B64288A
:108C0000F6D9C5E7B2F5041F04D11A6842F4001280
:108C10001A60E6E7196821F480311960196821F4B7
:108C200000111960002AE0D1FAF7E2FF0746FFF7CA
:108C3000F9FD00283FF476AFFAF7DAFFC01B64288D
:108C4000F5D9A5E7042D236903D00C2D0ED1022EF2
:108C50000CD1002B3FF443AF4FF0B0426169536831
:108C600023F0FE4343EA016353605FE74FF0B046F1
:108C7000BBB1336843F480733360FAF7B9FF07463A
:108C800033685A0505D4FAF7B3FFC31B022BF7D993
:108C90007EE77368626923F0FE4343EA0263736010
:108CA00044E7336823F480733360FAF7A1FF074683
:108CB00033685B057FF53AAFFAF79AFFC31B022BC7
:108CC000F6D965E74FF0B042E169D2F8943023F06D
:108CD00010030B43C2F894304FF0B047D7F89430EC
:108CE00043F00103C7F89430FAF782FF0646D7F83D
:108CF00094309A0718D4FAF77BFF831B112BF6D90F
:108D000046E7D6F8943023F00103C6F89430FAF71A
:108D10006FFF0746D6F894309B0705D5FAF768FF32
:108D2000C31B112BF6D933E72368580754D50B4FD3
:108D30003B68D90514D4FFF701FDFAF759FF064641
:108D40003B68DA050CD4FAF753FF831B022BF7D9E3
:108D50001EE700BF8C030020900300200004005891
:108D6000E3684FF0B046002B58D023F08003052B6A
:108D700002BFD6F8903043F00403C6F890304FF0AD
:108D8000B046FAF735FFD6F8903043F001030746B6
:108D9000C6F8903041F28838D6F890309B0705D459
:108DA000FAF726FFC31B4345F6D9F1E6E36823F043
:108DB0000403812B1BD1FAF71BFFD6F8903043F048
:108DC0008003C6F8903007464FF0B04641F288382D
:108DD000D6F89030180504D5E36A002B4AD100205C
:108DE00068E6FAF705FFC01B4045F1D9D0E6FAF76F
:108DF000FFFED6F8903023F08003C6F89030074687
:108E00004FF0B04641F28838D6F890301905E3D5D6
:108E1000FAF7EEFEC01B4045F6D9B9E6FAF7E8FED0
:108E2000D6F8903023F080030746C6F8903041F220
:108E30008838D6F890301A0516D4FAF7D9FED6F845
:108E4000903023F00103C6F8903007464FF0B04849
:108E500041F28836D8F890309B07BDD5FAF7C8FEA6
:108E6000C31BB342F6D993E6FAF7C2FEC01B4045D6
:108E7000DFD98DE60C2D4ED0022B4FF0B0431A688F
:108E800022F080721A6033D1FAF7B2FE0546FFF77E
:108E9000DEFC38BBD4E90C314FF0B0420B43D06854
:108EA0002D4901400B43E16B0B43216C0B43616C7B
:108EB0000B43A16B43EA0123D360136843F0807333
:108EC0001360D36843F08053D360FAF791FE0446F1
:108ED000FFF7BDFC002882D1FAF78AFE001B0A28A2
:108EE000F6D955E6FAF784FE401B0A28CFD94FE69B
:108EF000FAF77EFE0446FFF7AAFC30B94FF0B04205
:108F0000164BD1680B40D36069E7FAF771FE001B7E
:108F10000A28F0D93CE6012B3FF4E1AD4FF0B04315
:108F2000D868236B00F003029A427FF4D8AD626BDD
:108F300000F0700393427FF4D2ADA26B00F4FE43C5
:108F4000B3EB022F7FF4CBAD636C00F06040C01A2E
:108F500018BF0120AEE500BF8C80C111FCFFFEEE02
:108F60002DE9F0410D46044610B90120BDE8F0811D
:108F7000684E336803F007038B4216D323689A07C1
:108F800027D54FF0B047A268BB6823F0F003134326
:108F9000BB60FAF72DFE0646BB68DB0319D4FAF76F
:108FA00027FE831B022BF7D911E0336823F0070358
:108FB0000B433360FAF71CFE0746336803F00703E0
:108FC000AB42DBD0FAF714FEC01B0228F5D9032010
:108FD000CCE72368580617D54FF0B0476269D7F839
:108FE000083123F00F0343EA1213C7F80831FAF7E8
:108FF000FFFD0646D7F80831D90305D4FAF7F8FD86
:10900000831B022BF6D9E2E723685A0713D54FF0EA
:10901000B047E268BB6823F4E0631343BB60FAF730
:10902000E7FD0646BB689B0305D4FAF7E1FD831B09
:10903000022BF7D9CBE72368180714D54FF0B047B8
:109040002269BB6823F4605343EAC203BB60FAF7AA
:10905000CFFD0646BB68590305D4FAF7C9FD831B4B
:10906000022BF7D9B3E72368DA070FD4294C23681A
:1090700003F00703AB4239D8FFF7C8FC264B186052
:10908000264BBDE8F0411868FAF7B0BD6268022AC5
:109090001DD1FFF7C7FB00283FF467AF4FF0B04684
:1090A00041F28838B36823F003031343B360FAF73F
:1090B0009FFD0746B368626803F00C03B3EB820FB1
:1090C000D4D0FAF795FDC01B4045F3D97FE7032ABA
:1090D00002D1FFF7BCFBDEE712B9FFF7A9FBDAE725
:1090E0004FF0B0431B685B05D8D43EE7236823F0FC
:1090F00007032B432360FAF77BFD0646236803F042
:109100000703AB42B8D0FAF773FD801B0228F5D9EC
:109110005DE700BF004000588C0300209003002052
:1091200008B5FFF773FC4FF0B043044A9B68C3F3E4
:10913000022352F82330D84008BD00BF60700308F6
:1091400008B5FFF763FC4FF0B043044A9B68C3F3D4
:10915000C22352F82330D84008BD00BF6070030816
:109160004FF0B043D3F89000C0F3400070474FF089
:10917000B0410209D1F8883002F47F22000123EACD
:10918000020300F47F200343C1F8883070474FF09A
:10919000B041020CD1F88830120423EA020343EAFA
:1091A0000040C1F8880070470368DA0370B50446D0
:1091B00039D5FFF7C3FAFAF71BFD614E0546336850
:1091C000DB0532D54FF0B043616BD3F8902002F449
:1091D000407291421DD0D3F89010D3F8902042F401
:1091E0008032C3F89020D3F8902021F4407022F40C
:1091F00080328D07C3F89020C3F8900009D5FAF7A4
:10920000F7FC41F288360546FFF7AAFF012840F037
:1092100090804FF0B042616BD2F8903023F44073ED
:109220000B43C2F89030002605E0FAF7E1FC401B42
:109230000228C4D903262568E8070AD54FF0B041B3
:109240006268D1F8883023EA124392B21343C1F81E
:109250008830A9070AD54FF0B041A268D1F888300C
:1092600023EA124392B21343C1F88830AA0609D503
:109270004FF0B0422169D2F8883023F440630B43A9
:10928000C2F88830AB0502D5206AFFF780FF680579
:1092900002D5606AFFF77BFF290502D5A06AFFF7B8
:1092A00076FF6A0602D56069FFF761FF2B0602D5DB
:1092B000A069FFF75CFFE80502D5E069FFF757FFFB
:1092C000E90610D54FF0B042E168D2F8883023F4B7
:1092D00040730B43C2F88830B1F5807F02BFD3687A
:1092E00043F08073D3602A040ED54FF0B042216B57
:1092F000D2F8883023F040430B43C2F8883019B9C4
:10930000D36843F08073D3606B0410D54FF0B04244
:10931000E16AD2F8883023F040530B43B1F1005F8B
:10932000C2F8883003D1D36843F48033D360304629
:1093300070BDFAF75DFC401BB0427FF665AF79E780
:109340000004005830B590F82C30012B02464FF045
:10935000020022D0174B82F82D00CA24012582F882
:109360002C505C6253245C62B1F5807F146B996968
:1093700014D121F488519961596C24F0010421F031
:10938000004159641463DD650A4BFF2159620020D6
:10939000012382F82D3082F82C0030BD21F40851D1
:1093A0009961D96C24F0020421F00041D96414635E
:1093B000D865E9E70028004070B50B4E036B756D6A
:1093C0001D40EA07044603D50123F365FAF785FE3D
:1093D000AB0704D50223F365204600F0C9F9012349
:1093E00084F82D3070BD00BF0028004038B50A4C0D
:1093F000E36823F02003E360FAF7FAFB0546E3682D
:109400009B0601D5002038BDFAF7F2FB401BB0F5F2
:109410007A7FF4D90320F6E700280040F8B5114D13
:10942000EC6814F0400406461AD1EB6843F0800360
:10943000EB60FAF7DDFB23460746EC6814F04004C6
:1094400001D1032B01D11846F8BDFAF7D1FBC01B9F
:10945000B0F57A7F234684BF032386F82D30ECE7EE
:109460000023F0E70028004038B50F4CE36823F0F4
:109470008003E360A3699B06054606D4FFF7B6FFA9
:1094800010B1032085F82D0038BDA36923F0200317
:10949000A361FFF7ABFF10B1032085F82D00A3698E
:1094A00043F02003A361EFE70028004038B50446ED
:1094B00000284BD090F82D3003F0FF021BB980F844
:1094C0002C20F9F775FE0223214D84F82D30EB682E
:1094D000DB0636D4CA236B6253236B622046FFF748
:1094E0009DFF10B1FF236B6238BDAB6923F08E6323
:1094F00023F04003AB6121696368AA690B431343FE
:10950000A2691343AB61D4E9022343EA02432B610E
:10951000D4E90931EA680B4322F4F8521343EB60B3
:109520002046FFF7A1FF0028DCD1D4E90713AA6980
:109530000B4322F06042134362691343AB61FF2384
:109540006B62012384F82D300020CDE70120CBE7AA
:10955000002800400023092803D840EA0310C0B2C5
:1095600070470A380133C0B2F5E700002DE9F04733
:1095700090F82C30012B05464FF0020069D00123F2
:1095800085F82C304E4B85F82D00DE6806F44076C9
:10959000B6F5807F78D04C69087891F8019091F801
:1095A00002A091F82470002A55D19B6913F0400362
:1095B00008BFCB70FFF7CEFF80464846FFF7CAFFD3
:1095C00002465046FFF7C6FF81463846FFF7C2FF06
:1095D0000B6ACF78234343EA875343EA090343EAFC
:1095E000084343EA022343EA0063354ACA20506233
:1095F000532050628C6A8869B4F5807F946945D1A4
:1096000024F4885494610124D465B6F5807F09BFA1
:10961000CB6913640343536418BF5064284B4A68F2
:109620001A672A6B42F001022A639A6942F488524F
:109630009A61244AD2F8803043F40033C2F8803073
:109640001F4BFF225A620020012385F82D3085F838
:109650002C00BDE8F087B4F1803F07D0B4F5000FCF
:1096600004D09B6913F0400308BFCB700B6ACA7823
:109670001C4344EA0A0444EA004343EA092343EA58
:10968000825343EA0763B0E70023AEE724F40854AB
:1096900094610224D465B6F5807F09BFCB699364D9
:1096A0000343D36418BFD064054B4A685A672A6BDA
:1096B00042F002022A639A6942F40852B8E700BFF6
:1096C000002800400008005890F82C20012A03468A
:1096D0004FF0020012D00A4A83F82D00CA215162CD
:1096E00053215162916941F020019161FF21516242
:1096F0000020012283F82D2083F82C00704700BF42
:109700000028004090F82C20012A03464FF0020068
:1097100019D00D4A83F82D00CA215162532151629C
:1097200091690A4841F080019161D0F8801041F4BC
:109730008021C0F88010FF2151620020012283F8AF
:109740002D2083F82C0070470028004000080058A6
:10975000064B5A6D520610B5044603D54022DA6511
:10976000FAF7BEFC012384F82D3010BD002800401C
:109770007047890001F1804101F531410A6070476D
:10978000890001F1804101F531410868704700000E
:109790002DE9F3471F46894690460446FAF728FA12
:1097A0000A9D3D442D1AFAF723FA264B1E68C6F38C
:1097B000CB366E43824601962268936839EA0303EA
:1097C0000CBF01230023434501D100202EE07B1C68
:1097D000F3D0FAF70DFAA0EB0A00A84229D32368C8
:1097E0005A6822F0E0025A606268B2F5827F0AD1BC
:1097F000A268B2F5004F02D0B2F5806F03D11A68AB
:1098000022F040021A60A26AB2F5005F07D11A681E
:1098100022F400521A601A6842F400521A600123BE
:1098200084F85D30002384F85C30032002B0BDE88A
:10983000F087019A019B002A03F1FF33019308BFCF
:109840001546B9E78C0300202DE9F74F9946002310
:109850008DF80330044688461746FAF7C9F90C9D7F
:109860004D442D1AFAF7C4F92C4BD4F800B01E68F9
:1098700023235E43360D6E43824601962268936829
:1098800003EA0803BB4201D100203AE0B8F5C06FFB
:1098900007D137B99BF80C30DBB28DF803309DF857
:1098A0000330B9F1FF3FEAD0FAF7A2F9A0EB0A00C2
:1098B000A84229D323685A6822F0E0025A606268FD
:1098C000B2F5827F0AD1A268B2F5004F02D0B2F59C
:1098D000806F03D11A6822F040021A60A26AB2F5C2
:1098E000005F07D11A6822F400521A601A6842F425
:1098F00000521A60012384F85D30002384F85C3044
:10990000032003B0BDE8F08F019A019B002A03F108
:10991000FF33019308BF1546B0E700BF8C0300205A
:1099200073B50B4600920D4616464FF4C051002207
:109930000446FFF789FF024630B1236E43F020034F
:109940002366032002B070BD00962B46802120467E
:10995000FFF71EFF02460028EFD100962B464FF47A
:10996000C0612046FFF770FF0028EBD0E5E74368B1
:10997000B3F5827FF7B504460E4617460BD18368D0
:10998000B3F5004F02D0B3F5806F04D1226813689D
:1099900023F04003136000973346002280212046C5
:1099A000FFF7F6FE054628B1236E43F02003236639
:1099B000032514E06368B3F5827F10D1A368B3F583
:1099C000004F02D0B3F5806F09D1009733460022D3
:1099D0004FF4C0612046FFF737FF0028E4D1284646
:1099E00003B0F0BDF8B5044600287ED0436A002BD2
:1099F00050D14268B2F5827F00D0C36194F85D30E7
:109A000003F0FF0223B984F85C202046F9F736FC06
:109A10002268E068022384F85D301368B0F5E06FD7
:109A200023F0400313604FF0000337D91D46B0F513
:109A3000706F18BFA362A7686368A169A66A07F47C
:109A4000044703F482733B43276907F002073B4353
:109A5000676907F001073B4301F400773B43E7697F
:109A600007F038073B43276A07F080073B4306F4BB
:109A700000573B43B6F5005F136014D1236B8BBBDB
:109A8000B0F5E06F0DD902232363136843F400633C
:109A9000136008E00023C0E90433AFE74FF48055BA
:109AA000C7E701232363636A676B03F0100307F0C2
:109AB000080700F470603B43090C034301F0040104
:109AC0000B432B43B6F5005F536004BFA38D1361B6
:109AD000D36923F40063D36100200123206684F856
:109AE0005D30F8BD022BDED1CFE70120F9E70000A1
:109AF00070B5044690F85C00012800F0CF8001208A
:109B000084F85C0094F85D0066680128C5B20AD04C
:109B1000B6F5827F40F0C080A068002840F0BC808D
:109B2000042D40F0B980002951D0002A4FD0002BDD
:109B30004DD094F85D00A16304281CBF052084F873
:109B40005D0000202066C4E91300A06AE387B0F539
:109B5000005F2168A3872264A4F84430A4F846304B
:109B600007D1086820F400500860086840F40050ED
:109B70000860486820F4C0404860E068B0F5E06FD5
:109B8000A06D29D94B6823F480534B6094F85D3065
:109B9000434E444D042B444B18BF1D46434B18BF46
:109BA0003346C0E90B35424B436300238363B4F86B
:109BB00046300C319BB2FEF785FA0346002848D0A8
:109BC000236E43F010032366012384F85D300120E7
:109BD000002384F85C3070BD4D6845F480554D60BD
:109BE000656DAD69B5F5806F0AD113F0010F4B6853
:109BF0001ED123F480434B60E38FC3F34E03E3870E
:109C00008369B3F5806FC1D14B6823F480534B60F7
:109C1000B4F8463013F0010F4B6811D123F4005310
:109C20004B60B4F84630C3F34E03A4F84630ADE7BA
:109C300043F480434B60E38FC3F34E030133DEE70D
:109C400043F400534B60B4F84630C3F34E03013382
:109C5000EBE72268606D516841F001015160C0E995
:109C60000B33C0E90D33E38FA16B9BB20C32FEF7CF
:109C700029FA0028A4D123681A6852065EBF1A6820
:109C800042F040021A605A6842F020025A605A6854
:109C900042F002025A609BE7022099E702209AE70D
:109CA000E99D0008B99C0008C59C0008F39C0008C9
:109CB000D19C00087047704708B5806AFFF7FBFF2A
:109CC00008BD704708B5806AFFF7FBFF08BD704705
:109CD000806A026808B5536823F003035360036E7B
:109CE00043F010030366012380F85D30FFF7EFFFB8
:109CF00008BD7FB5064600230393846A8DF80B30B8
:109D0000F9F776FF33681B689A06054668D422681F
:109D1000536823F020035360A36AB3F5005F13D1A7
:109D200001220090642311462046FFF731FD18B14F
:109D3000236E43F002032366E3682668B3F5E06F01
:109D40002ED9F3680393039BA2682368002A43D1AA
:109D50006268B2F5827F3FD15A6822F003025A60EE
:109D600064212A462046FFF702FE08B1202323661D
:109D70000023A4F846302268012384F85D309368FC
:109D8000DB0606D5236E43F0020323664FF6EF731E
:109D90009360236E23B32046FFF799FF04B070BD94
:109DA000337BDBB28DF80B309DF80B30236B022B2D
:109DB000CAD101220095642311462046FFF7E8FC32
:109DC00018B1236E43F002032366337BDBB28DF8B8
:109DD0000B309DF80B30B7E75A6822F00102BEE75E
:109DE0002046FFF767FFD9E77FB5064600230393B8
:109DF000846A8DF80B30F9F7FBFE33681B6899060F
:109E000005465ED42268536823F020035360A36A9A
:109E1000B3F5005F1BD1E368B3F5E06F3ED1236B70
:109E2000012B3BD1009064234FF400724FF4C061CA
:109E30002046FFF709FD18B1236E43F002032366A5
:109E400023681B7BDBB28DF80B309DF80B302A4664
:109E500064212046FFF764FD18B1236E43F0200310
:109E6000236623685A6822F003025A600022E287C0
:109E7000A4F84620012284F85D209A68D20606D50F
:109E8000226E42F0020222664FF6EF729A60236E53
:109E9000BBB12046FFF71BFF04B070BD00956423E3
:109EA0004FF480624FF4C0612046FFF7CDFC18B13B
:109EB000236E43F0020323662368DB680393039B4E
:109EC000C5E72046F8F7F8FCE6E70000036830B580
:109ED00059689A6802F04105012D85B0044606D103
:109EE0004D0604D5C36C05B0BDE830401847950752
:109EF00004D5080602D5236D2046F4E712F4B07F9E
:109F000059D08D0657D550060FD594F85D0003281B
:109F10004FF0000549D0206E40F004002066009507
:109F2000D868009098680090009895060CD5206E2F
:109F300040F00100206600200290986802901868A6
:109F400020F0400018600298D00508D5226E42F03B
:109F500008022266002203929A680392039A226EF4
:109F60004AB35A6822F0E0025A60012284F85D2068
:109F70008A0722D05A68A06D22F003025A6040B1CD
:109F8000104B8363FEF717F918B1236E43F04003BB
:109F90002366606D78B10B4B8363FEF70CF950B10B
:109FA000236E43F04003236605E00195DA680192D1
:109FB0009B680193019B05B030BD2046FFF787FEEB
:109FC000F9E700BFC99F000808B5806A0023A0F820
:109FD0004630C387FFF77BFE08BD0000034AD2F876
:109FE000903043F40043C2F89030704700040058AA
:109FF000034AD2F8903023F40043C2F890307047FF
:10A0000000040058074B1A6822F040021A6040F41E
:10A0100041704FF4B85218605A601A6842F040021A
:10A020001A6070470000015837B5054600284ED029
:10A03000837903F0FF046BB1032C0BD0254B4FF455
:10A0400000629A612868FFF7DDFF002401232B716D
:10A05000AC602FE000236B712846F9F7DDFC1E4A47
:10A06000D2F8903043F48053C2F89030002CE5D100
:10A0700002234FF0B042AB71D2F8943023F4004386
:10A08000C2F89430154B1B681C214B43DB0C642138
:10A090004B430193019B93B90124AC60FFF79EFFF2
:10A0A0000C4B9A6842F400629A604FF400629A6125
:10A0B000002CC7D00123AB71204603B030BD019BFB
:10A0C000013B0193D2F894305B04E3D4E6E701242A
:10A0D000F2E700BF00040058000800588C0300207D
:10A0E00037B5174D2B6802461C204343DB0C642018
:10A0F000434314480193019B93B901209060114C94
:10A1000021732B681C214B43DB0C64214B430193CF
:10A11000019B6BB9012090600A4BDB6803B030BD36
:10A12000019B013B019383689C07E4D50020E6E78F
:10A13000019B013B0193A368DB07E9D5ECE700BF76
:10A140008C0300200000015837B5184D2B680246DB
:10A150001C204343DB0C6420434315480193019BBF
:10A16000A3B901209060124CFF2323732B681C2598
:10A170006B43DB0C64256B430193019B73B9012096
:10A1800090600B4BDB680B7003B030BD019B013B53
:10A19000019383689C07E2D50020E4E7019B013B23
:10A1A0000193A368DB07E8D5EBE700BF8C03002031
:10A1B000000001580E4B0F491B681822534382B010
:10A1C0001B0D6422534301934B69019AC3F380032F
:10A1D00022B902238360012002B07047019A013A3C
:10A1E00001924A69920701D5002BEDD10020F3E7D7
:10A1F0008C0300200004005807B50379012B0FD110
:10A200000A4B1B68182253431B0C0193FFF7F0FE07
:10A21000019B013B0193019B002BF9D1FFF7DEFE6F
:10A2200003B05DF804EBFFF7C5BF00BF8C0300204F
:10A23000F8B51E468379012B154604460F46DAB25F
:10A240002DD14379012B2AD0022342718371FFF76C
:10A25000D3FF0D212046FFF7CBFEFFF741FF390A60
:10A260002046FFF73DFFF9B22046FFF739FF2E44A5
:10A27000B5420ED12046FFF7B1FEFFF79BFFA06865
:10A2800001230038A3714FF0000318BF0120637150
:10A29000F8BD15F8011B2046FFF722FFE8E7022072
:10A2A000F6E7F8B51E468379012B154604460F469E
:10A2B000DAB22FD14379012B2CD04271FFF79CFFEA
:10A2C0001D212046FFF794FEFFF70AFF390A2046BA
:10A2D000FFF706FFF9B22046FFF702FF00212046F4
:10A2E000FFF7FEFE2E44B5420ED12046FFF776FE64
:10A2F000FFF760FFA06801230038A3714FF000034F
:10A3000018BF01206371F8BD29462046FFF71CFFE6
:10A310000135E8E70220F6E7F8B51F468379012BFF
:10A32000154604460E46DAB22CD14379012B29D0CA
:10A330004271FFF761FF06F0EF03A3F1840253427D
:10A340005341237131462046FFF752FEFFF7C8FE06
:10A350002F44AF4210D1FFF741FE842E02D0204699
:10A36000FFF728FFA06801230038A3714FF0000316
:10A3700018BF01206371F8BD15F8011B2046FFF7D7
:10A38000AFFEE6E70220F6E7F8B51E468379012B1B
:10A39000154604460F46DAB227D14379012B24D063
:10A3A0004271FFF729FF39462046FFF721FEFFF7EC
:10A3B00097FE00212046FFF793FE2E44B5420ED1B2
:10A3C0002046FFF70BFEFFF7F5FEA06801230038DB
:10A3D000A3714FF0000318BF01206371F8BD294637
:10A3E0002046FFF7B1FE0135E8E70220F6E737B572
:10A3F0000023ADF8043001AA022312210546FFF71D
:10A40000C3FFBDF80440022364BA01AAA4B21946EE
:10A410002846FFF781FFE20702D528460AF01EF81A
:10A42000A30702D528460AF01FF8600702D5284680
:10A430000AF044F8210702D528460AF045F8E2065A
:10A4400002D528460AF046F8A30602D528460AF0A7
:10A450002FF8600602D528460AF00CF8210606D52A
:10A4600014F4807118BF012128460AF009F8A205EA
:10A4700002D528460AF014F8630402D528460AF0EB
:10A480002FF803B030BDF8B51E468379012B154671
:10A4900004460F46DAB227D14379012B24D042710A
:10A4A000FFF7AAFE0E212046FFF7A2FDFFF718FED8
:10A4B00039462046FFF714FE2E44B5420ED1204601
:10A4C000FFF78CFDFFF776FEA06801230038A3712B
:10A4D0004FF0000318BF01206371F8BD15F8011B90
:10A4E0002046FFF7FDFDE8E70220F6E7F8B51E4637
:10A4F0008379012B154604460F46DAB22BD14379F6
:10A50000012B28D04271FFF777FE1E212046FFF76E
:10A510006FFDFFF7E5FD39462046FFF7E1FD00211D
:10A520002046FFF7DDFD2E44B5420ED12046FFF751
:10A5300055FDFFF73FFEA06801230038A3714FF0DF
:10A54000000318BF01206371F8BD29462046FFF7BC
:10A55000FBFD0135E8E70220F6E70000036A23F07F
:10A5600001030362036A70B5446882690D6822F4CE
:10A57000803222F073022A438D6823F002032B43BA
:10A58000124DA84206D0124EB04203D0A6F5806606
:10A59000B04214D1CE6823F008033343A84223F01D
:10A5A000040306D00B4DA84203D005F58065A842F0
:10A5B00005D124F44075D1E9054634432C43446069
:10A5C00082614A684263036270BD00BF002C014093
:10A5D0000048014000440140036A23F48073036291
:10A5E000036A426870B5C4690D6824F4803424F0AD
:10A5F00073042C438D6823F4007343EA05230F4D45
:10A60000A8420ED1CD6823F4006343EA052323F466
:10A610008063D1E9055622F44052354342EA0512DF
:10A6200006E0074DA842F4D005F58065A842F0D0B9
:10A6300042604A68C461C263036270BD002C01407D
:10A6400000440140036A23F480530362026A30B578
:10A650004468C3690D6823F0807323F4E64343EA3A
:10A6600005238D6822F4005242EA05320A4DA842C1
:10A6700007D005F5C055A84203D005F58065A8426E
:10A6800004D14D6924F4804444EA85144460C361D4
:10A690004B680364026230BD002C0140036A23F45E
:10A6A00080330362026A30B54468436D0D6823F459
:10A6B000803323F070032B438D6822F4003242EA8A
:10A6C00005420B4DA84207D005F5C055A84203D05E
:10A6D00005F58065A84204D14D6924F4803444EA2C
:10A6E0000524446043654B688365026230BD00BF4A
:10A6F000002C0140036A23F480130362026A30B520
:10A700004468436D0D6823F0807323F4E04343EA0B
:10A7100005238D6822F4001242EA05520A4DA84230
:10A7200007D005F5C055A84203D005F58065A842BD
:10A7300004D14D6924F4802444EA852444604365AF
:10A740004B68C365026230BD002C0140704710B5F4
:10A75000846A626A82420BD101232377D2690AB9E3
:10A7600084F83E302046F9F71DF90023237710BD09
:10A77000A36A834208D102222277DB69002BF1D140
:10A78000012384F83F30EDE7E36A834208D10422D5
:10A790002277DB69002BE5D1012384F84030E1E723
:10A7A000236B8342DED108222277DB69002BD9D1CB
:10A7B000012384F84130D5E7704710B5846A636A95
:10A7C000834207D1012323772046FFF7F5FF0023BB
:10A7D000237710BDA36A834201D10223F3E7E36A22
:10A7E000834201D10423EEE7236B8342ECD108239B
:10A7F000E9E7704710B5846A636A834209D101238F
:10A80000237784F83E302046FFF7F3FF00232377B9
:10A8100010BDA36A834205D102232377012384F864
:10A820003F30F0E7E36A83424FF0010304D1042292
:10A83000227784F84030E6E7226B824203BF082289
:10A84000227784F8413084F83D30DCE71A4A036807
:10A85000904210B502D0B0F1804F09D14C6823F07E
:10A860007003904243EA040309D0B0F1804F06D050
:10A87000124A904203D002F58062904203D1CA6826
:10A8800023F4407313434A6923F0800313430360A6
:10A890008B68C3620B688362074B984207D003F54D
:10A8A000C053984203D003F58063984201D10B69ED
:10A8B00003630123436110BD002C014000440140AB
:10A8C00010B5044650B390F83D3003F0FF021BB9B9
:10A8D00080F83C20F9F764FA0223206884F83D30C0
:10A8E000211DFFF7B3FF012384F84830002084F8CE
:10A8F0003E3084F83F3084F8403084F8413084F8AA
:10A90000423084F8433084F8443084F8453084F889
:10A91000463084F8473084F83D3010BD0120FCE714
:10A9200010B5044650B390F83D3003F0FF021BB958
:10A9300080F83C20FFF70AFF0223206884F83D30AE
:10A94000211DFFF783FF012384F84830002084F89D
:10A950003E3084F83F3084F8403084F8413084F849
:10A96000423084F8433084F8443084F8453084F829
:10A97000463084F8473084F83D3010BD0120FCE7B4
:10A98000036A23F010030362036A426870B58469A6
:10A990000D6824F0807424F4E64444EA05248D68AC
:10A9A00023F0200343EA05130F4DA8420ED1CD68D2
:10A9B00023F0800343EA051323F04003D1E9055651
:10A9C00022F44062354342EA850206E0074DA84280
:10A9D000F4D005F58065A842F0D042604A688461F1
:10A9E0008263036270BD00BF002C0140004401403F
:10A9F00038B590F83C30012B044673D001200C2A66
:10AA000084F83C004ED008D8042A2BD0082A39D02C
:10AA1000BAB1002384F83C3038BD102A52D0142A31
:10AA2000F7D12068FFF766FE436D0A6943F40063BF
:10AA30004365436D23F480634365436D43EA02231A
:10AA40004EE02068FFF78AFD83690A6943F0080336
:10AA50008361836923F00403836183691343836102
:10AA60000020D6E72068FFF78BFF83690A6943F46B
:10AA700000638361836923F480638361836943EAAC
:10AA80000223ECE72068FFF7A7FDC3690A6943F0DA
:10AA90000803C361C36923F00403C361C36913439B
:10AAA000C361DDE72068FFF7CDFDC3690A6943F4A0
:10AAB0000063C361C36923F48063C361C36943EA6C
:10AAC0000223EDE72068FFF7E9FD436D0A6943F0D3
:10AAD00008034365436D23F004034365436D13434B
:10AAE0004365BDE7022097E710B584680A4324F464
:10AAF0007F4442EA03222243826010BD38B590F8B9
:10AB00003C30012B04464FF0020000F0958084F8A1
:10AB10003D000122206884F83C208568474B2B408B
:10AB200083600B68602B54D037D8402B6BD019D87A
:10AB3000202B0DD00AD833F0100109D0012384F85E
:10AB40003D30002384F83C30104638BD302BF5D121
:10AB5000826822F4401222F070021A4342F0070287
:10AB600082602BE0502BE9D14A68CD68016A036A04
:10AB700023F001030362836921F00A0123F0F0034B
:10AB800043EA05130A4383610262836823F4401396
:10AB900023F0700343F057030FE0B3F5805F0DD04F
:10ABA000B3F5005F0CD0702BC8D1CB68D1E901217F
:10ABB000FFF79AFF836843F0770383600022BDE7C5
:10ABC000CB68D1E90121FFF78FFF836843F480430D
:10ABD000F3E7036A4D68C96823F0100303628269D2
:10ABE000036A22F4704223F0A00343EA051342EA09
:10ABF000013282610362836823F4401323F07003FF
:10AC000043F06703D9E74A68CD68016A036A23F015
:10AC100001030362836921F00A0123F0F00343EA90
:10AC200005130A4383610262836823F4401323F00F
:10AC3000700343F04703C0E7024685E78800CEFF74
:10AC4000036A01F01F0110B501248C4023EA0403BC
:10AC50000362036A8A401A43026210BD38B50D468A
:10AC6000082D044611461BD005D85DB1042D14D023
:10AC700094F8430008E00C2D15D0102DF8D190F871
:10AC8000420001E090F83E00A0F1020CDCF100006F
:10AC900040EB0C0050B1022076E090F83F00F3E763
:10ACA00090F84000F0E790F84100EDE7082D1AD049
:10ACB00007D86DB1042D13D094F84320012A19D080
:10ACC0000CE00C2D27D0102DF6D194F842000CE0AA
:10ACD00094F83E20501E424242415AB9012053E0AE
:10ACE00094F83F20F6E794F84000421E504250414D
:10ACF0000028F3D00029F1D0002BEFD0082D4FF021
:10AD0000020256D00AD885B1042D3ED0042D84F815
:10AD10004320E3D13BE094F84100E6E70C2D5CD002
:10AD2000102DF3D184F84220D8E7606A84F83E20E1
:10AD30003A4AC2623A4A02633A4A42632268343269
:10AD4000FDF7C0F90028C9D12268D36843F4007325
:10AD50002068D36029460122FFF772FF324A9042F1
:10AD600050D0324B98424DD003F58063984249D081
:10AD7000B0F1804F4DD182682D4B1340062B02D08D
:10AD8000B3F5803F45D1002038BD84F83F20A06A4C
:10AD9000224AC262224A0263224A4263226838324D
:10ADA000FDF790F9002899D12268D36843F48063B5
:10ADB000CEE7E06A84F84020184AC262184A02636B
:10ADC000184A426322683C32FDF77CF9002885D19D
:10ADD0002268D36843F40063BAE7206B84F841200B
:10ADE0000E4AC2620E4A02630E4A42632268403231
:10ADF000FDF768F900287FF471AF2268D36843F447
:10AE00008053A5E7436C904243F400434364B2D0BF
:10AE1000AEE7036843F001030360B4E74FA70008FF
:10AE2000BBA70008F5A70008002C01400044014022
:10AE300007000100FFF712BF082938B504460D4688
:10AE40004FD004D861B1042944D0012038BD0C2969
:10AE5000FBD10268006BD36823F48053D36005E014
:10AE60000268406AD36823F40073D360FDF7A3F946
:10AE7000206800222946FFF7E3FE2A4B984207D0BC
:10AE800003F5C053984203D003F5806398420DD177
:10AE9000026A41F211131A4208D1026A40F2444395
:10AEA0001A4202BF436C23F400434364026A41F236
:10AEB00011131A4208D1026A40F244431A4202BFF7
:10AEC000036823F00103036001238DB984F83E3049
:10AED0000020BBE70268806AD36823F48063D360F4
:10AEE000C4E70268C06AD36823F40063D360BDE797
:10AEF0000C2D13D007D8042D0AD0082D0BD0012318
:10AF000084F84330E4E7102DF9D184F84230DFE7CC
:10AF100084F83F30DCE784F84030D9E784F84130EA
:10AF2000D6E700BF002C0140FFF786BF70B590F850
:10AF30003C30012B02464FF0020020D082F83D0049
:10AF40000F4D106843688468A84202BF4E6823F41E
:10AF5000700333430E6823F070033343A842436009
:10AF600002D0B0F1804F04D1896824F080030B43F4
:10AF700083600123002082F83D3082F83C0070BDE0
:10AF8000002C0140026852E8003F23F0C00342E871
:10AF9000003102680029F5D102F1080353E8003FAF
:10AFA00023F4000302F1080C4CE800310029F3D12E
:10AFB0002023C0F88830704710B5026852E8003F7F
:10AFC00023F4907342E8003102680029F5D10F4C58
:10AFD00002F1080353E8003F234002F1080C4CE85B
:10AFE00000310029F4D1C36E012B07D152E8003F94
:10AFF00023F0100342E800310029F7D12023C0F8E4
:10B000008C300023C366436710BD00BFFEFFFFEF17
:10B01000F8B504461346D4F88850202D32D1F1B14A
:10B02000EAB1E06FA4F85620A4F8542000262122AB
:10B03000C4F890602165C4F88820226888B1124F56
:10B04000C762124F0763124F2832C0E90D76FDF731
:10B0500039F830B11023C4F89030C4F8885001207A
:10B06000F8BD236840221A62226802F1080353E8FF
:10B07000003F43F0800302F1080141E8003000285E
:10B08000F3D1EDE70220EBE795B00008DDB0000852
:10B09000E9B0000808B50346806A1B681B6813F016
:10B0A000200317D1A0F85630026802F1080353E8D4
:10B0B000003F23F08003083242E800310268002993
:10B0C000F2D152E8003F43F0400342E8003100294A
:10B0D000F7D108BDF9F738F9FBE7704708B5806A82
:10B0E000FFF7FBFF08BD7047806A38B50468D0F8E9
:10B0F0008830D0F88C50A268120606D5212B04D1D6
:10B100000023A0F85630FFF73DFFA3685B0606D585
:10B11000222D04D10023A0F85E30FFF74DFFD0F8B8
:10B12000903043F01003C0F89030FFF7DCFF38BDDB
:10B1300008B5806A0023A0F85E30A0F85630FFF70B
:10B14000D2FF08BD704700000368D9691A682DE96D
:10B15000F04140F60F0631429D68044610D18E063C
:10B1600040F1978002F0200605F080573E4300F042
:10B170009080436F002B00F08580BDE8F0411847B8
:10B18000AB4EAC482E401040304300F08280CF07D9
:10B1900009D5D00507D501201862D4F8900040F0F9
:10B1A0000100C4F890008F0709D5E80707D50220F1
:10B1B0001862D4F8900040F00400C4F890004F07E3
:10B1C00009D5E80707D504201862D4F8900040F0AC
:10B1D0000200C4F890000F070BD502F020003043A6
:10B1E00007D008201862D4F8900040F00800C4F896
:10B1F00090000E050AD5500108D54FF40060186282
:10B20000D4F8903043F02003C4F89030D4F8903054
:10B21000002B37D08B0609D502F0200205F08055AF
:10B220002A4303D0636F0BB1204698472668D4F8B1
:10B230009020B36802F0280203F0400353EA0205AD
:10B24000204621D0FFF7B8FEB3685F0617D5226805
:10B2500002F1080353E8003F23F04003083242E8BC
:10B2600000310029F3D1D4F8800040B1724B8363E0
:10B27000FCF7A1FF30B1D4F88000836B7DE7204656
:10B28000FFF731FFBDE8F081FFF72DFFC4F89050C4
:10B29000F8E7E06E012840F08980CE0640F1868014
:10B2A000D00640F1838010221A629A6851064BD56D
:10B2B000D4F8802011684A6892B2002AE2D0B4F82B
:10B2C0005C009042DED9A4F85E200A6892062FD472
:10B2D00053E8002F22F4807243E800210029F7D1BF
:10B2E00003F1080252E8002F22F0010203F10800E6
:10B2F00040E800210029F3D103F1080252E8002FB1
:10B3000022F0400203F1080040E800210029F3D1B7
:10B310002022C4F88C20E16653E8002F22F01002AE
:10B3200043E800210029F7D1D4F88000FCF70EFF94
:10B3300002232367B4F85E30B4F85C10C91A89B2EE
:10B340002046FFF7FFFE9DE7B4F85E20B4F85E00EC
:10B35000B4F85C1080B292B2002893D0891A89B2F6
:10B3600000298FD053E8002F22F4907243E8002088
:10B370000028F7D1314D03F1080252E8002F2A408E
:10B3800003F1080646E800200028F4D12022C4F882
:10B390008C206067E06653E8002F22F0100243E83B
:10B3A00000200028F7D102232367C9E7CF0209D57F
:10B3B0006E0207D54FF4801220461A62BDE8F041B4
:10B3C00000F0A0BD08060BD502F0800005F40005D2
:10B3D000284305D0A36F002B3FF454AF2046CCE6A2
:10B3E0004F0611D556060FD553E8002F22F0400224
:10B3F00043E800210029F7D12023C4F88830A16751
:10B400002046F8F7A1FF3DE70D0206D5500004D510
:10B410002046BDE8F04100F077BDCB017FF532AFAB
:10B42000002ABFF62FAF2046BDE8F04100F06BBD0B
:10B43000010000102001000431B10008FEFFFFEF01
:10B44000D0F88C20B0F86010222A08B5036855D1D6
:10B450005B6A826D0B401370836D01338365B0F8B6
:10B460005E30013B9BB2A0F85E30B0F85E309BB21C
:10B47000002B42D1026852E8003F23F4907342E867
:10B48000003103680029F5D103F1080252E8002FCA
:10B4900022F0010203F1080C4CE800210029F3D14D
:10B4A0002022C0F88C20184A41679342016705D1D9
:10B4B000C26E012A0ED0F8F755FF1EE05A6811023D
:10B4C000F6D553E8002F22F0806243E800210029DE
:10B4D000F7D1EDE70022C26653E8002F22F01002F8
:10B4E00043E800210029F7D1DA69B0F85C10D206F0
:10B4F00044BF10221A62FFF725FE08BD9A6942F088
:10B5000008029A61F9E700BF00800040D0F88C2063
:10B51000B0F86010222A08B5036852D15A6A114067
:10B52000826D22F8021B8265B0F85E20013A92B269
:10B53000A0F85E20B0F85E2092B2002A40D153E815
:10B54000002F22F4907243E800210029F7D103F183
:10B55000080252E8002F22F0010203F1080C4CE827
:10B5600000210029F3D12022C0F88C20174A41671E
:10B570009342016705D1C26E012A0ED0F8F7F2FEA0
:10B580001EE05A681102F6D553E8002F22F08062BF
:10B5900043E800210029F7D1EDE70022C26653E815
:10B5A000002F22F0100243E800210029F7D1DA69C8
:10B5B000B0F85C10D20644BF10221A62FFF7C2FD39
:10B5C00008BD9A6942F008029A61F9E700800040DC
:10B5D0002DE9F84F0368B0F86060D3F81CB01F681D
:10B5E0009D68D0F88C20222A044640F0B980B0F83B
:10B5F000683043B1DFF87491DFF874A14FF00008B0
:10B600001BF0200F20D1B4F85E309BB2D3B1B4F858
:10B6100068209A4216D9226802F1080353E8003FD5
:10B6200023F08053083242E8003122680029F2D129
:10B63000504B636752E8003F43F0200342E800317B
:10B640000029F7D1BDE8F88F2368A26D5B6A33400B
:10B650001370A36D0133A365B4F85E30013B9BB258
:10B66000A4F85E302368D3F81CB01BF0070F2ED06F
:10B670001BF0010F09D0F90507D501221A62D4F891
:10B68000902042F00102C4F890201BF0020F09D074
:10B69000EA0707D502221A62D4F8902042F0040289
:10B6A000C4F890201BF0040F09D0E80707D5042246
:10B6B0001A62D4F8903043F00203C4F89030D4F802
:10B6C000903023B12046FFF70EFDC4F89080B4F807
:10B6D0005E309BB2002B93D1226852E8003F23F4E6
:10B6E000807342E8003123680029F5D103F1080294
:10B6F00052E8002F02EA090203F1080040E80021A5
:10B700000029F3D120225345C4F88C2061672167BA
:10B710000AD05A68110207D553E8002F22F0806240
:10B7200043E800210029F7D1E26E012A14D100225A
:10B73000E26653E8002F22F0100243E800210029BE
:10B74000F7D1DA69B4F85C10D20644BF10221A624D
:10B750002046FFF7F7FC53E72046F8F703FE4FE7D4
:10B760009A6942F008029A616CE700BFFEFFFFEFA2
:10B770000080004041B400082DE9F84F0368B0F89C
:10B780006060D3F81CB01F689D68D0F88C20222A16
:10B79000044640F0B780B0F8683043B1DFF87091EC
:10B7A000DFF870A14FF000081BF0200F20D1B4F893
:10B7B0005E309BB2D3B1B4F868209A4216D92268A1
:10B7C00002F1080353E8003F23F08053083242E8B7
:10B7D000003122680029F2D14F4B636752E8003FE5
:10B7E00043F0200342E800310029F7D1BDE8F88F8B
:10B7F0002368A26D596A314022F8021BA265B4F891
:10B800005E20013A92B2A4F85E20D3F81CB01BF07F
:10B81000070F2ED01BF0010F09D0F90507D5012223
:10B820001A62D4F8902042F00102C4F890201BF074
:10B83000020F09D0EA0707D502221A62D4F8902035
:10B8400042F00402C4F890201BF0040F09D0E8076E
:10B8500007D504221A62D4F8903043F00203C4F8EA
:10B860009030D4F8903023B12046FFF73CFCC4F868
:10B870009080B4F85E309BB2002B95D1226852E8DC
:10B88000003F23F4807342E8003123680029F5D19A
:10B8900003F1080252E8002F02EA090203F108004E
:10B8A00040E800210029F3D120225345C4F88C2020
:10B8B000616721670AD05A68110207D553E8002F43
:10B8C00022F0806243E800210029F7D1E26E012ACC
:10B8D00014D10022E26653E8002F22F0100243E860
:10B8E00000210029F7D1DA69B4F85C10D20644BF10
:10B8F00010221A622046FFF725FC55E72046F8F78C
:10B9000031FD51E79A6942F008029A616EE700BF83
:10B91000FEFFFFEF008000400DB5000838B504467B
:10B9200003682169A2681D68C0690A4361690A4306
:10B930007749024329400A431A605A68E16822F4B1
:10B9400040520A435A60734AA16993421CBF226A5B
:10B9500011439A6822F06E4222F430620A439A60E0
:10B96000DA6A616A22F00F020A43DA626A4A934293
:10B9700019D14FF0B043694AD3F8883003F003037C
:10B9800043F44033934200F0B480B3F1031F24D05A
:10B99000013A934240F0B580B0F5004F40F08F80FF
:10B9A000FCF7C6FF6EE05E4A93421CD14FF0B043F5
:10B9B0005C49D3F8883003F00C0343F440228A42F8
:10B9C00000F0978006D8002B7CD0574B9A42E3D0EA
:10B9D000012026E0B2F10C1FFAD1B0F5004F53D090
:10B9E0004FF4004075E04B4A9342F1D14FF0B04321
:10B9F000D3F8883003F44063B3F5006F18D006D84D
:10BA00005BB1B3F5806FE3D1FCF792FF07E0B3F5CC
:10BA1000406FDDD14FF400400BE0FDF781FB40B9F2
:10BA200000204FF00113A3660023C4E91D3338BD85
:10BA30003E4865683E4B626A05EB450133F81220CB
:10BA4000B0FBF2F39942C3D8B3EB053FC0D8002353
:10BA50001946F6F729FD090241EA10616B08000258
:10BA6000C0182A464FF0000341F10001F6F71CFD13
:10BA7000304BA0F540729A42AAD82368D860CFE72D
:10BA8000FDF74EFB0028CBD06168294B626A33F882
:10BA90001220B0FBF2F24B0803EB42034FF6EF72B9
:10BAA000B3FBF1F3A3F11001914291D823F00F02FF
:10BAB000216892B2C3F342031343CB60B0E7FCF7B3
:10BAC00037FF04E0B0F5004FDAD0FDF729FB00287E
:10BAD000A6D06368616A164A32F81120B0FBF2F012
:10BAE00000EB5300B0FBF3F04FF6EF73A0F1100240
:10BAF000C1E7B0F5004F0D48EBD1C5E7FDF720FBDE
:10BB0000C0E7B0F5004FF9D0FDF71AFBDFE700BF43
:10BB1000F369FFCF008000400038014002000300BD
:10BB20000044004008000C0004000C000024F40055
:10BB3000C0700308FFFC0F00836ADA0710B506D552
:10BB40000168C46A4A6822F4003222434A609C07B2
:10BB500006D50168046B4A6822F4803222434A60A9
:10BB6000590706D50168446B4A6822F480222243B3
:10BB70004A601A0706D50168846B4A6822F40042BD
:10BB800022434A60DC0606D50168C46B8A6822F449
:10BB9000805222438A60990606D50168046C8A683F
:10BBA00022F4005222438A605A060FD50168446C81
:10BBB0004A6822F480122243B4F5801F4A6005D1FE
:10BBC0004A68846C22F4C00222434A601B0606D5F0
:10BBD0000268C16C536823F400230B43536010BD0B
:10BBE0002DE9F843DDF8209005460F4616469846A5
:10BBF0002A68D36937EA03030CBF01230023B34249
:10BC000001D0002029E0B9F1FF3FF2D0F7F7F0FFB3
:10BC1000A0EB080048452C6802D8B9F1000F1ED1EE
:10BC200054E8003F23F4D07344E80032002AF7D1EF
:10BC300004F1080353E8003F23F0010304F1080175
:10BC400041E80032002AF3D12023C5F88830C5F836
:10BC50008C30002385F884300320BDE8F883236806
:10BC60005A07C5D5E3691B05C2D54FF400632362AB
:10BC700054E8003F23F4D07344E80032002AF7D19F
:10BC800004F1080353E8003F23F0010304F1080125
:10BC900041E80032002AF3D12023C5F88830C5F8E6
:10BCA0008C30C5F89030D4E773B504460026C0F850
:10BCB0009060F7F79DFF23681B681A07054619D4A3
:10BCC00023681B685B070AD56FF07E430093002250
:10BCD0002B464FF480012046FFF782FFB0B90020C9
:10BCE0002023C4F8883084F88400C4F88C30E066DF
:10BCF00020670CE06FF07E430093324603464FF41A
:10BD000000112046FFF76CFF0028D9D0032002B0B5
:10BD100070BD10B5044650B3D0F888301BB980F818
:10BD20008430F8F71FFA22682423C4F88830136897
:10BD300023F0010313602046FFF7F0FD012816D021
:10BD4000A36A13B12046FFF7F7FE23685A6822F46E
:10BD500090425A609A6822F02A029A601A6842F069
:10BD6000010220461A60BDE81040FFF79DBF012088
:10BD700010BD000030B581658168A0F85C2000230B
:10BD8000B1F5805FA0F85E20436735D10369002BD1
:10BD900040F2FF1318BFFF23A0F860300023C0F863
:10BDA00090302223C0F88C30016801F1080353E879
:10BDB000003F43F00103083141E800340368002CE0
:10BDC000F2D1456E84680169B5F1005F32D1B0F8F7
:10BDD000685095422ED8B4F5805F244A03D1244C94
:10BDE000002908BF22464267B1B153E8002F42F450
:10BDF000807243E80021F7E729B90369002B14BFDB
:10BE00007F23FF23C8E7B1F1805FC5D10369002B11
:10BE100014BF3F237F23BFE703F1080252E8002F3E
:10BE200042F0805203F1080040E800210029F3D1DC
:10BE3000002030BDB4F5805F0E4A03D10E4C0029BE
:10BE400008BF2246426741B153E8002F42F4907286
:10BE500043E800210029F7D1EAE753E8002F42F038
:10BE6000200243E800210029F7D1E1E7D1B500081D
:10BE700079B7000841B400080DB50008D0F88C303F
:10BE8000202B30B415D1B9B1B2B100230468C36618
:10BE90000A4B9C420AD063681B0207D554E8003F56
:10BEA00043F0806344E80035002DF7D130BCFFF744
:10BEB00061BF022030BC70470120FBE700800040DA
:10BEC000436E30B52BB90123A0F86A30A0F8683072
:10BED00030BD0368094D9A689968094C490FC2F34F
:10BEE00042626B5C615CDB00B3FBF1F3A0F86A308B
:10BEF000AB5CA25CDB00B3FBF2F3E7E7E0700308A6
:10BF0000D87003087047704770471FB504AB03E94A
:10BF1000060090F88430012B04463AD0012380F8C3
:10BF200084302423C0F8883003681A6822F00102A4
:10BF30001A609A6822F440120A439A6071B95A68EA
:10BF4000BDF80C009DF80E1022F0100202435A605A
:10BF50005A6822F07F4242EA01625A601A6842F04F
:10BF600001021A60F7F744FE6FF07E42034600922A
:10BF70004FF4800100222046FFF732FE38B920231B
:10BF8000C4F88830002384F8843004B010BD032046
:10BF9000F8E70220F9E790F88430012B0FD0012355
:10BFA00080F88430016851E8002F42F0020241E835
:10BFB0000023002BF6D180F8843018467047022009
:10BFC000704710B590F88430012B044617D0242315
:10BFD000C0F8883003681A68196821F001011960F7
:10BFE00042F000524FF0005141661A60FFF768FFBF
:10BFF0002023C0F88830002084F8840010BD02207F
:10C00000FCE770B590F88430012B044617D0056822
:10C010002423C0F888302E682B6823F001032B609E
:10C02000AB6823F060431943A960FFF749FF202361
:10C030002E60C0F88830002084F8840070BD022093
:10C04000FCE770B590F88430012B044617D00568E2
:10C050002423C0F888302E682B6823F001032B605E
:10C06000AB6823F060631943A960FFF729FF202321
:10C070002E60C0F88830002084F8840070BD022053
:10C08000FCE7000038B5084D052455F8043B2BB9F2
:10C09000013C14F0FF04F8D1204638BDDB68984716
:10C0A0000028F5D0F9E700BFD81C0020034BD8705A
:10C0B000034B1B681B6C03B118477047C01C002062
:10C0C000BC1C0020034B1874034B1B685B6C03B152
:10C0D00018477047C01C0020BC1C0020F0B5314D33
:10C0E000314B95F90420314E91B00C46012795F95A
:10C0F00005108DF8047002288DF809208DF80A10BB
:10C1000010D18DF80800D8711C7202F063FD3378ED
:10C1100003B114B101A803F0C1F9254B059A1A60C7
:10C1200011B0F0BD59714FF480711A71D9801C7231
:10C1300033788DF8087053BB1F2306A88DF81C2098
:10C140008DF8183002F024FF20238DF8183006A84F
:10C150002B798DF81C3002F01BFF22238DF818304C
:10C1600006A86B798DF81C3002F012FF21238DF8A0
:10C17000183006A86B798DF81C3002F009FF2923CE
:10C180008DF8183006A80B4B079302F001FF02F060
:10C1900021FD012306A88DF818308DF81C3002F01F
:10C1A000F7FEB4E7C01C0020C40300209C1B002045
:10C1B000901C0020000400017FB5092301A88DF820
:10C1C000043003F06BF90038044B059A1A6018BF6D
:10C1D0000120404207B05DF804FB00BF901C002026
:10C1E00070B504460B46144962784A700020A27864
:10C1F0000A7208701A884A729A788A72DB780B740D
:10C200006368CB600D4B1B68DA6A2AB1237803F0B0
:10C21000FB030A2B00D09047094E002556F8043B3B
:10C220001BB15B6A0BB1204698470135EBB2052B79
:10C230006DB2F3D170BD00BF94030020BC1C002080
:10C24000D81C002070B504461148012303706378A0
:10C250004370A3788372E368C360E378037623694D
:10C260004376237943720B4B1B689B6A03B1984753
:10C27000094E002556F8043B1BB19B690BB12046C3
:10C2800098470135EBB2052B6DB2F3D170BD00BFFD
:10C29000A8030020BC1C0020D81C0020014B1868FB
:10C2A000704700BF901C002000B58BB0012368468A
:10C2B0008DF8003002F046FD38B99DF804000038D2
:10C2C00018BF01200BB05DF804FB0020FAE7000066
:10C2D00008B501F037FE40B9FFF7E6FF012806D0A8
:10C2E000054B197AD879FFF7F9FE012008BDBDE8A2
:10C2F0000840FFF7C7BE00BFC40300202DE9F0418E
:10C3000086B005460E46174601F01CFE002873D184
:10C3100001F030FE044640B9FFF7C6FF01280AD0FD
:10C320003D4B197AD879FFF7D9FE6FF00204204609
:10C3300006B0BDE8F081DFF8E48088F80860003ED0
:10C3400018BF01268DF80460354E687833798DF872
:10C350001230694602F094FC00283FD08DF804406A
:10C360000394ADF810406FF0060495E803002D4BE0
:10C3700083E80300337988F80A30394601A803F0CE
:10C3800091F9294B059A1A6011283FD801A353F857
:10C3900020F000BFFFC30008F9C300080DC4000867
:10C3A0000DC400080DC400080DC400080DC4000829
:10C3B0002BC300080DC400080DC400080DC40008FC
:10C3C000F3C300080DC400080DC40008F9C3000839
:10C3D000F9C30008F9C3000813C400082B788DF8CE
:10C3E00008306B78ADF810306B6803934FF0FF3472
:10C3F000BBE76FF005049AE76FF0010497E70B4B7A
:10C4000000221A70E31D18BF144690E74FF0FF3466
:10C410008DE76FF004048AE7C4030020A80300201E
:10C42000C01C0020B8030020901C00208F1C00209E
:10C4300037B501F0A9FD134D052455F8043B4BB168
:10C440001A693AB19B682BB1984718B155F8043C6A
:10C450001B699847013C14F0FF04EED1FFF712FE70
:10C4600068B9094D2B7853B1084BADF80040D97825
:10C47000019422466846FFF741FF00B92C7003B0D3
:10C4800030BD00BFD81C00208F1C0020C01C002025
:10C4900030B58BB0044601F055FD0546002835D176
:10C4A000FFF702FF012834D168468DF8005002F0F2
:10C4B00049FC40BB9DF80430A34204D0012C22D09B
:10C4C000022C12D014B100200BB030BD002BFAD0DA
:10C4D00068468DF8044002F05BFDA0B90E4B1B6866
:10C4E0001B6B002BEFD09847EDE763B968468DF8DA
:10C4F000044002F04DFD30B9074B1B681B6B002B4D
:10C50000E1D02046EFE74FF0FF30DDE76FF00100AC
:10C51000DAE76FF00200D7E7BC1C002010B5044634
:10C520008AB018B94FF0FF300AB010BD002368463A
:10C530008DF8003002F006FC0028F3D19DF804309D
:10C540002370F1E77FB500220B4620498DF80720C4
:10C5500001220A7042784A700446002A33D10279D7
:10C560000A721A884A729A788A72DB780B740369A5
:10C57000CB60C378164D8DF80830037B8DF80930F9
:10C58000836803932B68DB6A0BB102A898472B687A
:10C590009B6B13B1227E02B198470E4E052556F8CB
:10C5A000043B1BB1DB690BB120469847013D15F0F8
:10C5B000FF05F4D10DF10700FFF7B0FF637913B168
:10C5C000054B01221A7004B070BD00BF9403002017
:10C5D000BC1C0020D81C00208F1C002010B5044675
:10C5E0008AB018B94FF0FF300AB010BD202368465A
:10C5F0008DF8003002F0A6FB0028F3D1024A9DF925
:10C60000043023701371EFE7C01C002000B58BB01D
:10C610002323019068468DF8003002F0B9FC003801
:10C6200018BF012040420BB05DF804FB70B5654CAB
:10C6300001468EB01822204606F08CF8624B00228C
:10C640001A70FAF7C5FE23784068012202FA03F156
:10C65000014004D15D4B084608F068F8FEE75C49EC
:10C660005C481A4602F0F8F818B14FF0FF300EB0EF
:10C6700070BD272304A88DF8103002F089FC564EB7
:10C68000564D002870D1012333702B68DB690BB144
:10C6900000209847272304A88DF8103002F052FBA1
:10C6A000059B93F84820227093F8182193F81A31CB
:10C6B0006270A370464BD3E9020105F03BFF0546CB
:10C6C0000028D2D1464E062304A88DF8103002F07F
:10C6D00039FB059B736104A802F05AFC022304A8ED
:10C6E0008DF81030059602F02DFB0836032304A8C0
:10C6F0008DF81030059602F025FB0F2605F0E0FFBF
:10C70000012304A88DF814308DF8106002F040FC6D
:10C7100010230DEB03008DF810308DF8145002F04B
:10C7200037FC04238DF8103004A8A3788DF814305A
:10C7300002F02EFC3A238DF8103004A863690593AB
:10C7400002F026FC02A920788DF8086004F09CF81D
:10C75000003818BF0120E0711420FFF757FFE0797F
:10C7600003F062F9284682E728238DF810302B6801
:10C770001B6943B104A802F0E5FA2B6805981B6910
:10C7800040F2C4519847272304A88DF8103002F0D6
:10C79000FFFB50B9012304A88DF8103002F0D2FA43
:10C7A0009DF81430002B7FF46EAF3378002B7FF4AC
:10C7B0006CAF052204A88DF81020059302F0E8FB69
:10C7C00078E700BFC01C00208F1C0020E870030821
:10C7D000941C0020AC1C00209C1B0020BC1C0020D2
:10C7E000FC1C002037B500230D4601930446D0B948
:10C7F00000F0A8FB0190019BD3B10F4A42F824300E
:10C800000E4A9A620E4A1268916B1963916C5963D1
:10C8100092690C49D9625A6128465B680A49F2223A
:10C820009847002006E001A900F092FB0028E2D022
:10C830004FF0FF3003B030BDD81C0020DDC0000831
:10C84000BC1C0020B9C100089D1B0020194B07B576
:10C850001860194B194A1A60194A5A60194A9A60A5
:10C86000194ADA60194B02681A6042685A60826895
:10C870009A60C268DA60164A1A6182695A61154B79
:10C88000C26B5A60144A019119609A601946134AA2
:10C89000DA600020FFF7A6FF48B901A800F056FBB8
:10C8A000003818BF0120404203B05DF804FB4FF090
:10C8B000FF30F9E7BC1C0020AC1C002045C200087A
:10C8C00045C5000859C90008E1C10008941C0020B2
:10C8D00039080108EC1C0020ADC00008C5C00008E4
:10C8E00049B118B1012804D000207047034B0B60F8
:10C8F000FAE7034BFBE74FF0FF30704700040001FD
:10C900000100010208B503F0ABF8002814BF6FF076
:10C910000100002008BD08B502F084F9002814BF0A
:10C920006FF00100002008BD10B504468AB018B9A8
:10C930004FF0FF300AB010BD212368468DF800305B
:10C9400002F000FA0028F3D1024A9DF90430237066
:10C950005371EFE7C01C00202DE9F0412F4D304FFF
:10C9600000232B7043786B703B689B6A8AB0044647
:10C970000BB128469847DFF8AC80002658F8043BF6
:10C980001BB11B6A0BB1204698470136F3B2052B49
:10C9900076B2F3D12378052B2FD00B2B35D0012B7A
:10C9A00025D1214C062368468DF8003002F0CAF9E3
:10C9B0000199E07905F004FE10B91C4B019A5A6107
:10C9C0001B48FFF70BFE1B48FFF7AEFF6B788BB9D8
:10C9D000A371194B5878FFF75BFD3B685B6A0BB19D
:10C9E000114898476B7813B9E07905F07BFE0AB0DF
:10C9F000BDE8F081FF23A371EFE7104B01225A74C9
:10CA0000227A9A74627ADA74F1E76378002BEED0B6
:10CA10000AB0BDE8F041FFF7CFBB00BFA80300207C
:10CA2000BC1C0020D81C0020C4030020FC1C0020DB
:10CA3000C8030020C9030020C01C0020940300206C
:10CA400030B58BB0FFF767FF0446F0B903F0FCFE8A
:10CA5000831C1DD0F8B9134D2B685B69DBB127230C
:10CA600068468DF8003002F06DF92B6801985B691B
:10CA70004FF4B961984703F0F9FE78B92CB9094B26
:10CA80001B68DB690BB10120984720460BB030BD15
:10CA90006FF00704EFE74FF0FF34ECE74FF0FF349F
:10CAA000F3E700BFBC1C0020014B1878704700BFA3
:10CAB000301D0020014B5878704700BF301D00200A
:10CAC00070470000044B9A7A0AB101225A70034B56
:10CAD0005B6903B118477047301D0020D003002068
:10CAE00073B5224C6378002B33D008F007F96668E1
:10CAF0000546FFF7D3FB0644AE4214D2A37A93B1A6
:10CB0000E0228DF800208DF80130217AE36801934E
:10CB100001226846FFF7F2FB08B1073010D100236D
:10CB20006370A372656094F83430EBB1002384F82D
:10CB300034300F4B5B6BBBB102B0BDE8704018479F
:10CB400040F2DC510B4808F0A5F90A4808F068F9F2
:10CB5000E8E794F83520002AE5D094F8360084F808
:10CB60003530FFF795FCDEE702B070BD301D0020C8
:10CB7000D0030020141D002037B5104D104CC8B153
:10CB8000C1B16272012300222860E16023700D4868
:10CB90000D4B00924FF0FF3108F096F800250B483E
:10CBA00025822022294605F0E9FD6570A574A58639
:10CBB00003B030BD00232B602370EFE72C1D002055
:10CBC000301D0020141D0020C5CA0008441D00208F
:10CBD0002DE9F0478E4C23788CB0002B56D0C278CC
:10CBE0000AB9837B13B1238A01332382437B002B51
:10CBF0004CD0E02A4AD10023A372876897F80080BE
:10CC0000B8F1220F27D8B8F1220F30D8DFE818F09A
:10CC10004100FB0052005A0061006E0075008E005A
:10CC20009D00B400C7002F002F002F002F002F0001
:10CC30002F002F002F002F002F002F002F002F007C
:10CC40002F002F002F002F002F002F002F002F006C
:10CC5000C900D000D400B8F17E0F00F0CC80B8F14C
:10CC60007F0F00F0DF80B8F17D0F00F0AB80A57A78
:10CC7000002D00F05B81674C637A3BB94FF47A7109
:10CC8000204608F007F9204608F0CAF80CB0BDE8C5
:10CC9000F087E36801220021A2721970A37AE1688B
:10CCA0009818A0720620C854A37AE1689818A07258
:10CCB000CA54DCE7584B9B6A002BD8D001210220D4
:10CCC0009847D4E77B7884F83630012384F83530F0
:10CCD000CDE704238DF804307B78003B18BF012397
:10CCE00001A88DF8083002F053F9C0E778780038D1
:10CCF00018BF012002F098FEB9E7484E0FCE01ADF3
:10CD00000FC50FCE0FC596E8070085E807007B78B2
:10CD10000A2BACD8424A12685268002AA7D00CA944
:10CD200001EB830353F82C0C9047A0E77878431E5F
:10CD3000012B9CD83A4B01381B6818BF0120207288
:10CD40009B68002B93D0984791E7E2680123082164
:10CD5000A3721170627A057BA17AAA4228BF2A4683
:10CD6000934284D285685A1CEB5CE56801334E1C03
:10CD7000A6726B54D3B2EDE7E3680122A2720922D6
:10CD80001A70A37AE268218A581CA072D154A27A40
:10CD9000238AE1681B0A501CA0728B5467E7238228
:10CDA00065E705238DF8043001A802F077FB5EE704
:10CDB000194BDB6A98475AE7194B78781B686075FE
:10CDC000DB68BEE7037B072B7FF451AF06238DF8AA
:10CDD0000430B7F80130ADF808307B793A791B049C
:10CDE00043EA0223FA781343642253430393BB7943
:10CDF0008DF81030D8E73B2201A88DF804208DF87B
:10CE0000083002F0C5F8012384F834302FE700BF62
:10CE1000301D0020141D0020D0030020E419030859
:10CE20002C1D00202A2301A88DF8043001F08AFF70
:10CE300094F80A90E6689DF808009DF809509DF85E
:10CE40000A709DF80BC09DF80D309DF80E209DF8DE
:10CE50000F109DF80CE009F1010A84F80AA006F809
:10CE60000980354E94F80A903668D4F80C8009F1A0
:10CE7000010A84F80AA096F803A008F809A094F81B
:10CE80000A90D4F80C8009F1010A84F80AA096F8F7
:10CE900002A008F809A094F80A90D4F80C8009F1CF
:10CEA000010A84F80AA096F801A008F809A094F8ED
:10CEB0000A9009F1010A84F80AA096F80080E66851
:10CEC00006F8098094F80A80E66808F1010984F8F8
:10CED0000A9006F808C094F80AC0E6680CF1010848
:10CEE00084F80A8006F80C70A77AE66807F1010C4E
:10CEF00084F80AC0F555A57AE6686F1CA7727055CC
:10CF0000A07AE568461CA6722954A17AE0684D1CF7
:10CF1000A5724254A27AE168501CA0728B54A37A85
:10CF2000E268591CA17202F803E0A0E6034807F08A
:10CF300029FF6570AAE600BF2C1D0020141D0020EB
:10CF40007047000000487047D00300200020704761
:10CF50004FF0FF3070470000044B054A93F818313A
:10CF6000022B18BF062382F890347047D423002088
:10CF700098290020034BD3F8483313B15B6903B100
:10CF80001847704798290020034A137843F0040398
:10CF90001370FFF7EFBF00BF7C1D00201FB50A4BC9
:10CFA0008DF8090093F87C208DF80A2093F88C20E6
:10CFB00093F848000D3202A98DF8082003F064FCB4
:10CFC000C0B205B05DF804FBD423002008B50748C3
:10CFD00007F0D8FE064B93F81A2412B1012283F809
:10CFE0001924BDE80840FFF7C5BF00BF982D0020F9
:10CFF0009829002010B50C4CD4F8403343F080033E
:10D00000C4F8403394F81A3413B10020FFF7DEFF60
:10D0100094F8913423F0120343F0120384F891340E
:10D02000BDE81040FFF798BF982900202DE9F04196
:10D03000DFF8AC8098F81831022B06460D4602D076
:10D04000284BDB6A984702F0A6FD044628B102206F
:10D0500002F097FD002002F099FD98F81831012B9D
:10D0600017D102F09AFD074630B1002002F08AFD88
:10D07000002002F08CFD3C4602F091FD48B10020FA
:10D0800002F081FD002002F083FDBDE8F041FFF7D2
:10D0900063BF002CF9D1144C94F8902494F81A34FE
:10D0A000BAB90BB184F84164304602F017FFD8F8E2
:10D0B0002C0007F02DFED4F8B4339842E5D30B488A
:10D0C00007F060FE94F8913443F0100384F8913433
:10D0D000DBE70BB184F84154284602F0FFFEF1E78C
:10D0E000D42300206078030898290020302D0020E8
:10D0F000074A10B5137843F002031370FFF73AFFA5
:10D10000BDE81040034B01220021022007F00EBBB6
:10D110007C1D002031710308074A10B5137843F0D5
:10D1200008031370FFF726FFBDE81040034B0122F0
:10D130000021022007F0FABA7C1D0020417103088B
:10D140002DE9F0410F4616461D46804607F0D6FDF4
:10D150000B4A0C4C1378278123F0110343F0110381
:10D16000C4E90008137066812573FFF703FFBDE86B
:10D17000F041054B01220021022007F0D7BA00BF81
:10D180007C1D0020681D00205171030813B507F0B5
:10D19000B5FD0D4B6C461860204607F003FD94E882
:10D1A00003000A4A0A4B83E80300137843F0200384
:10D1B0001370FFF7DFFE074B01220021022002B0AF
:10D1C000BDE8104007F0B2BA781D00207C1D002099
:10D1D000D02C00205E7103082DE9F04192B0064684
:10D1E00002F0D9FC002840F05881AD4D95F8183177
:10D1F000012B09D02B6BAB4C93B194F80431BBB12C
:10D20000042B6FD0032003E002F0C7FC18B10F20FD
:10D2100012B0BDE8F08102F0C2FC0028EAD0F6E7C7
:10D22000B5F82031D4F81C24013B53432B63E4E7C9
:10D230009D4803F060FA002840F0128194F80C3108
:10D2400023802B6B0C930DF1180895F839308DF86D
:10D250003830404695F81C318DF83A3007F0C8FC5C
:10D26000D5F82831009302AF98E80600D5F82431AC
:10D27000384607F054FC97E803000FAB83E803003F
:10D28000EB6A0D9300238DF844302388ADF84630C7
:10D2900095F8303101228DF839201BB98DF84420E2
:10D2A0008DF83930814B0093814B95F84800A3F1FC
:10D2B00079020CA903F05DFBC0B10B28A8D1D4F80A
:10D2C000941499B1002EA3D0D4F84033794843F098
:10D2D0002003C4F8403307F0DDFD764807F0A0FDD9
:10D2E000002095E7704803F03AFAA4E795F84870F3
:10D2F00095F9693095F9392095F87D106E4E3846CC
:10D3000003F044FB009641B2EB6C95F85020384690
:10D31000183603F0DFFA0096EB6C95F8502095F97B
:10D32000701095F8480003F0D5FAD4F8C413AB6D2B
:10D33000D4F8DC230B44C4F8B033EB6D1344C4F8C9
:10D34000B43394F80431042B07D02B6E0B44C4F88B
:10D35000B0336B6E1344C4F8B4330023089395F8CC
:10D360003031002B40D100238DF8133095F839303F
:10D370008DF8213095F838308DF82230D5F880308E
:10D380000993D5F884300A932388ADF82C3095F8AA
:10D39000303194F81B648DF82E3095F84800474BD7
:10D3A0008DF820600DF1130208A903F0A7FA0123FC
:10D3B00084F8413495F8393084F842349DF81330BC
:10D3C00084F84334D4F81C34C4F85064C4F84834A6
:10D3D000C4F8583402F0E5FBC8B1D4F81C0402F0DC
:10D3E000F2FBA0B1102013E708A802F0A7FC60B977
:10D3F00095F9390094F837629DF82070FFF7CEFD5B
:10D400003E44B042AFD2082002E7132000E795F86F
:10D410001831012B01D102F0D8FB02F0C5FB00232B
:10D42000059394F8043195F9395094F81B649BB135
:10D43000042B7FF4E7AE05A802F0B4FE58BB94F8C5
:10D44000183413B1059B013B0593174B05983246E1
:10D45000E9B202F00DFF02E0134802F0DDFE08B170
:10D460001120D5E6D4F8403394F80C11218043F014
:10D470000203C4F8403394F8183411480133DBB286
:10D4800084F8183484F845340E4B00259B6AC4F8A0
:10D490009854984724E71220BAE60E20B8E600BF59
:10D4A000D423002098290020A02A00200424002052
:10D4B0002C2E0020002D0020502D0020B42D002007
:10D4C0009A2900206078030873B5134D134E009617
:10D4D000EB6C95F8502095F9781095F8480003F01A
:10D4E000F9F995F83031337595F8480040F2012389
:10D4F00006F13C023146738203F0F8F950B196F818
:10D500003C3086F88230064B00205B6B9847F37CFA
:10D5100086F8A83002B070BDD4230020802D0020F2
:10D5200060780308F8B5324C94F81831012B0546A1
:10D530000ED0022B4ED0002B57D138B9D4E91B01A5
:10D5400004F1740383E803000020F8BD012806D12C
:10D5500002F02CFB0028F8D184F81851F5E70228D6
:10D5600043D1244E84F8180106F5747CBCE80F0002
:10D5700006F57A770FC79CE8030094F8E92094F841
:10D58000003187E8030086F8FB53D2B1022B18D193
:10D59000D4F804316367C6F8EC3394F87D3094F81E
:10D5A000082186F8F83394F88C3084F8782086F8CF
:10D5B000F93396F81B2486F8E82340F20133A6F8E5
:10D5C000FA33002386F81A340B4BDB6A9847FFF7CF
:10D5D0007BFFB9E748B9074B84F81801062283F8A6
:10D5E0009024054BDB6A9847AEE70320ADE700BF08
:10D5F000D42300209829002060780308F0B5504C0F
:10D60000504EB4F8DC202287D4E92D0194F8B120E3
:10D6100084F8692004F16C0282E80300D4E92F0148
:10D6200004F1740282E80300B4F8C420A4F87C205A
:10D6300091B0D4F8CC20D4F8C810C4F884200025C8
:10D64000D4F8D020C4F888200123A4F82031C4F8ED
:10D65000801084F83051A56284F81B5184F83A5048
:10D6600084F81D5184F81E51C4F83451C6F89854FA
:10D67000A6F8185486F81A54A4F838518DF81830C2
:10D6800004F50973039304F50A7394F848000493AE
:10D6900003A92D4B84F84551C4E94F55A4F84651D0
:10D6A000059303F0FFF8E36EC6F8D43394F87D30A9
:10D6B00086F8E03394F88C3086F8E1334FF48073C9
:10D6C000A6F8E23386F8D05394F8303186F8E43384
:10D6D00006F574770FCF06F57A740FC497E8030048
:10D6E00040F2012384E80300A6F8FA33D6F8483361
:10D6F00086F81B54CDE901551BB15A685B6901924C
:10D700000293124B0793A3F148020892A3F114026B
:10D7100009920F4A0B9229330A93A2F19C030C93AE
:10D72000A2F198030D93131D0E9301A902F14C036E
:10D7300007A802F599620F9302F022FA11B0F0BD2A
:10D74000D423002098290020801D0020002E0020D6
:10D75000B8240020F8B50D4F0D4E0C4607F012FB13
:10D760003B6B98470B4A96F84800214603F0BEF8F9
:10D7700050B1094D706D95F8243485F86A347B6B8F
:10D780009847E37C85F89034F8BD00BF60780308C3
:10D79000D4230020BC2D0020982900200F4890F8A9
:10D7A0001B3480F8B8330E4B93F8692080F8BB2304
:10D7B00093F87D2080F8C82393F88C2080F8C92343
:10D7C00093F8303180F8CC330022A0F8CA2300F55A
:10D7D0006E7100F56070FFF7BDBF00BF9829002093
:10D7E000D4230020114890F89034EBB190F81B340A
:10D7F00080F8D0330E4BDA6EC0F8D42393F87D2036
:10D8000080F8E02393F88C2080F8E12393F83031FE
:10D8100080F8E4334FF48072A0F8E22300F57471CD
:10D8200000F56670FFF796BF704700BF982900208B
:10D83000D423002070B5344C2421204604F0A0FFEE
:10D84000636A984218BF60624FF01C012F4814BFF2
:10D850000125002504F094FF636C984218BF6064B2
:10D860004FF480712A4818BF45F0020504F088FF84
:10D87000D4F84831984218BFC4F848014FF0D40199
:10D88000244818BF45F0040504F07AFFD4F820328C
:10D89000984218BFC4F820024FF000011E4818BF7C
:10D8A00045F0080504F06CFFD4F82432984218BF04
:10D8B000C4F824024FF46071184818BF45F01005F1
:10D8C00004F05EFFD4F8A835984218BFC4F8A80544
:10D8D0004FF01401124818BF45F0200504F050FF26
:10D8E000D4F8C03598420F4B18BFC4F8C005D3F820
:10D8F000483318BF45F040052BB11B691BB12846C2
:10D90000BDE87040184770BDD4230020FC230020E0
:10D910001C24002020250020F8250020FC250020C4
:10D9200080290020982900202DE9F04F8FB04FF07A
:10D930000009012B06460F4690468DF80D90ADF874
:10D94000109002D84C46BC4202D30FB0BDE8F08F15
:10D95000305D02F033FA2044B842F6DC335D651CDA
:10D96000023BEDB2112BF0D801A252F823F000BF18
:10D97000B9D90008E3D90008E1DA000809DB00089A
:10D9800087DB0008ADDB000813DC00083BDC000887
:10D99000C1DC00084BD900084BD9000815DD000890
:10D9A0004BD900084BD90008BDDD0008E5DD0008B3
:10D9B0001DDE000851DE0008052002F0A7FA70B154
:10D9C0000521002002F068FA725DBA4BE51C0234B2
:10D9D000E4B283F85C24325D83F85D24EDB22C461A
:10D9E000B1E700238DF80E308DF80F308DF814302C
:10D9F0008DF81830B9F1000F6DD1AF4C4FF005091B
:10DA000094F87C208DF831206B1E94F839208DF825
:10DA10003320334494F838200B938DF8342094F855
:10DA20001A3194F868208DF83520D4F82C218DF81F
:10DA300032300A9273B37B1C5B1BDBB28DF8303043
:10DA400006AB019305AB009394F848000DF10F036A
:10DA50000DF10E020AA902F05DFF8DF80D0000F035
:10DA60000700072813D194F939209DF90E3084F866
:10DA700039309A429DF80F3084F83830B8BF01220F
:10DA80009DF81430B8BF84F81D2184F868304FF039
:10DA9000000A09E00523D1E701220DF10D01032061
:10DAA00002F0A4F80AF1010A5FFA8AF29DF8183030
:10DAB000B3FBF9F19142EFD82B44DDB26B1EDBB220
:10DAC0009F420BD9F25C032A9AD0AF4288BF1D4611
:10DAD0004FF0010983E70534E5B2F9E71D46F7E7A2
:10DAE000735D754903F00F03012281F81B31023485
:10DAF00002FA03F3A1F82031E4B2002204A90420C1
:10DB000002F074F825466AE707238DF80D30735D3F
:10DB1000C3F3021203F00F038DF82830E31CDBB2CD
:10DB20008DF82920F25C231DDBB2651DF35C023405
:10DB3000E4B21B0443EA0223325D5F4C13436422C8
:10DB4000534394F848000B930AA902F0F2FE00F048
:10DB50000703072BEDB28DF80D000CD19DF828308E
:10DB600084F8703084F878300B9BE36663679DF827
:10DB7000293084F869308DF81000012204A90520AD
:10DB800002F034F82BE74B4BD3F8483363B11B68F2
:10DB900053B1984708F03F038DF810008DF811300D
:10DBA000022204A90620EBE7FF20F3E703238DF808
:10DBB0000D30735D8DF81C300AAB0693E31CDBB2AD
:10DBC000A51DF25C231DDBB206A9F35C1B0443EA2E
:10DBD0000223A21CD2B20534B25C13436422534325
:10DBE000E4B20A9300230B93335D8DF83030324B4F
:10DBF00093F8480002F0A3FEC3B20028EDB28DF8FE
:10DC00000D30FFF6ECAE8DF81030012204A907208C
:10DC1000B6E7735D03F00F03012B4FF47A7238BF40
:10DC200001235343244A0234936503F57A73D36581
:10DC3000E4B2002204A9082062E7735D1E4DC3F31D
:10DC400040128DF8152095F84800C3F3001205A97D
:10DC500003F00F038DF814208DF8163002F075FED6
:10DC600002340130E4B23FF44DAFBDF81430134A32
:10DC7000A5F87C309DF816309DF814A0D05CF4F720
:10DC800099F90223C5F880000AA995F848008DF893
:10DC900028308DF82AA002F0F7FD95F9393006906A
:10DCA00040B29842B8BF184685F83900002204A94E
:10DCB000092025E798290020D42300206B71030850
:10DCC00003238DF80D30735D8DF82830E31CDBB233
:10DCD000651DF25C231DDBB20234F35CE4B21B046D
:10DCE00043EA0223325D1343642253430B93644B94
:10DCF0000AA993F8480002F02EFEC3B20028EDB244
:10DD00008DF80D30FFF66BAE8DF81030012204A9AE
:10DD10000A2035E7092002F0F9F8DFF868B1002899
:10DD200049D00921002002F0B7F80023ADF81E30D9
:10DD3000A31CDBB2F25CE31CDBB216F803A0735D3C
:10DD40004FEA0A4A4AEA022A4AEA030A231DDBB2D8
:10DD5000A51D0534F35CE4B24AEA036A335D4FF46F
:10DD60007A7253430AAC1B122046ADF81C3006F001
:10DD700019FF454B53440693DBF83C3300930DF1F8
:10DD8000180A9AE80600DBF8383308A806F0C7FE40
:10DD9000099B009394E80600089B504606F0A4FEF9
:10DDA0009AE8030006F0D6FE01F00AFF0123EDB267
:10DDB0008BF8383413E68BF8380410E60C2002F0A8
:10DDC000A5F800283FF40BAE0C21002002F064F807
:10DDD0002C4B93F89034043B012B7FF600AE01F0FE
:10DDE000EBFEFCE5A31CDBB2725DF15CE31CDBB275
:10DDF000651DF35C0434E4B21B04305D43EA012387
:10DE000013436421594300F00F0001F0D6FEEDB238
:10DE10008DF81000012204A91120B1E60D2002F0B6
:10DE200075F800283FF4DBAD0D21002002F034F836
:10DE3000A31CDBB2154AF05C735D1268251D033428
:10DE4000E4B243EA0020315DEDB201F0B8FEC6E570
:10DE5000725DA31C251D0334DBB2E4B2F15C335DBB
:10DE60001B0443EA012313436420584301F0A9FE35
:10DE7000EDB28DF81000012204A9132080E600BF46
:10DE8000D423002098290020803DD512681D002051
:10DE90000E4B93F89124920703D593F88F24012A0F
:10DEA00008D90B4991F81A2122B18A6A501C18BF6F
:10DEB00001328A620022A3F8182483F81A24D3F8C6
:10DEC000402322F00202C3F8402370479829002023
:10DED000D423002070B5184C1848194D06F052FF95
:10DEE000D4F84033D4F89804D5F8906023F0200398
:10DEF000C4F8403338B106F00BFF864203D200234A
:10DF000085F83A3070BD0120FFF766F90028F9D096
:10DF10000B28F7D095F8393084F84234092094F86A
:10DF2000183484F8453484F8410401F0D7FFBDE883
:10DF30007040FFF7ADBF00BF98290020002D0020E2
:10DF4000D4230020094BD3F84023012A0AD00849E2
:10DF50000978C90708D43AB993F89204013818BF70
:10DF60000120704700207047012070479829002049
:10DF70007C1D0020034BD3F84003431E58425841F8
:10DF8000704700BF982900202DE9F04FA9B0EFF3AA
:10DF9000108272B6DFF8F0B20021DBF80030CBF867
:10DFA000001082F31088B94C002B00F0E180DAB247
:10DFB0009B06039264D5B64D95F81831022B02D01A
:10DFC000B44BDB6A9847EFF3108872B6B24F06F095
:10DFD00095FE3E68D4F8B013361A3144AF4806F0C7
:10DFE00059FFAE4806F01CFFD4F8B413AC483144D6
:10DFF00006F050FFAA4806F013FF88F3108894F843
:10E000001A34002B00F06B81152312A995F84800F3
:10E010008DF8483002F038FCD4F8B4130F90014466
:10E02000A04806F037FF9F4806F0FAFE3B6894F8D8
:10E030001B24EB620DAF38468DF870201D9306F05F
:10E04000D7FDD5F82831009306AE97E80600D5F83D
:10E050002431304606F063FD96E803001FAB83E8E9
:10E060000300D4F81C341E9395F8303195F848001D
:10E07000003B18BF01231CA98DF8713002F00DFC84
:10E08000039BDF0648D5824DDFF81CA2D5F8E420BB
:10E0900004929BF80020BAF90A809AF90C90A4F82F
:10E0A0008C84002363F300020A9384F84434A4F8B8
:10E0B000223484F82534C4F82834A4F82C3484F8A5
:10E0C0002E34C4F8303484F82034C4F8343484F85E
:10E0D0003834C4F83C346F4B8BF8002094F890240B
:10E0E000DB6A84F88E9484F88F24DAF80470BAF826
:10E0F0000860984794F88F3413B9694806F042FED7
:10E100003146384601F045FD8346002800F0EA809C
:10E11000A4F87E8484F88094039B19071AD55C4B7D
:10E1200093F81831022B02D05A4BDB6A9847022031
:10E13000FEF712FF84F8410401F0D0FE94F81A347F
:10E1400013B1012384F8193494F8913443F0100387
:10E1500084F89134039B5A0703D506210520FEF766
:10E1600065FF039B9B0703D504210320FEF75EFF99
:10E1700001F02DFD94F89124D7065FD5002384F893
:10E180009234D4F840331E0644BF23F08203C4F80F
:10E19000403312F0050F00F0FB820B2001F0B6FEB9
:10E1A000002800F0F58294F89134DD0700F1F08248
:10E1B000580740F10783D4F8403323F00203C4F832
:10E1C0004033D4F8402382BB94F8915415F00101F8
:10E1D0001EBF2B4662F3000384F8913494F8913407
:10E1E0005E0744BF6FF3820384F89134012384F8FF
:10E1F000923421B1D4F844332C481B6898476D07FA
:10E200000BD52B4801F08EFE01F0BCFE28B194F82E
:10E21000913443F0040384F8913401F0C6FC94F87F
:10E2200091346FF3041384F89134012384F8923409
:10E2300094F8913443F0200384F8913494F89134A5
:10E2400018070AD56FF3C3031A4984F89134D4F838
:10E250004433A1F12400DB68984794F8913499077E
:10E260000AD56FF34103134984F89134D4F8443349
:10E27000A1F16C005B68984794F89034022B1BD195
:10E28000FFF722F918E000BF7C1D0020982900202C
:10E29000D423002060780308781D0020182D00206A
:10E2A000302D0020982D0020681D0020D82D002042
:10E2B000EC2D0020242E002094F891349A0640F191
:10E2C000C4826FF3451384F89134D4F84033002BA3
:10E2D00040F0BB8229B0BDE8F04FFFF7ABBA84F83D
:10E2E0004134A3E695F81831012B0CD101F055FC0F
:10E2F000804668B1584601F045FC584601F047FC9D
:10E30000042384F88F347EB9012384F821344FE14B
:10E3100001F045FC0028F6D0404601F034FC4046B0
:10E3200001F036FC0523ECE73B7805935B09013BE4
:10E33000062B00F21782DFE813F0070015029500A4
:10E340001502920015020602102EDDD995F8303123
:10E350001297F6B28DF84C60002BD5D11CA804F0B2
:10E3600021F912AA1CA9FF2002F09EF89DF858304E
:10E37000C3F3030307468DF82C3095F8480095F851
:10E380007D308DF82D3007220BA902F090FA002F76
:10E390005DD100285BD09DF853309DF8522015992F
:10E3A000C5F8E4101B0443EA02239DF85120022023
:10E3B0001343C5F8E03004F003F99DF8583095F8A0
:10E3C000480085F82E71C3F30212C3F3030385F8E6
:10E3D000703085F878309DF8593085F86920012B28
:10E3E00038BF01234FF47A725343AB651344EB6596
:10E3F0000DF15A034FF001081093113E94F81B34AD
:10E400008DF83C300FA985F868808DF8446002F0E3
:10E4100056FA0223404685F8303101F077FD18B1F5
:10E420004146384601F038FD94F88F34012B00F254
:10E43000A78194F81A34002B40F09A8194F8913413
:10E4400043F0100384F89134FEF786FD64E6012062
:10E4500001F05CFD0028E7D001210720E2E701235D
:10E4600084F8203495F87D308DF82E3094F82434DB
:10E470008DF82D3095F88C3095F848000D330BA9A8
:10E480008DF82C3002F000FAA6F10D031BB20990B2
:10E4900023EAE37300B283423FF736AF0B2E7FF6D9
:10E4A00033AFBA4B25931CA8FF231C978DF87460DB
:10E4B0008DF8983002F0C4F8074600287FF424AFA6
:10E4C00095F81831012B13D101F067FB002872D0A9
:10E4D000384601F057FB384601F059FB04239DF8FC
:10E4E0007C101E9884F88F34C1F3001101F06EFB8C
:10E4F0009DF87C301E99C4F8341413F00F0203D039
:10E500009DF89000002862D19DF89800002861D005
:10E51000002A7FF4F9AE9DF89020002A14BF4FF036
:10E5200003084FF0020800220A92D5F8EC2095F873
:10E53000E900914251D100284FD0D5F80C1195F83F
:10E54000EAB009680A9195F81811022902D103214D
:10E5500084F88F14B8F1030F7FF4D6AE13F0600F78
:10E560007FF4D2AE0492012795F82E31BBF1000F53
:10E5700036D0BBF1010F13D1012B33D16FF0090657
:10E5800046FA08F606F00106C6F10206F6B2BDF834
:10E590007E100AAA304601F011FE38B3072823D0B6
:10E5A000012384F821340A9BC4F83034C4F86C3455
:10E5B000FEF720FDB0E501F0F2FA002898D03846C9
:10E5C00001F0E1FA384601F0E3FA052387E74FF05E
:10E5D0000008A8E74FF00108A5E74FF0010BC3E7DB
:10E5E0000426D4E70326D2E70823DAE71CAB00931E
:10E5F00004990A9B3246584601F0A2FE20B1022837
:10E6000014BF0B230A2380E60A9BC4F83034C4F8F5
:10E610006C349DF87C3084F82104C3F3401384F8F3
:10E620002E3484F8443494F88F3484F82274012B07
:10E630009EBF0122A86285F81E21012FC4F828047C
:10E6400084F82C0484F8410438D1022284F8202470
:10E6500095F83A20002A4AD19DF87C20D60646D467
:10E66000012B94F840149DF87C2005D8012901D194
:10E67000900601D501F04CFBB8F1020F94F88F34ED
:10E6800043D0B8F1030F0AD09DF87C10B8F1010F08
:10E690004A4601F00F0120A83BD0FFF745F99DF84D
:10E6A000903084F82334259BC4F828349DF89830A2
:10E6B00084F82C34012384F82D3430E0059A02F0DC
:10E6C000E002A02A1BD195F82E11012285F83A20EC
:10E6D00009B927996963012B84F8202407D9D5F853
:10E6E0009020C4F83C24DAF80020C4F8982495F867
:10E6F0001821002AB4D1012284F82524B0E7002291
:10E7000085F83A2084F82024A6E79DF898102598EB
:10E710004A46FFF709F99DF8903084F823349DF8B4
:10E720009020E02A08D195F81F312BB984F82324D2
:10E73000C4F82834A4F82C3494F8913443F002033C
:10E7400084F8913470E6114D013EB2B2791C28462E
:10E7500004F000F80323A4F82034C4F8285484F803
:10E760002C64E9E7012384F82134FEF743FC5BE6DF
:10E7700094F84434002B3FF461AE0020FEF726FCF1
:10E7800094F88F34022B3FF45FAE57E6D02B002075
:10E7900094F89134590715D5012001F0B7FB60B109
:10E7A000012001F08BFB08B984F81804D4F8403339
:10E7B00023F00203C4F8403304E0062001F0A6FB76
:10E7C0000028F3D194F89134DA077FF5FAAC94F885
:10E7D00040240AB1032A18D11D4A94F8181492F85B
:10E7E0006820914205D29B0723D594F88F34012BE2
:10E7F0001FD8184806F0C6FAD4F8403323F0200397
:10E80000C4F84033FFF744FBDBE4012A11D194F84C
:10E810001924002A3FF4D5AC0D4A94F8181492F844
:10E8200068209142E5D29F0703D594F84434002B29
:10E83000DFD194F8913400206FF3041384F89134FD
:10E8400084F81904FFF746FBBBE429B0BDE8F08F5C
:10E85000D4230020002D00202DE9F04F89468DB0F3
:10E8600090460746002800F08F81002900F08C8137
:10E870000368002B00F088814368002B00F084813E
:10E880008368002B00F08081C368002B00F07C813E
:10E89000104601F0F5FF002800F07881BD4CBE4D18
:10E8A000384601F0AFFA40F2C4520021204603F08E
:10E8B00065FF40F21C520021284603F05FFFB74B72
:10E8C000C4F82C3104F50973089304F50A73002683
:10E8D0004046099308A9B24B84F848800A9384F80B
:10E8E000186184F88C608DF82C6001F0DBFF0F2339
:10E8F00006A994F848008DF8183001F0C5FF801B78
:10E9000018BF01204FF00A0B84F81C0106A994F8E7
:10E9100048008DF818B001F0B7FF4FF0060A84F8F0
:10E92000DC0006A994F848008DF818A001F0ACFFAF
:10E93000102384F8DD0006A994F848008DF81830FB
:10E9400001F0A2FF1123C4F89C0006A994F8480026
:10E950008DF8183001F098FF1223C4F8A00006A922
:10E9600094F848008DF8183001F08EFF1323C4F896
:10E97000A40006A994F848008DF8183001F084FF2F
:10E980001423C4F8A80006A994F848008DF818309C
:10E9900001F07AFF1623C4F8AC0006A994F84800E9
:10E9A0008DF8183001F070FF172384F8B10006A924
:10E9B00094F848008DF8183001F066FF18230DEB2D
:10E9C0000301C4F8B400C4F8BC0094F848008DF802
:10E9D000183001F059FFC0B21D2384F8B80084F844
:10E9E000C00006A994F848008DF8183001F04CFFDB
:10E9F0001E2384F8C40006A994F848008DF8183046
:10EA000001F042FF1F2384F8C50006A994F84800CE
:10EA10008DF8183001F038FF2023C4F8C80006A98B
:10EA200094F848008DF8183001F02EFF0B23C4F83D
:10EA3000CC0006A994F848008DF8183001F024FFA6
:10EA40000C2306A9A4F8D00094F848008DF81830DB
:10EA500001F01AFFD4F89C306365D4F8A030A365A8
:10EA6000D4F8A430E365D4F8A83023664FF0010849
:10EA7000D4F8AC300590A4F8D200636684F8B08076
:10EA8000C4F894B084F898A0C4F84CB084F850A0AE
:10EA900084F8688084F81F81C5F84893FEF7AEFDBE
:10EAA000C5F84473C4E90B663E4B84F8198185F8B8
:10EAB0009164C5F8408332464FF0FF31009605F56A
:10EAC0005A7006F001F9384B009632464FF0FF318C
:10EAD00005F5607006F0F8F8344B009632464FF0BA
:10EAE000FF3105F5667006F0EFF802AF304B009687
:10EAF00032464FF0FF3105F5806006F0E5F8384604
:10EB000006F076F897E8030004F5927383E80300B3
:10EB1000284B294F1E60294BC5F84C33284BC5F8AC
:10EB20005433284BC5F85C33274BC5F85033274B7B
:10EB3000C5F8583305F553703B68984704F5A6703F
:10EB400003F04CFB20B1112630460DB0BDE8F08F2C
:10EB5000204601F003FB0028F5D101F039F8B8B9DF
:10EB60001B4801F04DFB06460028ECD17B69984715
:10EB700003F0CEFDBB6D94F819019847FB6A9847E6
:10EB8000012385F89234DFE70326DDE70926DBE77A
:10EB90001326D9E7D423002098290020000400017F
:10EBA000801D0020D5DE00089DD70008E5D70008AD
:10EBB000CDCF00087C1D0020607803088DD10008AF
:10EBC00041D1000889CF000819D10008F1D0000810
:10EBD000BC24002008B5034B0020C3F84003FEF717
:10EBE000BBF908BD9829002010B5FFF7ABF90A4C16
:10EBF00060B90A4B93F81831022B02D1084BDB6A3B
:10EC000098470123C4F84033002010BDD4F84003D6
:10EC1000013818BF0120F8E798290020D4230020EC
:10EC20006078030838B5124C204606F0ABF804F1C2
:10EC3000180006F0A7F804F1300006F0A3F804F17C
:10EC4000980006F09FF800F0AFFF0A4B0025DB6A42
:10EC5000984744F8285CFEF7EDFD0749074840F265
:10EC6000C45203F077FD012344F8283C284638BD00
:10EC7000002D002060780308D4230020101E0020FF
:10EC800070B52E4B8AB0054693F8DD008DF809006B
:10EC900093F8DC008DF80A0029489A6A90F8180465
:10ECA000039200268DF80B0004960C46002940D0F4
:10ECB0000692D3F8882007921A8F93F81A118DF8CC
:10ECC000151052BAADF8202093F87C2093F8483004
:10ECD0008DF8243003AB8DF822008DF823200093AB
:10ECE0000DF10A020DF10B030DF1090105A88DF8D4
:10ECF000146000F0D7FE9DF90900FEF74FF960702F
:10ED000004A801F01BF8B0B9049A0F2A0DD8637853
:10ED10009A420AD81544AB42A3EB02012CBF002053
:10ED200001202170C0000AB070BD002323700820AC
:10ED3000F9E70320F7E71320F5E700BFD42300200D
:10ED4000982900201FB50446002800F010810378A0
:10ED5000412B00F20781DFE813F0420049004D002B
:10ED60005100550059005E0005010501050105012E
:10ED70000501050105010501650069006D007800C8
:10ED80007F00820085008A0088008C00900093003C
:10ED9000960099009C009F00AE00B200BA00B60039
:10EDA000BE00C100C500CE00CA00CC000501D200E3
:10EDB0000501050105010501050105010501050123
:10EDC0000501050105010501050105010501DA003F
:10EDD000DE00E200E700EB00EF00F300FC00664B12
:10EDE00093F818312371002004B010BD624B93F8E2
:10EDF0003031F7E7406803F08FFBF4E7406803F039
:10EE0000D1FBF0E75C4B93F81A31EBE75A4BD3F8A0
:10EE1000E0306360E7E7584B011D93F8300103F0E1
:10EE2000D9FBE0E7544B93F81931DBE7524B93F8E9
:10EE30008C30D7E71C238DF808304F4B02A993F88C
:10EE4000480001F021FD6060CDE74C4B043493E8AD
:10EE5000030084E80300C6E7494B0434F7E7494B55
:10EE60000434F4E7484B0434F1E71A23E3E71923A9
:10EE7000E1E7414B93F86830B4E73F4B5B6DC8E77F
:10EE80003D4B9B6DC5E73C4BDB6DC2E73A4B1B6EC0
:10EE9000BFE7394B5B6EBCE702238DF80830364B79
:10EEA00002A993F87C2093F848008DF80A2001F01D
:10EEB000EBFC207197E7304B93F8DD3092E72E4B57
:10EEC00093F839308EE72C4B93F8DC308AE72A4BE5
:10EED00093F8383086E7284BDB6C9AE7264B93F89B
:10EEE00050307FE7244BD3F8843063607BE7224BBC
:10EEF0008FE7264B8DE7204BD3F8CC30F5E71E4B40
:10EF0000D3F82C31436001F04DFDA0606BE71A4B44
:10EF1000D3F890307DE7184B93F81F3162E7164B1A
:10EF2000B3F88830A3805EE7134BB3F88A30F9E773
:10EF3000114BB3F8D030F5E70F4BB3F8D230F1E70F
:10EF40000D4B93F848200AB1062A12D1B3F8A03528
:10EF5000E8E7094B93F848200AB1062A09D1D3F80B
:10EF6000A43556E704B0BDE8104000F021BE0320F0
:10EF70003AE7182038E700BFD423002040240020BF
:10EF8000882400204824002090240020101E002007
:10EF90007FB5044610B9032004B070BDA34DD5F869
:10EFA00040339A0700F16F820278412A00F26882AA
:10EFB000DFE812F04200470055005B005F0064008C
:10EFC00069007600810087008D00930099009F0002
:10EFD000A500AB00B5006602BA00DC00EF00160128
:10EFE0003801290142014B014F01530157015B01D7
:10EFF00066025F01710199018701AB01B101B8019E
:10F00000BD01C2016602280266026602660266024D
:10F0100066026602660266026602660266026602B0
:10F020006602660266026602340239023E0243024A
:10F0300048024D0252025C020079FEF773FA30B1C9
:10F04000AAE70379022BA6D0794A82F8303195F8E5
:10F05000913443F0200385F8913400209CE7406808
:10F0600003F04CFA0028F2D095E7406803F08AFAE2
:10F07000F8E76F4B027983F81A21E8E76C4B426896
:10F08000C3F8E020E3E76A4E416896F8300103F0E8
:10F0900097FA00287FF47FAF6368C6F8E430D6E7BC
:10F0A000416800293FF477AF002001F0DDF9002826
:10F0B000CDD0112070E7416800293FF46CAF0120EA
:10F0C000F3E7416800293FF466AF0820EDE74168A7
:10F0D00000293FF460AF0920E7E7416800293FF4C9
:10F0E0005AAF0C20E1E7416800293FF454AF0D20EE
:10F0F000DBE7416800293FF44EAF0E20D5E74168B9
:10F1000000293FF448AF0F20CFE74A4C484B007925
:10F1100083F81901A36D9847E36A984797E7444B32
:10F12000027983F88C2092E7414E037A8DF80430FF
:10F1300096F8480096F87D308DF80530072201A931
:10F1400001F0B5FB00283FF426AF636896F848004D
:10F150000193002201A901F0AAFB00283FF41BAF94
:10F160006C36D4E9010186E8030070E7304E037A7B
:10F170008DF8043096F8480096F87D308DF805300B
:10F18000072201A901F093FB00283FF404AFB43635
:10F19000E7E7274E037A8DF8043096F8480096F892
:10F1A0007D308DF80530072201A901F080FB002891
:10F1B0003FF4F1AED4E9010106F1740383E80300E2
:10F1C00096F81831022B7FF442AF96F83031002BBD
:10F1D0003FF43DAF174BDB6A9847FEF775F936E70A
:10F1E000134E037A8DF8043096F8480096F87D3077
:10F1F0008DF80530072201A901F059FB00283FF4E2
:10F20000CAAEBC36ADE74368029301238DF80C30DB
:10F21000074B02A993F8480001F056FB00287FF441
:10F2200016AFB8E6436802930023EFE79829002061
:10F23000D42300206078030803795A1E0E2A3FF673
:10F24000AAAE934A82F8683001E7914B42685A654A
:10F25000FDE68F4B42689A65F9E68D4B4268DA65A8
:10F26000F5E68B4B42681A66F1E6894B42685A66AE
:10F27000EDE6874C037994F848008DF804300622B7
:10F2800001A901F014FB00283FF485AE9DF804307D
:10F2900084F8DD30DBE67E4C03798DF8043094F899
:10F2A000480094F87C308DF80630052201A901F061
:10F2B000FEFA00283FF46FAE9DF8043084F8393030
:10F2C000C5E6734C037994F848008DF804300A229F
:10F2D00001A901F0ECFA00283FF45DAE9DF804307E
:10F2E00084F8DC30B3E66A4C037994F848008DF872
:10F2F0000430092201A901F0DAFA00283FF44BAEEC
:10F300009DF8043084F83830A1E6614B4268C3F8B8
:10F310009420DA649BE65E4B027983F8982083F8A8
:10F32000502094E65A4B4268C3F884208FE6584B2D
:10F330004268C3F8CC208AE6012B40F0A480554CEB
:10F340002421204603F01CFA636A984201D017205A
:10F3500022E61C2104F1280003F012FA636C9842A3
:10F36000F5D14FF4807104F1480003F009FAD4F8A4
:10F3700048319842EBD1D42104F5A67003F000FA8D
:10F38000D4F820329842E2D1002104F5097003F04C
:10F39000F7F9D4F824329842D9D14FF4607104F5CA
:10F3A0000A7003F0EDF9D4F8A8359842CFD11421B2
:10F3B00004F2AC5003F0E4F9D4F8C0359842C6D159
:10F3C000334E2146304640F2C45203F0C3F9204682
:10F3D00040F2C452002103F0D1F995F81B3485F8AE
:10F3E000E833736FC5F8EC3396F87D3085F8F83361
:10F3F00040F20123A5F8FA33274B96F819019B6DCB
:10F40000984724E68379012B3FF6C5AD204B42682F
:10F410004068C3F82C2100F0BDFE48E61C4B426852
:10F42000C3F8902013E61A4B027983F81F210EE6E9
:10F43000174B8288A3F8882009E6154B8288A3F829
:10F440008A2004E6124B8288A3F8D020FFE5104BF7
:10F450008288A3F8D220FAE50D4B93F848200AB130
:10F46000062A12D1A288A3F8A025F0E5084B93F84C
:10F4700048200AB1062A08D16268C3F8A425E6E547
:10F4800000F098FBDBE5012086E5182084E500BF4D
:10F49000D4230020101E0020607803082DE9F043DB
:10F4A00087B00023ADF800300646002800F0EE805B
:10F4B0000361FEF747FD20B10124204607B0BDE8F7
:10F4C000F08300F065FD0028F6D100F05BFD0146F9
:10F4D00018B96F48142203F051F96E4D95F8913424
:10F4E000012243F0040385F8552485F891343378DC
:10F4F0008DF804300021013B8DF80520ADF8061091
:10F500000C2B00F2BB80DFE803F007B9B9B97982B0
:10F51000B9B990B9AD9AA900D5F8407317F0200792
:10F52000CAD196F80480B8F1020F46D1DFF868819D
:10F530005A4CFEF763F896F9051098F848003A46D9
:10F5400001F00FFA88F83900B37988F83830384676
:10F5500007238DF80530FDF7E5FFFF2304F58670DE
:10F56000A5F80C31C5F8084185F8047103F01AF8C4
:10F5700004F58A7002F0D0FF3846FDF72DFE0446F0
:10F58000002839D096F9051098F84800012201F0BA
:10F59000E8F988F83900D5F894343361002C71D03B
:10F5A00000F0F0FC002888D195F8913485F81A0411
:10F5B00060F3820385F891347FE7B8F1010F4FF0D3
:10F5C0000204E8D1DFF8D0908DF8144099F8480093
:10F5D00089F81D7102A901F065F9337989F8303194
:10F5E0008DF805708DF80680FDF7C4FC95F8913410
:10F5F00043F0100385F891340024CCE700226946DB
:10F60000022000F0F3FA0028F6D01324C3E7244BBD
:10F61000B288DB6B96F90C10B0689847D5F8403388
:10F6200043F00203C5F84033E6E702A90D2000F0DD
:10F6300053FB0028E0D0002269460D20E1E7164B7D
:10F6400093F81831D3B9347904F0070000F0ABFA1D
:10F650008DF80040012269461020D2E70022694659
:10F660001220CEE78DF8072000F08EFA044638B954
:10F6700000F087FA204600F089FABDE702248AE705
:10F68000012488E701A800F0D1FB16E7032414E762
:10F69000EC2D002098290020D42300209A29002056
:10F6A000607803082DE9F04F99B08046059118B9AC
:10F6B000032019B0BDE8F08F00230361FEF742FC80
:10F6C0000446002840F0A58046460FCE0EAD0FC57B
:10F6D0001422524898F800A0B8F80C7098F90EB0AF
:10F6E0004F4E214603F04AF84E4B012283F8412445
:10F6F00096F83021022A25460BD196F81821022AC5
:10F7000007D196F81E2122B9BAF1010F38BF4FF088
:10F71000010ABAF1010F2BD0BAF1030F2AD0BAF1C6
:10F72000000F33D102229DF83C30DDF84090029367
:10F7300062F34715012496F87C108DF832100222EE
:10F740000CA996F848008DF8302001F09DF896F845
:10F750001A3196F830C196F81D1140B2002B63D0D3
:10F76000BCF1010F57D1002955D1002C61D153E0D4
:10F770000422D8E70023DDF83C90BDF840709DF9E5
:10F7800042B0029365F01F050124D4E74FF0000B4F
:10F79000D946CDF808B0CEE74FF0010084F81A043E
:10F7A000D2E005F29A420BA900F0D4FA002800F04A
:10F7B00015811320049B33871A4B002283F81A24E7
:10F7C00023E105F29A452A460BA900F0C3FA002866
:10F7D000EFD10B9B84F82801C4F82C5184F8303108
:10F7E000FCE0B9F1000F00F0F980002A00F0F6808B
:10F7F0004946E01C02F0AEFF94F837320133238013
:10F80000ECE01220D6E70220D4E70720D4E713204B
:10F81000D2E701204DE7FCB90220F6E0D82D002008
:10F82000D423002098290020002CF5D05845B8BFDB
:10F83000584696F87C308DF82000052296F848004E
:10F840008DF8223008A901F032F800283FF430AFDB
:10F850009DF8203086F839306F4A704BD2F8980402
:10F86000D3F8904038B105F053FA6C4B84423CBF5A
:10F87000002283F83A20198F1A8F93F830010491EF
:10F88000996A099152BA0028BFD093F81B0100B9B8
:10F89000186393F81801ADF85820013893F87C20CC
:10F8A00093F81A411491D0F1000BD3F888108DF819
:10F8B0005B204BEB000B93F8482093F83A0093F849
:10F8C00068308DF85A3009AB0093554B03904FF0D8
:10F8D00001008DF84C0015918DF85C20A3F12F01EB
:10F8E000A3F1300213A88DF84D4000F0DBF8039B24
:10F8F0004FEA0B1B4BEA431B00264BEA801B4BEAEB
:10F90000C413B145444C039308BF37463A464946B1
:10F9100004F59C70CDE90A669B46268084F81A643B
:10F9200002F018FFE9B2A570C5F34215FAB2042D32
:10F930003A4E039B84F837223FF42EAF072D3FF455
:10F9400050AF022D7FF45FAF364D84F80D110420C7
:10F95000029984F80401FF2084F80C0184F828112E
:10F9600084F81431D6F8E410C4F8085105F59B73F7
:10F970000AA8C4F8101184F83021C4F82C3100F022
:10F9800011FC00287FF43DAF0A9BA4F844040BA8A7
:10F99000A4F81631C4F84C3400F0D0F900287FF4F4
:10F9A00008AF0B9BD3B196F93900FDF7F7FA94F83D
:10F9B0003732002B3FF405AF0B9B0F2B3FF6F1AE18
:10F9C00005F58B720BA90F2000F0C4F900287FF415
:10F9D000F0AE0B9B63F3030B84F814B10598FDF7AD
:10F9E000FBFB00287FF4E6AE099B86F83A00B36281
:10F9F00000F080F900287FF40AAF94F8913484F87D
:10FA000040A443F0010384F89134034BD3F89434B9
:10FA1000C8F810304DE600BF98290020D4230020FC
:10FA20003C2400209A29002037B50B4D8DF80400A6
:10FA300004460F2295F8480001A900F038FF40B1B4
:10FA4000064A85F81C4192F8913443F0200382F86D
:10FA5000913403B030BD00BFD4230020982900208A
:10FA600010B5FFF7C1F8044688B90A4805F08AF9CD
:10FA7000094805F087F9094805F084F900F094F881
:10FA8000FDF7BCFD064BDB6A9847204610BD0124FC
:10FA9000FBE700BF002D0020182D0020302D002096
:10FAA000607803082DE9F04F8BB047780093149BE2
:10FAB00090F90C8090F90D6090F80EB08A4641687C
:10FAC000196004469146002F58D002238DF810305B
:10FAD00004A9C37B007C8DF8123000F0D5FEB4F889
:10FAE00008C0618943B26068984545466144B8BF23
:10FAF0001D46604534BF00270127884209D30A21EB
:10FB00008DF81010207C019304A900F0BDFE019B2C
:10FB100046B2B4F808C0608961680CEB400E7145CC
:10FB200019D3A1EB0C01B1FBF0FC00FB1C1191B946
:10FB3000984503DC2378CBB94FF0010B21238DF8D6
:10FB40001030207CE37B8DF8115004A98DF8123021
:10FB500000F09AFE45B2009B8AF80050384689F8BA
:10FB6000006083F800B00BB0BDE8F08F0223207C6A
:10FB70008DF8243006A900F095FEDDE74546EAE75A
:10FB80007047704770477047002070477047704754
:10FB90007047002070470020704700207047002009
:10FBA00070470020704770477047704702207047C9
:10FBB000022070470220704770470020704770474E
:10FBC00070470020704700207047704770477047AB
:10FBD00010B5054C4FF403722046002102F0CEFD13
:10FBE0000020C4E9000010BDB42E00202DE9F84328
:10FBF0008146904600293CD01F4C2023224604F128
:10FC0000100012F8017F6FBB8242FAD11B4E33689D
:10FC1000013403B93460736803B11C6000252560AA
:10FC2000C4F8088074601FFA88F284F80490601D9C
:10FC300002F090FDB9F1110F4FF0000398BF104D85
:10FC40006373D6F8083298BF25FA09F503F101036A
:10FC500098BF05F0010543442573C6F808323846BD
:10FC6000BDE8F883013B13F0FF030446C6D1022729
:10FC7000F5E70127F3E700BFBB2E0020B42E0020DC
:10FC80002007020010B518B3124A1368984204D135
:10FC900003681360002305E00B46002BFAD01968B7
:10FCA0008842F9D15168884208BF53600BB101689E
:10FCB0001960D2F808328168013B00245B1A0460A5
:10FCC0002146C2F80832102202F058FD204610BD2D
:10FCD0000120FCE7B42E0020054B1B6813B11A79F4
:10FCE0008242FAD1002B0B600CBF0320002070472A
:10FCF000B42E002010B5054B186800B910BD037B69
:10FD000004680BB9FFF7BEFF2046F6E7B42E0020CB
:10FD100038B5084B084C186800B938BD0379056838
:10FD2000112B05D824FA03F3DB0701D5FFF7AAFF4F
:10FD30002846F1E7B42E00202007020028B1044B2A
:10FD4000D3F808320360002070470120704700BFDD
:10FD5000B42E00202DE9F04107460E46154642B369
:10FD600039B3154B1C6800232CB93046FFF7E6FF6A
:10FD70000020BDE8F081A268F91A0132914215D342
:10FD80002279EA54581C22895FFA80F8611D55FADD
:10FD900080F002F0DFFCA368246898445FFA88F3DF
:10FDA000E2E720462568FFF76DFF2C46002CF8D1CE
:10FDB000DBE70120DDE700BFB42E00200238C0B22F
:10FDC00011289ABF014B185C002070477B71030813
:10FDD00030B50B4B93F820200446084672B1002141
:10FDE0001C330578A54208D001319842CDB214BF2A
:10FDF00004301038AA42F4D8002030BD1046FCE789
:10FE0000C030002010B5084C00232060142204F1FB
:10FE10000C00FF2184F82030C4E9010002F0AEFCA0
:10FE2000012384F8213010BDC030002010B50E4AE7
:10FE300092F82010042915D8936804781C7044782F
:10FE40005C70C478807898700131DC7082F8201082
:10FE500002F11C018B4214BF043302F10C039360C6
:10FE6000012010BD0020FCE7C0300020094B93F8B2
:10FE7000200068B15A6803F11C018A4200F1FF308A
:10FE800014BF043203F10C0283F820005A600120F1
:10FE9000704700BFC030002010B5074B93F82020FA
:10FEA0000446084632B15968FFF792FF10B10123AA
:10FEB0004470837010BD00BFC030002008B5064BF1
:10FEC00093F820202AB15968FFF782FF08B14078E3
:10FED00008BD0120FCE700BFC030002030B50A4A51
:10FEE00092F82010536882F8210061B191680124D2
:10FEF0001C32DD78587005B99C70934214BF0433EE
:10FF0000103B9942F5D130BDC030002008B5044BFC
:10FF10005968FFF75DFF003818BF012008BD00BF1A
:10FF2000C0300020F7B50422154E044600210DEB29
:10FF3000020096F8207002F021FC0025EBB29F42EF
:10FF400001D803B0F0BD7368197821705A786270D7
:10FF5000987838B1336820469B689847FFF786FF4A
:10FF60000135EBE7DB788DF804108DF805208DF86E
:10FF70000730FFF77BFF01A8FFF758FFF0E700BF4E
:10FF8000C0300020014B93F820007047C0300020A3
:10FF9000034B93F82000042894BF002001207047F1
:10FFA000C03000201FB50024CDE90244C41F8DF8E5
:10FFB00000408DF801100C0AADF80420090C120C59
:10FFC0008DF803108DF806208DF8073002461B0AC5
:10FFD000012168468DF802408DF8083002F029FAB8
:10FFE000002818BF0E2004B010BD2DE9F04188B0E4
:10FFF00090460D460F9A0746002847D0002401215D
:020000040801F1
:10000000CDE904448DF810109DF838108DF81510C6
:10001000ADF81630190CCDE900441B0ECDE90244B1
:100020008DF81930ADF81A20130C120E07948DF8C4
:1000300018108DF81C308DF81D20E3B21E01002D24
:10004000F6B203DC002008B0BDE8F08101331021D6
:100050008DF81F3042466B460DEB010002F07FF930
:100060000346A8B9102D28463E44A8BF1020694673
:10007000327811F801CB013382EA0C02984206F87B
:10008000012BF5DC103D2DB20134D6E70920DAE76B
:100090000E20D8E70138032815D8DFE800F0020861
:1000A0000C100A4B1B681B690B6000207047074B44
:1000B0001B685B69F8E7054B1B689B69F4E7034B1A
:1000C0001B68DB69F0E70520704700BFE4300020C3
:1000D0002DE9F041C4B00C464A9E17461D468046A5
:1000E000B8B3B1F5807F36D84FF4887200216846E6
:1000F00002F044FB492300934FF48073ADF80430C1
:100100002B0C8DF80830330CADF80650ADF80A60B2
:100110008DF80C3022460023414604A82D0E360EE1
:100120008DF80E308DF809508DF80D608DF80F4068
:1001300002F010FB04F110014B9A3B4689B268466D
:1001400002F0F7F810B1012818BF0E2044B0BDE846
:10015000F0810920FAE70D20F8E7000010B590B112
:100160000A4C28220021206002F008FB2368084A7C
:100170001A6000204FF0FF32C3E90302C3E90522F1
:10018000C3E9072210BD0820FCE700BFE4300020CF
:1001900000010101024B1B6818600020704700BF7E
:1001A000E430002030B1044B1B68DB68013303608E
:1001B0000020704709207047E430002013B5002369
:1001C0000C460193CAB101A9FFF764FF18B9019B5E
:1001D000591C02D1146002B010BD99B2611A0029F5
:1001E00001DD5C18F6E702D113600720F3E71B0C72
:1001F0001B0403F580331C44ECE70920EBE7000007
:1002000028B1044B1B681C3343620020704709204F
:10021000704700BFE43000201FB5044600B3002340
:1002200003A8039302F05CF9104ABDF80C30126881
:1002300020469380E38200F05EFA98B904F1180337
:10024000009321680123132202F068F860B9204668
:1002500000F051FA003818BF0120000104B010BDB1
:100260000920FBE71020F9E70E20F7E7E430002033
:10027000F0B5054687B01C4613B9092007B0F0BD9C
:100280002E4E3368DB68834255D894F82020002A2C
:100290000CBF08220922834205D3204600F05FFAF2
:1002A00068B11020EAE7002301900093A36894F856
:1002B0002810606AFFF799FE0028EED0DEE7237968
:1002C0002168B4F808C0A768043B9AB20029D4D0CA
:1002D000B2F5807F2DD8ADF80EC08DF817304FEAFB
:1002E000174C04F12C033F0E8DF8117000932F0C66
:1002F00008234FF0490EADF80C008DF814708DF8FE
:1003000016002F0E0DEB0300CDF808E08DF810C09D
:10031000ADF812508DF8157002F000F808B10E20FB
:10032000ACE7204600F01BFA0028BAD13368DD6044
:10033000A4E70D20A2E70620A0E700BFE4300020DC
:100340002DE9FF410A9D80460F4616461C46002DAA
:100350005AD0002303A910460393FFF79BFE18B160
:10036000062004B0BDE8F081039B9C4201D8013314
:10037000F6D1284600F064F9002847D1264B1A78B8
:10038000424503D01A79424542D10120AA68BA42B7
:1003900040D103EB8002EB6A92F801802979CDE924
:1003A00000430439927828683B4689B2FFF790FEF3
:1003B0000028D6D195F820300194002B4FF001038E
:1003C000009314BF4246082295F82810686A3B46FD
:1003D000FFF70BFE0028C4D1013E032EC1D8DFE891
:1003E00006F002070B0F0D4B1B681C611C62B8E77F
:1003F0000A4B1B685C61F9E7084B1B689C61F5E7D9
:10040000064B1B68DC61ACE70920AAE70F20A8E7D0
:100410000B20A6E70220A4E708040020E430002017
:100420001FB50B294FF00003CDE90033CDE90233AE
:100430000A4607D00C2914D00A2910D00A2005B08A
:100440005DF804FB012802D120238DF80030002143
:10045000684601F0EEFF002818BF0E20EFE73023BA
:10046000F3E70B21F4E7000038B5054601F0DCFFA7
:10047000044610B10E24204638BD002DFBD1094B97
:100480001B680B219878FFF7CBFF0028F2D10C21D5
:10049000FFF7C6FF0028EDD10A21FFF7C1FF0028B2
:1004A000E9D0E7E7E43000202DE9F04380468FB043
:1004B0000C461746002A6BD0002969D00025294632
:1004C0001D2206A805951DF091FF8DF81350344D9F
:1004D0002B680DF114099E88CDF804900DF11303DB
:1004E00002933B7900933B6832462146404601F037
:1004F000BCFF00284ED138683A79494602F02AF903
:10050000384600F04FF8002846D13C7AFA79BB799A
:10051000240444EA02241C432B689A6894423DD97F
:100520009C609DF813000B21FFF77AFF034658BB30
:100530000C21FFF775FF034630BB0A21FFF770FF60
:10054000034608BB7B7ABA7AFF7A3F0447EA022760
:100550001F433A46334621460920FFF723FD034651
:1005600090B933463A4621460820FFF71BFD034663
:1005700050B92A689DF8131091700021D1604FF096
:10058000FF31C2E90411916118460FB0BDE8F08354
:100590000923F9E70E23F7E70F23F5E70323F3E732
:1005A000E430002010B50446002845D00168002939
:1005B00042D011F8013B43710322063002F0CAF821
:1005C0002046032250F8091B043102F0C3F82168C9
:1005D000CB79E3600A7A43EA0223E3604A7A43EA8A
:1005E0000243E3608A7A43EA0263E360CB7A2374CE
:1005F0000B7B63742379212B1AD110220D3104F166
:10060000120002F0A7F81D222168501C8B5C636267
:10061000085C43EA0023901C6362085C033243EAEF
:10062000004363628A5C43EA02636362002010BD98
:10063000112B03DC0D22E7E70220F8E70120F6E7A3
:1006400010B50446002854D00168002951D00B7819
:1006500043714B7883608A7843EA02238360CA78C7
:1006600043EA024383600A7943EA026383604B7979
:1006700003738B79C381CA7943EA0223027BC38166
:1006800002F00F020831103002F064F8237B0022E0
:1006900003F00F0384F8202084F82820227903F146
:1006A0000800111A04290DDD21680933043AD21A11
:1006B000085C84F82000D2B2606A84F828201944CB
:1006C00002F048F8237922681A44002012F8043C0A
:1006D000E36212F8031C43EA0123E36212F8021CEE
:1006E00043EA0143E36212F8012C43EA0263E36246
:1006F00010BD0220FCE710B5044660B3036853B395
:100700000279162A29D942791A700146082251F82D
:10071000060B013002F028F82146082251F80E0B92
:10072000093002F021F82368E28A5A74E38A2268C9
:100730001B0A93742368A269DA74A36922681B0AEE
:1007400013752368628B5A752368E27E9A751723A6
:100750002371002010BD0120FCE70220FAE738B524
:100760000446002863D00168002960D0037B90F81C
:10077000282003F00F03002A57D1083320790432D0
:100780001344984255D363790B702368A2685A705A
:10079000A36822681B0A937023686289DA70236851
:1007A000E27A1A712368227B5A712368E2899A716E
:1007B000E38922681B0A2146D371227B51F8100B72
:1007C00002F00F02083001F0C5FF237B94F82820C7
:1007D00003F00F0303F108052AB1226894F82010F2
:1007E000515503F10905206894F82820616A2844CE
:1007F00001F0B0FF94F828302268E16A2B44D1540C
:100800005A1CE16A206892B2090A81549A1C216834
:10081000E08D92B28854DA1C216894F82F0092B2CD
:10082000043388542371002038BD0933A6E7012022
:10083000FAE70220F8E70000024B1A8810431880FC
:10084000704700BFE830002008B5074B1B883BB15C
:10085000FEF7CAF9002814BF6FF00200002008BD9F
:100860006FF00100FBE700BFE830002010B5034B3C
:1008700000241C80FEF7AEF9204610BDE8300020B1
:10088000B0FA80F04009704782B018B9084602B04B
:1008900000F0CAB8002002B0704710B9084600F056
:1008A00079B9704710B9084600F090B9704703460F
:1008B000084611460BB900F0DDB90020704710B9A9
:1008C000084600F039BD704710B9084600F0FEB97F
:1008D0000020704710B40446084611461A46019B92
:1008E00014B910BC00F00CBA10BC7047034608469F
:1008F00011460BB900F036BA0020704710B4044618
:10090000084611461A4614B910BC00F0A3BA0020DC
:1009100010BC704730B40546084611461A46DDE95A
:1009200002341DB9029430BC00F022BB002030BC60
:10093000704710B9084600F0D3BB0020704710B9CB
:10094000084600F037BD0020704710B9084600F097
:10095000E2BB0020704710B9084600F0DFBB002062
:1009600070470346084611460BB900F0F9BB00205A
:10097000704710B40446084611461A46019B14B944
:1009800010BC00F0EFBB092010BC704710B4044647
:10099000084611461A4614B910BC00F02DBDC8B265
:1009A00010BC70470048704701000102064B10B5AB
:1009B0001B6A0446984730B10448054B20449842CE
:1009C0008CBF0020012010BD60780308403576C937
:1009D000405DC600F0B5114B85B00C4610491F565E
:1009E000054601F017F80F4BE4B25E6A072D4FF091
:1009F0000103CDE9024301460AD105220023CDE9D6
:100A000000234FF47A727A431846B04705B0F0BD20
:100A100008220020CDE900203A46F5E74872030895
:100A200028720308607803081FB500230093037839
:100A3000013B372B21D8DFE803F01C242020201EA7
:100A4000202020204143454E2055585B5E616420A4
:100A50006C1E6E73787A7D207F83262020202020D4
:100A6000202020202020202085878C2020858C207D
:100A70008E92C3780BB102230093009805B05DF805
:100A800004FB8378F6E743788DF8043007238DF86C
:100A900005308378003B18BF01235B008DF80630DA
:100AA00010238DF80730314B1B6801A803F55872ED
:100AB000CDE9022300F08EFF0090DEE74023DBE764
:100AC0002023D9E7827890F9013012B9284AD35C03
:100AD000D2E7284AFBE7827890F90130002AF8D162
:100AE000254AF4E740F6B833C6E74FF47A73C3E714
:100AF0004FF4FA63C0E741F28833BDE741F2707307
:100B0000BAE71E484FF47A7101F008FE00F5FA606A
:100B1000D2E71B4BB0E7154B1B6803F55873ABE7E7
:100B2000124B1B6803F55B73A6E71023A4E70F4B7A
:100B30001B68A1E701239FE74FF0834300939CE7E5
:100B4000104BFBE7104B97E740F21113ADF8003064
:100B500093E7032390E790F901300C4AB7E70C497B
:100B600090F9010000F056FFA6E700BFF03000202A
:100B70001D7203080D7203081572030818FCFFFFAD
:100B800000EA06379A99094040F709374872030886
:100B90002872030837B50B4B02781B680C2101FB48
:100BA00002335B7A03EB4304074B1D680369009330
:100BB000C3684278816805EBC40000F0A7FC03B06D
:100BC00030BD00BFF0300020EC30002030B587B0E1
:100BD000027B6423ADF80030012A4FF00003CDE919
:100BE0000133CDE903338DF802308DF8143028D06D
:100BF000022A2FD01ABB03680BB34368FBB11A4C0F
:100C000080682360194B18226946186001F0A2FD24
:100C1000174B246893E807000C3384E8070093E837
:100C2000070004F10C05032385E80700A4F86C33E2
:100C3000012204F55B7104F5587000F058FC07B010
:100C400030BD094908684360036100F55B7100F538
:100C50005870F2E7044B1B68B3F86023B3F86C13C9
:100C60000A43A3F86023EAE7F0300020EC300020CC
:100C7000101A030808B503460A2924D8DFE801F052
:100C800006232323230B161B23212100BDE8084044
:100C90000068FFF78BBE90F900009978072271B9C0
:100CA00000F0E5FB003818BF012008BD052293F9CC
:100CB00000000021F4E790F900005978EEE70221E6
:100CC000EEE70722F3E70020EFE7000008B502791E
:100CD0001AB1012A0BD0002008BD084B01681B681F
:100CE000012203F5587000F002FC0120F4E7034BE9
:100CF00001681B6803F55B70F5E700BFF03000206A
:100D0000F7B50728144D1C46A8BF072058700E469B
:100D10002946174600F07EFE94F90130A070072B9B
:100D200013D1322000F076FD0C4BDB6D0546984761
:100D300004F10C0208340346019200943A4631460D
:100D4000284600F06CFD03B0F0BD054A55F82310AD
:100D5000D05C00F057FDE7E72872030860780308CD
:100D6000487203082DE9F04F344F90F901607B6819
:100D7000D0F804908BB00446884698470546002872
:100D800059D1E37C73B92E4A2378126803EB4303ED
:100D9000990002EB8303D3F80490B9F1000F01D15D
:100DA00052F80190274B484613F906B0FB68984764
:100DB000A37C2289D7F818A00993072E28D10023F5
:100DC0000121CDE90223204A0693CDE90431CDE982
:100DD00007330521CDE900214FF47A7202FB0BF2B3
:100DE0004CF250311846D047637C13B3174B995DD2
:100DF0007B6D0D31C9B228469847E07C32464946A2
:100E000000F01AFE88F8006001200BB0BDE8F08FFA
:100E1000002101250823CDE90013CDE90715CDE90F
:100E20000511CDE903110292A1782B465A462846B6
:100E3000D9E7074BDBE70020E7E700BF607803084E
:100E4000F030002048720308854501001572030840
:100E50001D7203082DE9F04F8DB090F90130DFF8D5
:100E6000FCA0DFF8FC90CDE90A123E4A12F903B06B
:100E70000278DAF800300C2505FB02333A4A5B7A37
:100E8000126803EB430302EBC303044693F9021019
:100E900090F9020000F0B9FD3449064694F90100CA
:100EA00000F0B8FDA26861688046304600F0DFFCC3
:100EB0002178DAF80020D9F80C30694307465058F9
:100EC0009847D9F81C309C4694F901300025072B2F
:100ED0004FF47A63CDE90753CDE905552DD10123B0
:100EE000CDE903530523CDE901534FF47A7303FB96
:100EF0000BF300933946434646F2A812284667464C
:100F0000B8472378DAF800200C214B4394F90110FC
:100F1000D05800F0B3FDA18994F90100FFF75AFD04
:100F20000B9B217B1860D9F85430284698470A9BC0
:100F300001201E700DB0BDE8F08F01200823CDE91F
:100F40000350CDE901032A46CDF800B0654643467B
:100F50003946A84701200546D3E700BFF0300020FE
:100F60006078030848720308EC30002028720308F8
:100F70002DE9F04F8FB0002405468A4691469846E9
:100F80000494ADF81440ADF8024007264FF0010B71
:100F90002B7AA34206D9686804A9204400F0CAFB52
:100FA00000285DD102238DF8083002A86B7A8DF8F5
:100FB0000A30FFF739FDAB7A8DF81D309DF81130FE
:100FC0008DF81E309DF812308DF81F309DF81030CE
:100FD0008DF82030EB7A8DF821302B7B8DF8223084
:100FE0006B7B8DF8233010238DF81C608DF8243036
:100FF0003A4E8DF82C000DF102030A930723326854
:101000008DF82D30ADF834302B680C9206930DF12D
:10101000120204AB0DF1110106A800F0A5FB072890
:1010200005460BD130680C22002100F5587001F004
:10103000A5FB3368BDF80220A3F860239DF81130AA
:101040008AF800309DF8123089F800309DF8103091
:1010500088F80030189B28461C700FB0BDE8F08F50
:101060009DF81330BDF81470ADF802702044C4B27E
:10107000F3B917B3194A00201168072602464FF04A
:101080000C0C062B1BD10CFB00FE51F80EE0BEF140
:10109000000F04D00BFA00F23A4397B2012201305C
:1010A0001028EED1002A3FF473AFADF802706FE75D
:1010B0005A1E042A01D9062BDCD0062668E747FA17
:1010C00000FE1EF0010FEAD00CFB00FE51F80EE00E
:1010D000BEF1000F08BF0626E1E700BFF030002098
:1010E00038B505464068FFF761FC0722841D0021E2
:1010F00095F90000E4B200F0BAF908B904F0FD0473
:1011000095F901000722002100F0B1F908B904F0B7
:10111000FB04204638BD00207047000010B503785E
:101120000F2B044618D84068FFF740FC22780B4983
:1011300002EB42020968831C01EB820051F8222075
:10114000DBB21AB903F0FD0358B210BD032B06BF82
:10115000626842600223F7E70020F6E7F0300020E3
:10116000022070472DE9F0413A4D0446286896B0B8
:101170000E46904600211F460122032300F55870B9
:10118000CDE90411CDE906118DF80C108DF80D1084
:10119000ADF80E3000F08DF930B92A68B2F860333E
:1011A00043F00303A2F860332A68637A8DF8203095
:1011B00002F55871CDE90912274A94F908301268EE
:1011C0000B921022ADF830200DF10E020D92226824
:1011D0000E9262680F92D4E90301A27A8DF8402042
:1011E00001228DF8412011AA82E80300227DE18AC4
:1011F0008DF8213018468DF84C20FFF7EBFB08AB3B
:1012000015930DF10D0314900093CDF8048003ABFA
:1012100004AA39460EA800F099FB044678B99DF857
:101220000C10013901F07AFA00F158030DEB0300BC
:1012300010F8483C3370204616B0BDE8F0810C2809
:1012400001BF2A68B2F8603343F00303A2F86033A9
:10125000F1E700BFF0300020EC300020F8B506794F
:10126000012E054648D90F2E48D80368187A40F356
:1012700003000722002140B200F0F9F82B68044671
:10128000187A40F303100722002140B200F0EFF873
:10129000B8B1B4FA84F4640929680B7A086843F396
:1012A000030243F303135BB252B29A42C8BF012454
:1012B000FFF77CFB80F00103DBB224B10533D8B229
:1012C000F8BD0124E8E7DBB90E4F29683B6806EB5F
:1012D000460003EB80000C2201F03CFA3A680C2334
:1012E00003FB062320465C72B2F860130123B3406F
:1012F0000B43A2F86033E3E70620E1E70320DFE7D2
:101300000420DDE7F030002010B4017801290ED967
:10131000084B18680C234B43C4180022C250C4E980
:10132000012200F5587010BC102200F0A9B800206E
:1013300010BC7047F03000202DE9F04186B05023FA
:101340008DF81430037A102B074630D14368DD7BCB
:101350006DBB0224A8466426062C14D87A68535D17
:1013600003932A44517843EA01230393927843EA92
:1013700002437343CDE9033863B968468DF80040F2
:10138000FFF7C2FF0DE0CDF80C808DF81480CDF88A
:101390001080F2E703AB01A801938DF80840FFF736
:1013A0005DFF0134E4B2102C05F10305D4D106B081
:1013B000BDE8F0811FB502680379116849B901A839
:1013C0008DF80430FFF7A0FF78B1032005B05DF879
:1013D00004FB02A802928DF80C30FFF73FFF0428AF
:1013E00005D0052805D00028EFD00020EEE7022028
:1013F000ECE70120EAE70000C90020B9034B0B44E9
:101400009856C0B27047024BF9E700BFCD71030890
:101410008D710308F0B59A42069D03DB9DF91430E7
:101420009A4220DD0020F0BD03EB430331F814C0E5
:1014300005EB830300264CFA06F7FF0707D51F7A52
:1014400007F00F0E964502DCB2EB171F0DDD0136DB
:10145000102E03F10C03EED10134E4B22301DBB210
:101460009842E1D8DEE70024F8E70120DBE7884274
:1014700004DB9042CCBF0020012070470020704761
:1014800010B51409B4EB111F03464FEA11100ED327
:1014900091420CD202B201F00F0133F81240012048
:1014A00000FA01F124EA010123F8121010BD002016
:1014B000FCE7F0B528B100EB41050127002091427F
:1014C00000D3F0BD002435F802CB234607FA04F61A
:1014D00036EA0C0608BF013304F1010408BFDBB291
:1014E000102CF3D118440131C0B2C9B2E7E710B5EE
:1014F00000B149B910BD31F8134020F81340013351
:10150000DCB2A242F7D8F5E70023F9E782B030B5A4
:1015100004880493D2B9B3F5616F15D349F6AF25AA
:1015200042F21072AB4298BF4FF47A72944238BFC5
:1015300014466143BDE83040C3688B428CBF5B1AE0
:101540000023C36002B070476422EFE7012C38BF6C
:101550000124EEE72DE9F04F8FB01546199F039354
:101560009DF8603007930C46804603F0C7FB6A4A3B
:101570000590A7F5F633303BB3FBF2F3534303F585
:10158000F63B0493182313FB05430BF1300B069332
:1015900000254FF0FF3A069B9C4207D1002D14BF57
:1015A00050464FF0FF300FB0BDE8F08FBDF9683006
:1015B000ADF82430099919973846089703F02EFBA7
:1015C0002688B8F1000F5FD1B7F5616F5AD349F69D
:1015D000AF2242F21073974298BF4FF47A739E4243
:1015E00038BF1E46642E59D1DFF83091A060A16843
:1015F0000CA803F035FB0D9B0093DDE908120C9B52
:101600000AA803F08CFA039A0A9B0AB9079A2AB12E
:1016100022694A4502D1424A93420ED9414BC4F84D
:101620000C909F4209D90023ADF82C300B99CDF8CE
:1016300028B0584603F0F2FAA060606808B9C4F810
:101640000C90C4F81090B8F1000F04D003F060FBC8
:10165000E3680344E360D4E903329342059B88BF07
:10166000E26063601B9BE1687343994204D2039874
:10167000E8B9B8F1000F1AD001231D442375EDB26B
:10168000183488E76423AAE7039B0BB9234BE36074
:10169000012EDFF8889038BF0126CEE7B6F57A7FB5
:1016A0000ABFDFF88490DFF88490A0609FE70020F5
:1016B0009342207506D85B1A9A4505F1010528BFAB
:1016C0009A46EDB2B8F1000FDAD1642E184AADF89F
:1016D0002C801DD049F6B023B6F57A7F18BF13468B
:1016E000974281BF049A02F5A83202F5C0729B1896
:1016F0000A931A9B00930AAE96E80600199B30469F
:1017000003F00DFA96E8030003F088FA8246B7E783
:101710004FF46163E4E700BF8051010040771B0094
:101720007F5101002FEC010080A81201002E9302CE
:1017300030EC01000378032B14D1437803F00F023F
:101740001B098A704B7083788B80C27843EA02232E
:101750008B800379C3F3021203F00F03CA700B707E
:1017600005207047002070472DE9F3479A464379DA
:10177000057990F907609146044690F9062088465D
:10178000D3B190F90870002D37D00F2A1BD194F9EE
:1017900009200F2E27D194F90A00072D02D1002F1E
:1017A00008BF012788F8002089F8000028468AF839
:1017B000007002B0BDE8F08790F90B7090F9092035
:1017C00090F90A60DFE7A369019394F9153000935B
:1017D00094F914302169207BFFF71CFE0028D8D132
:1017E00005F0FD05D5E794F91D00B042D5DC94F96C
:1017F0001C30B34203DA05F0FB053046D2E7304631
:10180000CBE70000024B03FA00F0B0FBF1F07047A9
:1018100040420F004FF4FA53B3FBF0F0704730B57D
:101820004FF47A750C1F6A4300FB042252001EBF5E
:1018300000F1FF341219B2FBF0F2914238BF1146A9
:10184000039A1160820048431CBF013040084FF4E6
:101850007A71121A01FB1323002BCABF03F2E7337C
:1018600093FBF1F1B3FBF1F1049B196030BD38B586
:10187000400014460D46F0F79DFB01462846F0F760
:10188000E7FA2146F0F7E4FAEFF75EFF1EF0BCFE40
:10189000F0F762FA40B238BD2DE9F74F019300230B
:1018A0009C469E46048A1E01F6B2B44246D906EB17
:1018B00046054FEA4309AD000024476837F8097030
:1018C0002741FF0729D5876807EB050A7F5927B30A
:1018D000077837B9476927B137F809702741FF07FB
:1018E0001BD59AF8087090F901B047F303084FFA36
:1018F00088F8D84511DC47F303177FB25F450CDB4E
:101900009AF8097007EB4708C76807EBC8073F7DDF
:101910005FB90CF1010C5FFA8CFC0134102C05F15D
:101920000C05CAD10133DBB2BCE70EF1010706EBAF
:10193000040801F80E805FFA87FEEEE7019B82F84B
:1019400000E083F800C003B0BDE8F08F2DE9FF4749
:1019500004464068DDE90C671D468A46914603F05F
:10196000D7F923681B1A3B604FF00008012333703E
:1019700085F80080636813B12368834224D8D4F8C3
:101980001CC0CAF80080A3699CF800E00393D4E966
:10199000030101AB83E80300237D0093DCF80C1006
:1019A000237A627A7046FFF7D5FD334638602A46BF
:1019B000E0694946FFF770FF2B782BB1C7F800802C
:1019C000002004B0BDE8F0873378002B0CBF0C205A
:1019D0000B20F6E737B590F9002090F902509542B8
:1019E00004460FD0013A52B295420BD0A36801933E
:1019F00094F9013000936168E0782B46FFF70AFD07
:101A00000028EFD0104603B030BD8842B8BF08466A
:101A10007047000051F82000054B984205D0054B57
:101A2000C31A58425841400070470120704700BF18
:101A300090D0030020A1070005281FB50ED80C4B3D
:101A400053F820300093CDE901120A4B0122002106
:101A5000022002F06BFE05B05DF804FBCDE9001238
:101A6000054B01220021022002F060FEF3E700BFD7
:101A7000B8720308507203086F72030807B5054B6C
:101A8000CDE9000101220021022002F04FFE03B047
:101A90005DF804FB8B72030810B510220446002188
:101AA000F13000F06BFE0021C4F814112046F02242
:101AB000BDE8104000F062BE02460846102100F06A
:101AC000A5B92DE9F0430446D0F8140185B00E46BF
:101AD000154604F2011988B3C0F110089045474635
:101AE00028BF1746BAB2484400F034FED4F8143187
:101AF0003B440F2BC4F814312DD9A8452BD204F147
:101B0000F00304F5807113F8012F187C8B4282EAF0
:101B100000021A70F7D104F1F1081022414668461C
:101B200000F018FE22466946684600F0F1F91022DE
:101B30006946404600F00EFE3E44ED1B04F58078F9
:101B400004F1F107102D09D8AAB23146484600F039
:101B500001FEC4F8145105B0BDE8F08304F1F003B0
:101B6000711E13F8012F11F8010F434582EA00029C
:101B70001A70F6D110223946684600F0EBFD224675
:101B80006946684600F0C4F910226946384600F0FC
:101B9000E1FD1036103DD5E7F0B589B00C461022B6
:101BA00000210546684600F0E9FD22466946684680
:101BB00000F0AEF99DF90030002B6A464FF00001AD
:101BC00043DA137812F8010F01315B0043EAD013B6
:101BD0000F2902F8013CF4D19DF80F305B0083F02F
:101BE0008703D4F81401DBB210288DF80F303BD1F5
:101BF00004F58073694604F5887013F8016F11F8D5
:101C0000012B984282EA06021A70F6D104F1F00321
